BL51 BANKED LINKER/LOCATER V6.22                                                        02/06/2025  15:28:46  PAGE 1


BL51 BANKED LINKER/LOCATER V6.22, INVOKED BY:
D:\TOOL\KEIL\C51\BIN\BL51.EXE .\output\Main.obj, .\output\Initial.obj, .\output\InterruptApp.obj, .\output\Led.obj, .\ou
>> tput\KeyApp.obj, .\output\LowPower.obj, .\output\UartApp.obj, .\output\Memory.obj, .\output\AFE.obj, .\output\Balance
>> .obj, .\output\Calculate.obj, .\output\Calibrate.obj, .\output\ChargerLoad.obj, .\output\ExtE2PRom.obj, .\output\Inte
>> rrupt.obj, .\output\KeyScan.obj, .\output\McuFlash.obj, .\output\McuLib.obj, .\output\MosCtrl.obj, .\output\PorSelfTe
>> st.obj, .\output\Protect.obj, .\output\RTC.obj, .\output\TWI.obj, .\output\Uart.obj, .\output\Thermistor.obj, .\outpu
>> t\TwiIO.obj, .\output\STARTUP.obj, .\output\GasGaugeInter_V4_13.obj, .\code_gasguage\GasGaugeV4_13.LIB, .\output\Boot
>> App.obj, .\output\BootIAP.obj TO .\output\MCUCore_Load REGFILE (.\output\MCUCore_Load.ORC) PRINT (.\output\MCUCore_Lo
>> ad.m51) RAMSIZE (256) DISABLEWARNING (16) CODE (0X0000-0XFBFF, ?CO?BOOTIAP (0X0000)) XDATA (0X0200-0X0AFE)


MEMORY MODEL: LARGE WITH FLOATING POINT ARITHMETIC


INPUT MODULES INCLUDED:
  .\output\Main.obj (MAIN)
  .\output\Initial.obj (INITIAL)
  .\output\InterruptApp.obj (INTERRUPTAPP)
  .\output\Led.obj (LED)
  .\output\KeyApp.obj (KEYAPP)
  .\output\LowPower.obj (LOWPOWER)
  .\output\UartApp.obj (UARTAPP)
  .\output\Memory.obj (MEMORY)
  .\output\AFE.obj (AFE)
  .\output\Balance.obj (BALANCE)
  .\output\Calculate.obj (CALCULATE)
  .\output\Calibrate.obj (CALIBRATE)
  .\output\ChargerLoad.obj (CHARGERLOAD)
  .\output\ExtE2PRom.obj (EXTE2PROM)
  .\output\Interrupt.obj (INTERRUPT)
  .\output\KeyScan.obj (KEYSCAN)
  .\output\McuFlash.obj (MCUFLASH)
  .\output\McuLib.obj (MCULIB)
  .\output\MosCtrl.obj (MOSCTRL)
  .\output\PorSelfTest.obj (PORSELFTEST)
  .\output\Protect.obj (PROTECT)
  .\output\RTC.obj (RTC)
  .\output\TWI.obj (TWI)
  .\output\Uart.obj (UART)
  .\output\Thermistor.obj (THERMISTOR)
  .\output\TwiIO.obj (TWIIO)
  .\output\STARTUP.obj (?C_STARTUP)
  .\output\GasGaugeInter_V4_13.obj (GASGAUGEINTER_V4_13)
  .\code_gasguage\GasGaugeV4_13.LIB (GASGAUGEV4_12)
  .\output\BootApp.obj (BOOTAPP)
  .\output\BootIAP.obj (BOOTIAP)
  D:\TOOL\KEIL\C51\LIB\C51FPL.LIB (?C?FPADD)
  D:\TOOL\KEIL\C51\LIB\C51FPL.LIB (?C?FPMUL)
  D:\TOOL\KEIL\C51\LIB\C51FPL.LIB (?C?FPDIV)
  D:\TOOL\KEIL\C51\LIB\C51FPL.LIB (?C?FCAST)
  D:\TOOL\KEIL\C51\LIB\C51FPL.LIB (?C?CASTF)
  D:\TOOL\KEIL\C51\LIB\C51FPL.LIB (PRINTF)
  D:\TOOL\KEIL\C51\LIB\C51FPL.LIB (?C?FPGETOPN)
  D:\TOOL\KEIL\C51\LIB\C51FPL.LIB (?C?FPROUND)
  D:\TOOL\KEIL\C51\LIB\C51FPL.LIB (?C?FPCONVERT)
  D:\TOOL\KEIL\C51\LIB\C51FPL.LIB (?C?FTNPWR)
  D:\TOOL\KEIL\C51\LIB\C51L.LIB (?C?CLDPTR)
  D:\TOOL\KEIL\C51\LIB\C51L.LIB (?C?CLDOPTR)
BL51 BANKED LINKER/LOCATER V6.22                                                      02/06/2025  15:28:46  PAGE 2


  D:\TOOL\KEIL\C51\LIB\C51L.LIB (?C?CSTPTR)
  D:\TOOL\KEIL\C51\LIB\C51L.LIB (?C?IMUL)
  D:\TOOL\KEIL\C51\LIB\C51L.LIB (?C?UIDIV)
  D:\TOOL\KEIL\C51\LIB\C51L.LIB (?C?IILDX)
  D:\TOOL\KEIL\C51\LIB\C51L.LIB (?C?LADD)
  D:\TOOL\KEIL\C51\LIB\C51L.LIB (?C?LSUB)
  D:\TOOL\KEIL\C51\LIB\C51L.LIB (?C?LMUL)
  D:\TOOL\KEIL\C51\LIB\C51L.LIB (?C?ULDIV)
  D:\TOOL\KEIL\C51\LIB\C51L.LIB (?C?SLDIV)
  D:\TOOL\KEIL\C51\LIB\C51L.LIB (?C?LOR)
  D:\TOOL\KEIL\C51\LIB\C51L.LIB (?C?LNEG)
  D:\TOOL\KEIL\C51\LIB\C51L.LIB (?C?SLCMP)
  D:\TOOL\KEIL\C51\LIB\C51L.LIB (?C?ULCMP)
  D:\TOOL\KEIL\C51\LIB\C51L.LIB (?C?ULSHR)
  D:\TOOL\KEIL\C51\LIB\C51L.LIB (?C?SLSHR)
  D:\TOOL\KEIL\C51\LIB\C51L.LIB (?C?LSHL)
  D:\TOOL\KEIL\C51\LIB\C51L.LIB (?C?LLDIDATA)
  D:\TOOL\KEIL\C51\LIB\C51L.LIB (?C?LLDXDATA)
  D:\TOOL\KEIL\C51\LIB\C51L.LIB (?C?LLDIDATA0)
  D:\TOOL\KEIL\C51\LIB\C51L.LIB (?C?LLDXDATA0)
  D:\TOOL\KEIL\C51\LIB\C51L.LIB (?C?LILDXDATA)
  D:\TOOL\KEIL\C51\LIB\C51L.LIB (?C?LSTIDATA)
  D:\TOOL\KEIL\C51\LIB\C51L.LIB (?C?LSTXDATA)
  D:\TOOL\KEIL\C51\LIB\C51L.LIB (?C?LSTKIDATA)
  D:\TOOL\KEIL\C51\LIB\C51L.LIB (?C?LSTKXDATA)
  D:\TOOL\KEIL\C51\LIB\C51L.LIB (?C?OFFXADD)
  D:\TOOL\KEIL\C51\LIB\C51L.LIB (?C?PLDIXDATA)
  D:\TOOL\KEIL\C51\LIB\C51L.LIB (?C?PSTXDATA)
  D:\TOOL\KEIL\C51\LIB\C51L.LIB (?C?CCASE)
  D:\TOOL\KEIL\C51\LIB\C51L.LIB (?C?LIMUL)


LINK MAP OF MODULE:  .\output\MCUCore_Load (MAIN)


            TYPE    BASE      LENGTH    RELOCATION   SEGMENT NAME
            -----------------------------------------------------

            * * * * * * *   D A T A   M E M O R Y   * * * * * * *
            REG     0000H     0008H     ABSOLUTE     "REG BANK 0"
            DATA    0008H     0007H     UNIT         ?DT?KEYSCAN
            DATA    000FH     0006H     UNIT         ?DT?AFE
            DATA    0015H     0005H     UNIT         _DATA_GROUP_
            DATA    001AH     0004H     UNIT         ?DT?GASGAUGEINTER_V4_13
            IDATA   001EH     0001H     UNIT         ?ID?EXTE2PROM
                    001FH     0001H                  *** GAP ***
            DATA    0020H     0007H     BIT_ADDR     ?BA?MEMORY
            BIT     0027H.0   0001H.3   UNIT         ?BI?EXTE2PROM
            BIT     0028H.3   0001H.2   UNIT         ?BI?UARTAPP
            BIT     0029H.5   0001H.1   UNIT         _BIT_GROUP_
            BIT     002AH.6   0000H.6   UNIT         ?BI?GASGAUGEV4_12
            BIT     002BH.4   0000H.5   UNIT         ?BI?AFE
            BIT     002CH.1   0000H.5   UNIT         ?BI?BALANCE
            BIT     002CH.6   0000H.4   UNIT         ?BI?LOWPOWER
            BIT     002DH.2   0000H.4   UNIT         ?BI?CHARGERLOAD
            BIT     002DH.6   0000H.3   UNIT         ?BI?INTERRUPTAPP
            BIT     002EH.1   0000H.3   UNIT         ?BI?MCUFLASH
BL51 BANKED LINKER/LOCATER V6.22                                                      02/06/2025  15:28:46  PAGE 3


            BIT     002EH.4   0000H.2   UNIT         ?BI?LED
            BIT     002EH.6   0000H.2   UNIT         ?BI?MOSCTRL
            BIT     002FH.0   0000H.2   UNIT         ?BI?PROTECT
            BIT     002FH.2   0000H.2   UNIT         ?BI?RTC
            BIT     002FH.4   0000H.1   UNIT         ?BI?CALIBRATE
            BIT     002FH.5   0000H.1   UNIT         ?BI?KEYSCAN
            BIT     002FH.6   0000H.1   UNIT         ?BI?PORSELFTEST
                    002FH.7   0000H.1                *** GAP ***
            IDATA   0030H     000CH     UNIT         ?ID?GASGAUGEV4_12
                    003CH     0064H                  *** GAP ***
            IDATA   00A0H     0060H     ABSOLUTE     

            * * * * * * *  X D A T A   M E M O R Y  * * * * * * *
            XDATA   0000H     0002H     ABSOLUTE     
            XDATA   0002H     0014H     ABSOLUTE     
            XDATA   0016H     0004H     ABSOLUTE     
            XDATA   001AH     0004H     ABSOLUTE     
            XDATA   001EH     0004H     ABSOLUTE     
            XDATA   0022H     0002H     ABSOLUTE     
            XDATA   0024H     0002H     ABSOLUTE     
            XDATA   0026H     0002H     ABSOLUTE     
            XDATA   0028H     0002H     ABSOLUTE     
            XDATA   002AH     0001H     ABSOLUTE     
            XDATA   002BH     0001H     ABSOLUTE     
            XDATA   002CH     0002H     ABSOLUTE     
            XDATA   002EH     0001H     ABSOLUTE     
            XDATA   002FH     0001H     ABSOLUTE     
            XDATA   0030H     0002H     ABSOLUTE     
            XDATA   0032H     0002H     ABSOLUTE     
            XDATA   0034H     0001H     ABSOLUTE     
            XDATA   0035H     000CH     ABSOLUTE     
            XDATA   0041H     0004H     ABSOLUTE     
            XDATA   0045H     0002H     ABSOLUTE     
            XDATA   0047H     000CH     ABSOLUTE     
            XDATA   0053H     000CH     ABSOLUTE     
            XDATA   005FH     0002H     ABSOLUTE     
            XDATA   0061H     0001H     ABSOLUTE     
            XDATA   0062H     0002H     ABSOLUTE     
            XDATA   0064H     0002H     ABSOLUTE     
            XDATA   0066H     0001H     ABSOLUTE     
            XDATA   0067H     0001H     ABSOLUTE     
            XDATA   0068H     0002H     ABSOLUTE     
            XDATA   006AH     0002H     ABSOLUTE     
            XDATA   006CH     0001H     ABSOLUTE     
            XDATA   006DH     0004H     ABSOLUTE     
            XDATA   0071H     0001H     ABSOLUTE     
            XDATA   0072H     0001H     ABSOLUTE     
            XDATA   0073H     0001H     ABSOLUTE     
            XDATA   0074H     0002H     ABSOLUTE     
            XDATA   0076H     0002H     ABSOLUTE     
            XDATA   0078H     0001H     ABSOLUTE     
            XDATA   0079H     0001H     ABSOLUTE     
            XDATA   007AH     0002H     ABSOLUTE     
            XDATA   007CH     0001H     ABSOLUTE     
            XDATA   007DH     0004H     ABSOLUTE     
            XDATA   0081H     0001H     ABSOLUTE     
            XDATA   0082H     0004H     ABSOLUTE     
BL51 BANKED LINKER/LOCATER V6.22                                                      02/06/2025  15:28:46  PAGE 4


            XDATA   0086H     0001H     ABSOLUTE     
            XDATA   0087H     0001H     ABSOLUTE     
            XDATA   0088H     0001H     ABSOLUTE     
            XDATA   0089H     0002H     ABSOLUTE     
            XDATA   008BH     0001H     ABSOLUTE     
            XDATA   008CH     0001H     ABSOLUTE     
            XDATA   008DH     0001H     ABSOLUTE     
            XDATA   008EH     0002H     ABSOLUTE     
            XDATA   0090H     0002H     ABSOLUTE     
            XDATA   0092H     0002H     ABSOLUTE     
            XDATA   0094H     0002H     ABSOLUTE     
            XDATA   0096H     0001H     ABSOLUTE     
            XDATA   0097H     0001H     ABSOLUTE     
            XDATA   0098H     0001H     ABSOLUTE     
            XDATA   0099H     0002H     ABSOLUTE     
            XDATA   009BH     0002H     ABSOLUTE     
            XDATA   009DH     0002H     ABSOLUTE     
            XDATA   009FH     0002H     ABSOLUTE     
            XDATA   00A1H     0001H     ABSOLUTE     
            XDATA   00A2H     0002H     ABSOLUTE     
            XDATA   00A4H     0002H     ABSOLUTE     
            XDATA   00A6H     0002H     ABSOLUTE     
            XDATA   00A8H     0001H     ABSOLUTE     
            XDATA   00A9H     0001H     ABSOLUTE     
            XDATA   00AAH     0001H     ABSOLUTE     
            XDATA   00ABH     0004H     ABSOLUTE     
            XDATA   00AFH     0004H     ABSOLUTE     
            XDATA   00B3H     0004H     ABSOLUTE     
            XDATA   00B7H     0002H     ABSOLUTE     
            XDATA   00B9H     0001H     ABSOLUTE     
            XDATA   00BAH     0001H     ABSOLUTE     
            XDATA   00BBH     0001H     ABSOLUTE     
            XDATA   00BCH     0002H     ABSOLUTE     
            XDATA   00BEH     0001H     ABSOLUTE     
            XDATA   00BFH     0002H     ABSOLUTE     
            XDATA   00C1H     0002H     ABSOLUTE     
            XDATA   00C3H     0002H     ABSOLUTE     
            XDATA   00C5H     0002H     ABSOLUTE     
            XDATA   00C7H     0002H     ABSOLUTE     
            XDATA   00C9H     0001H     ABSOLUTE     
            XDATA   00CAH     0001H     ABSOLUTE     
            XDATA   00CBH     0133H     ABSOLUTE     
            XDATA   01FEH     0002H     ABSOLUTE     
            XDATA   0200H     00B5H     UNIT         ?XD?AFE
            XDATA   02B5H     006EH     UNIT         _XDATA_GROUP_
            XDATA   0323H     0067H     UNIT         ?XD?GASGAUGEINTER_V4_13
            XDATA   038AH     002EH     UNIT         ?XD?GASGAUGEV4_12
            XDATA   03B8H     0022H     UNIT         ?XD?PROTECT
            XDATA   03DAH     0015H     UNIT         ?XD?EXTE2PROM
            XDATA   03EFH     000DH     UNIT         ?XD?UARTAPP
            XDATA   03FCH     0003H     UNIT         ?XD?LED
            XDATA   03FFH     0001H     UNIT         ?XD?KEYAPP
            XDATA   0400H     0096H     ABSOLUTE     
            XDATA   0496H     0008H     UNIT         ?XD?RTC
            XDATA   049EH     0002H     UNIT         ?XD?INTERRUPTAPP
            XDATA   04A0H     0096H     ABSOLUTE     
            XDATA   0536H     0006H     UNIT         ?XD?BALANCE
BL51 BANKED LINKER/LOCATER V6.22                                                      02/06/2025  15:28:46  PAGE 5


            XDATA   053CH     0003H     UNIT         ?XD?LOWPOWER
            XDATA   053FH     0001H     UNIT         ?XD?PORSELFTEST
            XDATA   0540H     0096H     ABSOLUTE     
            XDATA   05D6H     0012H     UNIT         ?XD?CALIBRATE
            XDATA   05E8H     0003H     UNIT         ?XD?_MCUPWM0SET?MCULIB
            XDATA   05EBH     0003H     UNIT         ?XD?_MCUPWM1SET?MCULIB
            XDATA   05EEH     0002H     UNIT         ?XD?_UART0WRITEINFO?UARTAPP
            XDATA   05F0H     0002H     UNIT         ?XD?UART0RDCMDPROCESS?UARTAPP
            XDATA   05F2H     0002H     UNIT         ?XD?UART0WRCMDPROCESS?UARTAPP
            XDATA   05F4H     0002H     UNIT         ?XD?UART0IAPCHECKHANDSHAKE?UARTAPP
            XDATA   05F6H     0002H     UNIT         ?XD?CALCULATE
            XDATA   05F8H     0002H     UNIT         ?XD?CHARGERLOAD
            XDATA   05FAH     0002H     UNIT         ?XD?MCUFLASH
            XDATA   05FCH     0002H     UNIT         ?XD?GASGAUGEWKUP?GASGAUGEV4_12

            * * * * * * *   C O D E   M E M O R Y   * * * * * * *
            CODE    0000H     1000H     UNIT         ?CO?BOOTIAP
            CODE    1000H     0003H     ABSOLUTE     
            CODE    1003H     0020H     UNIT         ?PR?INTERRUPTTIMER3?INTERRUPT
            CODE    1023H     0003H     ABSOLUTE     
                    1026H     0005H                  *** GAP ***
            CODE    102BH     0003H     ABSOLUTE     
            CODE    102EH     0024H     UNIT         ?PR?_INTERRUPTINT4APP?INTERRUPTAPP
                    1052H     0001H                  *** GAP ***
            CODE    1053H     0003H     ABSOLUTE     
            CODE    1056H     0C24H     UNIT         ?PR?DATAFILTER?GASGAUGEV4_12
            CODE    1C7AH     08DFH     UNIT         ?C?LIB_CODE
            CODE    2559H     06CAH     UNIT         ?PR?GASGAUGEMANAGE?GASGAUGEV4_12
            CODE    2C23H     0483H     UNIT         ?PR?PRINTF?PRINTF
            CODE    30A6H     02EEH     UNIT         ?PR?MAIN?MAIN
            CODE    3394H     0258H     UNIT         ?PR?FCCUPDATE?GASGAUGEV4_12
            CODE    35ECH     0220H     UNIT         ?PR?GASGAUGEWKUP?GASGAUGEV4_12
            CODE    380CH     01F0H     UNIT         ?PR?_CALCUTEMP?CALCULATE
            CODE    39FCH     01C5H     UNIT         ?PR?GASGAUGEVARIN?GASGAUGEINTER_V4_13
            CODE    3BC1H     01C2H     UNIT         ?PR?_RTCREADTIME?RTC
            CODE    3D83H     01B9H     UNIT         ?PR?_TWIREAD?TWI
            CODE    3F3CH     01B3H     UNIT         ?PR?_E2PROMBKDATA?EXTE2PROM
            CODE    40EFH     0181H     UNIT         ?PR?AFECALCUCURR?CALCULATE
            CODE    4270H     016FH     UNIT         ?PR?_GASGAUGEINITSOC?GASGAUGEV4_12
            CODE    43DFH     0168H     UNIT         ?PR?GASGAUGEINIT?GASGAUGEV4_12
            CODE    4547H     0167H     UNIT         ?PR?UART0IAPCHECKHANDSHAKE?UARTAPP
            CODE    46AEH     0150H     UNIT         ?PR?UART0RDCMDPROCESS?UARTAPP
            CODE    47FEH     0147H     UNIT         ?PR?_TWIWRITE?TWI
            CODE    4945H     0144H     UNIT         ?PR?BALTURNONCHECK?BALANCE
            CODE    4A89H     0142H     UNIT         ?CO?THERMISTOR
            CODE    4BCBH     0138H     UNIT         ?PR?AFECALCUVOL?CALCULATE
            CODE    4D03H     011FH     UNIT         ?PR?GASGAUGEGETOCV?GASGAUGEV4_12
            CODE    4E22H     0100H     UNIT         ?CO?TWI
            CODE    4F22H     00DEH     UNIT         ?PR?AFECALCUTEMPE?CALCULATE
            CODE    5000H     00D7H     UNIT         ?PR?CORRECTCHGDFRC?GASGAUGEV4_12
            CODE    50D7H     00D3H     UNIT         ?PR?E2PROMBKCHECK?EXTE2PROM
            CODE    51AAH     00C4H     UNIT         ?PR?PROTECTOV?PROTECT
            CODE    526EH     00C1H     UNIT         ?PR?MCUFLASHPROCESS?MCUFLASH
            CODE    532FH     00BDH     UNIT         ?PR?UART0CALICURRENT?UARTAPP
            CODE    53ECH     00BCH     UNIT         ?PR?PROTECTUV?PROTECT
            CODE    54A8H     00BCH     UNIT         ?PR?PROTECTOTC?PROTECT
            CODE    5564H     00BCH     UNIT         ?PR?PROTECTUTC?PROTECT
BL51 BANKED LINKER/LOCATER V6.22                                                      02/06/2025  15:28:46  PAGE 6


            CODE    5620H     00BCH     UNIT         ?PR?PROTECTOTD?PROTECT
            CODE    56DCH     00BCH     UNIT         ?PR?PROTECTUTD?PROTECT
            CODE    5798H     00BAH     UNIT         ?PR?BALPROCESS?BALANCE
            CODE    5852H     00B3H     UNIT         ?PR?OFFSETCALCULATE?CALCULATE
            CODE    5905H     00ACH     UNIT         ?PR?E2PROMBKPROCESS?EXTE2PROM
            CODE    59B1H     00ABH     UNIT         ?PR?INTERRUPTUART0APPTX?UARTAPP
            CODE    5A5CH     00ABH     UNIT         ?PR?_AFEWRITEREG?AFE
            CODE    5B07H     00A7H     UNIT         ?PR?UART0WRCMDPROCESS?UARTAPP
            CODE    5BAEH     00A2H     UNIT         ?PR?KEYSCAN?KEYSCAN
            CODE    5C50H     00A1H     UNIT         ?CO?MAIN
            CODE    5CF1H     00A1H     UNIT         ?PR?SYSPARAINIT?INITIAL
            CODE    5D92H     009CH     UNIT         ?PR?_RTCMODIFYTIME?RTC
            CODE    5E2EH     0097H     UNIT         ?PR?_INTERRUPTUART0APPRX?UARTAPP
            CODE    5EC5H     0097H     UNIT         ?PR?_MCUFLASHWRITE?MCUFLASH
            CODE    5F5CH     008EH     UNIT         ?PR?LOWPOWERCHECK?LOWPOWER
            CODE    5FEAH     008DH     UNIT         ?PR?_RTCINITTIME?RTC
            CODE    6077H     008CH     UNIT         ?PR?_MCUFLASHWRSECTOR?MCUFLASH
            CODE    6103H     0087H     UNIT         ?PR?AFEINIT?AFE
            CODE    618AH     0086H     UNIT         ?PR?AFEINITREG?AFE
            CODE    6210H     0081H     UNIT         ?PR?_MCUPWM0SET?MCULIB
            CODE    6291H     0081H     UNIT         ?PR?_MCUPWM1SET?MCULIB
            CODE    6312H     0081H     UNIT         ?PR?_MCUPWM2SET?MCULIB
            CODE    6393H     007DH     UNIT         ?PR?E2PROMINIT?EXTE2PROM
            CODE    6410H     0076H     UNIT         ?PR?PROTECTOCRECOVER?PROTECT
            CODE    6486H     0070H     UNIT         ?PR?_UART0WRITEINFO?UARTAPP
            CODE    64F6H     006FH     UNIT         ?PR?UART1RDE2PROM?EXTE2PROM
            CODE    6565H     006FH     UNIT         ?PR?UART2RDE2PROM?EXTE2PROM
            CODE    65D4H     006FH     UNIT         ?PR?INTERRUPTINT4?INTERRUPT
            CODE    6643H     006DH     UNIT         ?PR?CALIVOLTAGE?CALIBRATE
            CODE    66B0H     006CH     UNIT         ?PR?E2PROMERASE?EXTE2PROM
            CODE    671CH     006BH     UNIT         ?PR?_AFEREADREG?AFE
            CODE    6787H     0069H     UNIT         ?PR?UART0RDE2PROM?EXTE2PROM
            CODE    67F0H     0066H     UNIT         ?PR?KEYSWITCHSPEED?KEYAPP
            CODE    6856H     0066H     UNIT         ?PR?RAMCHECKPROCESS?MCULIB
            CODE    68BCH     0063H     UNIT         ?PR?_UART0READINFO?UARTAPP
            CODE    691FH     0061H     UNIT         ?PR?AFERAMCHECK?AFE
            CODE    6980H     0061H     UNIT         ?PR?UART0INIT?UART
            CODE    69E1H     005FH     UNIT         ?PR?_E2PROMWRITE?EXTE2PROM
            CODE    6A40H     005FH     UNIT         ?PR?_E2PROMREAD?EXTE2PROM
            CODE    6A9FH     005FH     UNIT         ?PR?_MCUFLASHREAD?MCUFLASH
            CODE    6AFEH     005DH     UNIT         ?PR?_GETCYCLEGAIN?GASGAUGEV4_12
            CODE    6B5BH     005CH     UNIT         ?PR?LEDDISPLAY?LED
            CODE    6BB7H     005BH     UNIT         ?PR?_RTCWRITE?RTC
            CODE    6C12H     005BH     UNIT         ?PR?_RTCREAD?RTC
            CODE    6C6DH     005AH     UNIT         ?PR?_MCUFLASHDATACHECK?MCUFLASH
            CODE    6CC7H     0059H     UNIT         ?PR?PROTECTOCC?PROTECT
            CODE    6D20H     0059H     UNIT         ?PR?PROTECTOCD1?PROTECT
            CODE    6D79H     0059H     UNIT         ?PR?PROTECTOCD2?PROTECT
            CODE    6DD2H     0054H     UNIT         ?PR?UART0CALIRTC?UARTAPP
            CODE    6E26H     0052H     UNIT         ?PR?UART0CALIVOLTAGE?UARTAPP
            CODE    6E78H     0051H     UNIT         ?PR?GASGAUGEVAROUT?GASGAUGEINTER_V4_13
            CODE    6EC9H     004FH     UNIT         ?PR?CALIPROCESS?CALIBRATE
            CODE    6F18H     004FH     UNIT         ?PR?PORPROTECTOTC?PORSELFTEST
            CODE    6F67H     004FH     UNIT         ?PR?PORPROTECTUTC?PORSELFTEST
            CODE    6FB6H     004FH     UNIT         ?PR?PORPROTECTOTD?PORSELFTEST
            CODE    7005H     004FH     UNIT         ?PR?PORPROTECTUTD?PORSELFTEST
            CODE    7054H     004EH     UNIT         ?PR?LOADCHECK?CHARGERLOAD
BL51 BANKED LINKER/LOCATER V6.22                                                      02/06/2025  15:28:46  PAGE 7


            CODE    70A2H     004CH     UNIT         ?PR?INITIAL?INITIAL
            CODE    70EEH     004CH     UNIT         ?PR?E2PROMBKRTC?EXTE2PROM
            CODE    713AH     004CH     UNIT         ?PR?UART1RDRTC?EXTE2PROM
            CODE    7186H     004CH     UNIT         ?PR?UART2RDRTC?EXTE2PROM
            CODE    71D2H     004AH     UNIT         ?PR?AFEGETVOL?CALCULATE
            CODE    721CH     004AH     UNIT         ?PR?MOSSTATUSCHECK?MOSCTRL
            CODE    7266H     0049H     UNIT         ?PR?UART0CALITS1?UARTAPP
            CODE    72AFH     0049H     UNIT         ?PR?UART0CALITS2?UARTAPP
            CODE    72F8H     0049H     UNIT         ?PR?CHGERCHECK?CHARGERLOAD
            CODE    7341H     0048H     UNIT         ?CO?UARTAPP
            CODE    7389H     0048H     UNIT         ?PR?AFEGETTEMPE?CALCULATE
            CODE    73D1H     0048H     UNIT         ?PR?_DELAY1MS?MCULIB
            CODE    7419H     0048H     UNIT         ?PR?PORPROTECTOV?PORSELFTEST
            CODE    7461H     0048H     UNIT         ?PR?PORPROTECTUV?PORSELFTEST
            CODE    74A9H     0046H     UNIT         ?PR?UART0RDRTC?EXTE2PROM
            CODE    74EFH     0045H     UNIT         ?PR?UART0WRITEMANUFACTURE?UARTAPP
            CODE    7534H     0045H     UNIT         ?PR?CALITS1?CALIBRATE
            CODE    7579H     0045H     UNIT         ?PR?CALITS2?CALIBRATE
            CODE    75BEH     0044H     UNIT         ?PR?CALIRTCTIME?CALIBRATE
            CODE    7602H     0044H     UNIT         ?C?LDIV
            CODE    7646H     0042H     UNIT         ?PR?INITVAR?INITIAL
            CODE    7688H     0041H     UNIT         ?PR?E2PROMBKBOOT?EXTE2PROM
            CODE    76C9H     0040H     UNIT         ?PR?WAKEUPPROCESS?LOWPOWER
            CODE    7709H     0040H     UNIT         ?PR?LOWPOWERPROCESS?LOWPOWER
            CODE    7749H     003FH     UNIT         ?PR?_LEDGETDISNUM?LED
            CODE    7788H     003FH     UNIT         ?PR?_AFEBALCTL?AFE
            CODE    77C7H     003DH     UNIT         ?PR?AFERDFLG?AFE
            CODE    7804H     003CH     UNIT         ?PR?AFECLRFLG?AFE
            CODE    7840H     003BH     UNIT         ?PR?CALICURRENTGAIN?CALIBRATE
            CODE    787BH     003BH     UNIT         ?PR?PORSELFTEST?PORSELFTEST
            CODE    78B6H     0037H     UNIT         ?PR?UART0READSUBCLASSID?UARTAPP
            CODE    78EDH     0036H     UNIT         ?PR?SYSTEMINTOSLEEP?LOWPOWER
            CODE    7923H     0036H     UNIT         ?PR?UART0CALICUROFFSET?UARTAPP
            CODE    7959H     0035H     UNIT         ?PR?CTOCHECKVOL?BALANCE
            CODE    798EH     0035H     UNIT         ?PR?_MCUFLASHWRONEBYTE?MCUFLASH
            CODE    79C3H     0035H     UNIT         ?PR?GASGAUGEIDLE?GASGAUGEV4_12
            CODE    79F8H     0034H     UNIT         ?CO?CALCULATE
            CODE    7A2CH     0033H     UNIT         ?PR?_MEMORYCOPY?MCULIB
            CODE    7A5FH     0030H     UNIT         ?PR?KEYPROCESS?KEYAPP
            CODE    7A8FH     0030H     UNIT         ?PR?_MCUTIMER3SET?MCULIB
            CODE    7ABFH     002DH     UNIT         ?PR?MOSCTRL?MOSCTRL
            CODE    7AECH     002CH     UNIT         ?PR?SYSTEMRESETPROCESS?MCULIB
            CODE    7B18H     002BH     UNIT         ?PR?INITGPIO?INITIAL
            CODE    7B43H     002AH     UNIT         ?PR?_MEMORYSET?MCULIB
            CODE    7B6DH     0027H     UNIT         ?PR?_MCUFLASHCHECKFLG?MCUFLASH
            CODE    7B94H     0027H     UNIT         ?PR?_TWICHECKSTATUS?TWI
            CODE    7BBBH     0026H     UNIT         ?PR?AFEENTERPD?AFE
            CODE    7BE1H     0026H     UNIT         ?PR?CTOTURNONCHECK?BALANCE
            CODE    7C07H     0026H     UNIT         ?PR?_MCUFLASHBLANKCHECK?MCUFLASH
            CODE    7C2DH     0024H     UNIT         ?PR?INTERRUPTTIMER3APP?INTERRUPTAPP
            CODE    7C51H     0022H     UNIT         ?PR?_MCUCLOCKSET?MCULIB
            CODE    7C73H     0020H     UNIT         ?C_C51STARTUP
            CODE    7C93H     001FH     UNIT         ?PR?PROTECTPROCESS?PROTECT
            CODE    7CB2H     001FH     UNIT         ?PR?INTERRUPTUART0?UART
            CODE    7CD1H     001EH     UNIT         ?PR?INITIRQ?INITIAL
            CODE    7CEFH     001DH     UNIT         ?PR?E2PROMTWICHECK?EXTE2PROM
            CODE    7D0CH     001DH     UNIT         ?PR?RTCTWICHECK?RTC
BL51 BANKED LINKER/LOCATER V6.22                                                      02/06/2025  15:28:46  PAGE 8


            CODE    7D29H     001DH     UNIT         ?PR?ISPPROCESS?BOOTAPP
            CODE    7D46H     001CH     UNIT         ?PR?_CRC8CAL?TWI
            CODE    7D62H     001AH     UNIT         ?PR?AFETWICHECK?AFE
            CODE    7D7CH     0018H     UNIT         ?PR?AFERDSTATUS?AFE
            CODE    7D94H     0017H     UNIT         ?PR?_AFEALARMDIS?AFE
            CODE    7DABH     0017H     UNIT         ?PR?TWIINIT?TWI
            CODE    7DC2H     0015H     UNIT         ?PR?_AFEMOSCTL?AFE
            CODE    7DD7H     0015H     UNIT         ?PR?MCUFLASHWRWAITCHECK?MCUFLASH
            CODE    7DECH     0014H     UNIT         ?PR?UART0CHECK?UARTAPP
            CODE    7E00H     0014H     UNIT         ?PR?AFEINFOPROCESS?CALCULATE
            CODE    7E14H     0013H     UNIT         ?PR?LEDAUTOOFF?LED
            CODE    7E27H     0013H     UNIT         ?PR?AFECHGERCHECKEN?AFE
            CODE    7E3AH     0013H     UNIT         ?PR?AFECHGERCHECKDIS?AFE
            CODE    7E4DH     0013H     UNIT         ?PR?AFELOADCHECKEN?AFE
            CODE    7E60H     0013H     UNIT         ?PR?AFELOADCHECKDIS?AFE
            CODE    7E73H     0013H     UNIT         ?PR?AFEWDTEN?AFE
            CODE    7E86H     0013H     UNIT         ?PR?AFEWDTDIS?AFE
            CODE    7E99H     0013H     UNIT         ?PR?AFEADCEN?AFE
            CODE    7EACH     0013H     UNIT         ?PR?AFEADCDIS?AFE
            CODE    7EBFH     0013H     UNIT         ?PR?AFECADCEN?AFE
            CODE    7ED2H     0013H     UNIT         ?PR?AFECADCDIS?AFE
            CODE    7EE5H     0013H     UNIT         ?PR?AFETEMPADCEN?AFE
            CODE    7EF8H     0013H     UNIT         ?PR?AFETEMPADCDIS?AFE
            CODE    7F0BH     0012H     UNIT         ?PR?SYSTEMINTOPD?LOWPOWER
            CODE    7F1DH     0012H     UNIT         ?PR?UART0HANDSHAKE?UARTAPP
            CODE    7F2FH     0012H     UNIT         ?PR?_AFEALARMEN?AFE
            CODE    7F41H     0010H     UNIT         ?PR?CALICURZERO?CALIBRATE
            CODE    7F51H     000EH     UNIT         ?PR?_PUTCHAR?MAIN
            CODE    7F5FH     000CH     UNIT         ?PR?MCUINTOIDLE?MCULIB
            CODE    7F6BH     000CH     UNIT         ?PR?MCUINTOPD?MCULIB
            CODE    7F77H     000AH     UNIT         ?PR?BALANCEPROCESS?BALANCE
            CODE    7F81H     0006H     UNIT         ?CO?GASGAUGEV4_12



OVERLAY MAP OF MODULE:   .\output\MCUCore_Load (MAIN)


SEGMENT                                           BIT_GROUP          DATA_GROUP          XDATA_GROUP
  +--> CALLED SEGMENT                          START    LENGTH     START    LENGTH     START    LENGTH
------------------------------------------------------------------------------------------------------
?PR?INTERRUPTINT4?INTERRUPT                    -----    -----      -----    -----      -----    -----
  +--> ?PR?_INTERRUPTINT4APP?INTERRUPTAPP

?PR?_INTERRUPTINT4APP?INTERRUPTAPP             -----    -----      -----    -----      -----    -----
  +--> ?PR?_MCUCLOCKSET?MCULIB

?PR?_MCUCLOCKSET?MCULIB                        -----    -----      -----    -----      02B7H    0001H

*** NEW ROOT ***************************************************

?PR?INTERRUPTTIMER3?INTERRUPT                  -----    -----      -----    -----      -----    -----
  +--> ?PR?INTERRUPTTIMER3APP?INTERRUPTAPP

?PR?INTERRUPTTIMER3APP?INTERRUPTAPP            -----    -----      -----    -----      -----    -----
  +--> ?PR?KEYSCAN?KEYSCAN

BL51 BANKED LINKER/LOCATER V6.22                                                      02/06/2025  15:28:46  PAGE 9


*** NEW ROOT ***************************************************

?PR?INTERRUPTUART0?UART                        -----    -----      -----    -----      02B6H    0001H

*** NEW ROOT ***************************************************

?C_C51STARTUP                                  -----    -----      -----    -----      -----    -----
  +--> ?PR?MAIN?MAIN

?PR?MAIN?MAIN                                  -----    -----      -----    -----      -----    -----
  +--> ?PR?INITIAL?INITIAL
  +--> ?CO?MAIN
  +--> ?PR?PRINTF?PRINTF
  +--> ?PR?AFEINFOPROCESS?CALCULATE
  +--> ?PR?BALANCEPROCESS?BALANCE
  +--> ?PR?PROTECTPROCESS?PROTECT
  +--> ?PR?PORSELFTEST?PORSELFTEST
  +--> ?PR?LOADCHECK?CHARGERLOAD
  +--> ?PR?CHGERCHECK?CHARGERLOAD
  +--> ?PR?MOSCTRL?MOSCTRL
  +--> ?PR?PROTECTOCRECOVER?PROTECT
  +--> ?PR?UART0CHECK?UARTAPP
  +--> ?PR?GASGAUGEMANAGE?GASGAUGEV4_12
  +--> ?PR?AFERAMCHECK?AFE
  +--> ?PR?AFETWICHECK?AFE
  +--> ?PR?E2PROMTWICHECK?EXTE2PROM
  +--> ?PR?RTCTWICHECK?RTC
  +--> ?PR?RAMCHECKPROCESS?MCULIB
  +--> ?PR?SYSPARAINIT?INITIAL
  +--> ?PR?MCUFLASHWRWAITCHECK?MCUFLASH
  +--> ?PR?E2PROMBKCHECK?EXTE2PROM
  +--> ?PR?SYSTEMRESETPROCESS?MCULIB
  +--> ?PR?ISPPROCESS?BOOTAPP
  +--> ?PR?CALIPROCESS?CALIBRATE
  +--> ?PR?MCUFLASHPROCESS?MCUFLASH
  +--> ?PR?E2PROMBKPROCESS?EXTE2PROM

?PR?INITIAL?INITIAL                            -----    -----      -----    -----      -----    -----
  +--> ?PR?_MCUCLOCKSET?MCULIB
  +--> ?PR?INITGPIO?INITIAL
  +--> ?PR?SYSPARAINIT?INITIAL
  +--> ?PR?INITVAR?INITIAL
  +--> ?PR?_MCUTIMER3SET?MCULIB
  +--> ?PR?UART0INIT?UART
  +--> ?PR?TWIINIT?TWI
  +--> ?PR?_MCUPWM2SET?MCULIB
  +--> ?PR?AFEINITREG?AFE
  +--> ?PR?AFEINIT?AFE
  +--> ?PR?AFECLRFLG?AFE
  +--> ?PR?E2PROMINIT?EXTE2PROM
  +--> ?PR?_RTCINITTIME?RTC
  +--> ?PR?INITIRQ?INITIAL

?PR?SYSPARAINIT?INITIAL                        -----    -----      -----    -----      -----    -----
  +--> ?PR?_MCUFLASHCHECKFLG?MCUFLASH
  +--> ?PR?_MCUFLASHREAD?MCUFLASH
  +--> ?PR?_MCUFLASHWRITE?MCUFLASH
BL51 BANKED LINKER/LOCATER V6.22                                                      02/06/2025  15:28:46  PAGE 10



?PR?_MCUFLASHCHECKFLG?MCUFLASH                 0029H.5  0000H.1    -----    -----      -----    -----

?PR?_MCUFLASHREAD?MCUFLASH                     0029H.5  0000H.1    0015H    0002H      02B7H    0004H

?PR?_MCUFLASHWRITE?MCUFLASH                    0029H.7  0000H.1    -----    -----      02B9H    0004H
  +--> ?PR?_MCUFLASHBLANKCHECK?MCUFLASH
  +--> ?PR?_MCUFLASHWRSECTOR?MCUFLASH
  +--> ?PR?_MCUFLASHDATACHECK?MCUFLASH

?PR?_MCUFLASHBLANKCHECK?MCUFLASH               002AH.0  0000H.1    -----    -----      -----    -----

?PR?_MCUFLASHWRSECTOR?MCUFLASH                 002AH.0  0000H.1    -----    -----      02BDH    0004H

?PR?_MCUFLASHDATACHECK?MCUFLASH                002AH.0  0000H.1    -----    -----      02BDH    0004H

?PR?INITVAR?INITIAL                            -----    -----      -----    -----      -----    -----
  +--> ?PR?_MEMORYSET?MCULIB

?PR?_MEMORYSET?MCULIB                          -----    -----      -----    -----      02C3H    0002H

?PR?_MCUTIMER3SET?MCULIB                       -----    -----      -----    -----      02B7H    0001H

?PR?UART0INIT?UART                             -----    -----      -----    -----      02B7H    0002H

?PR?_MCUPWM2SET?MCULIB                         -----    -----      -----    -----      02BCH    0003H

?PR?AFEINIT?AFE                                0029H.5  0000H.1    -----    -----      02BAH    0004H
  +--> ?PR?_AFEWRITEREG?AFE
  +--> ?PR?_AFEREADREG?AFE

?PR?_AFEWRITEREG?AFE                           0029H.6  0000H.1    -----    -----      02BEH    0006H
  +--> ?PR?_TWIWRITE?TWI
  +--> ?PR?_DELAY1MS?MCULIB
  +--> ?PR?TWIINIT?TWI

?PR?_TWIWRITE?TWI                              002AH.1  0000H.1    -----    -----      02F3H    000EH
  +--> ?PR?_CRC8CAL?TWI
  +--> ?PR?_TWICHECKSTATUS?TWI

?PR?_CRC8CAL?TWI                               -----    -----      -----    -----      -----    -----
  +--> ?CO?TWI

?PR?_TWICHECKSTATUS?TWI                        002AH.2  0000H.1    -----    -----      -----    -----

?PR?_AFEREADREG?AFE                            0029H.6  0000H.1    -----    -----      02C1H    0005H
  +--> ?PR?_TWIREAD?TWI
  +--> ?PR?_DELAY1MS?MCULIB
  +--> ?PR?TWIINIT?TWI

?PR?_TWIREAD?TWI                               002AH.0  0000H.1    -----    -----      02E9H    003AH
  +--> ?PR?_TWICHECKSTATUS?TWI
  +--> ?PR?_CRC8CAL?TWI

?PR?AFECLRFLG?AFE                              -----    -----      -----    -----      -----    -----
  +--> ?PR?_AFEREADREG?AFE
  +--> ?PR?_AFEWRITEREG?AFE
BL51 BANKED LINKER/LOCATER V6.22                                                      02/06/2025  15:28:46  PAGE 11



?PR?E2PROMINIT?EXTE2PROM                       0029H.5  0000H.1    -----    -----      02B7H    0008H
  +--> ?PR?_E2PROMREAD?EXTE2PROM

?PR?_E2PROMREAD?EXTE2PROM                      0029H.6  0000H.1    -----    -----      02C3H    0006H
  +--> ?PR?_TWIREAD?TWI
  +--> ?PR?_DELAY1MS?MCULIB

?PR?_RTCINITTIME?RTC                           0029H.5  0000H.1    -----    -----      02B7H    000CH
  +--> ?PR?_MEMORYSET?MCULIB
  +--> ?PR?_E2PROMREAD?EXTE2PROM
  +--> ?PR?_MEMORYCOPY?MCULIB
  +--> ?PR?_RTCREADTIME?RTC

?PR?_MEMORYCOPY?MCULIB                         -----    -----      -----    -----      02D9H    0002H

?PR?_RTCREADTIME?RTC                           0029H.6  0000H.1    -----    -----      02D9H    000BH
  +--> ?PR?_RTCREAD?RTC
  +--> ?PR?_RTCMODIFYTIME?RTC

?PR?_RTCREAD?RTC                               0029H.7  0000H.1    -----    -----      02E4H    0005H
  +--> ?PR?_TWIREAD?TWI
  +--> ?PR?_DELAY1MS?MCULIB

?PR?_RTCMODIFYTIME?RTC                         0029H.7  0000H.1    -----    -----      02E4H    000AH
  +--> ?PR?_RTCWRITE?RTC

?PR?_RTCWRITE?RTC                              002AH.0  0000H.1    -----    -----      02EEH    0005H
  +--> ?PR?_TWIWRITE?TWI
  +--> ?PR?_DELAY1MS?MCULIB

?PR?PRINTF?PRINTF                              0029H.5  0001H.1    0015H    0005H      02B7H    0030H
  +--> ?PR?_PUTCHAR?MAIN

?PR?AFEINFOPROCESS?CALCULATE                   -----    -----      -----    -----      -----    -----
  +--> ?PR?AFERDFLG?AFE
  +--> ?PR?AFECALCUVOL?CALCULATE
  +--> ?PR?AFECALCUTEMPE?CALCULATE
  +--> ?PR?AFECALCUCURR?CALCULATE

?PR?AFERDFLG?AFE                               -----    -----      -----    -----      -----    -----
  +--> ?PR?_AFEREADREG?AFE
  +--> ?PR?AFEINIT?AFE

?PR?AFECALCUVOL?CALCULATE                      -----    -----      -----    -----      02B7H    0009H
  +--> ?PR?AFEGETVOL?CALCULATE

?PR?AFEGETVOL?CALCULATE                        0029H.5  0000H.1    -----    -----      02C0H    0001H
  +--> ?PR?_AFEREADREG?AFE

?PR?AFECALCUTEMPE?CALCULATE                    -----    -----      -----    -----      -----    -----
  +--> ?PR?AFEGETTEMPE?CALCULATE
  +--> ?PR?_CALCUTEMP?CALCULATE

?PR?AFEGETTEMPE?CALCULATE                      0029H.5  0000H.1    -----    -----      -----    -----
  +--> ?PR?_AFEREADREG?AFE

BL51 BANKED LINKER/LOCATER V6.22                                                      02/06/2025  15:28:46  PAGE 12


?PR?_CALCUTEMP?CALCULATE                       -----    -----      -----    -----      02B7H    0007H
  +--> ?CO?THERMISTOR

?PR?AFECALCUCURR?CALCULATE                     -----    -----      -----    -----      02B7H    0005H
  +--> ?PR?_AFEREADREG?AFE
  +--> ?PR?OFFSETCALCULATE?CALCULATE
  +--> ?PR?_MCUPWM2SET?MCULIB

?PR?OFFSETCALCULATE?CALCULATE                  -----    -----      -----    -----      02BCH    0003H
  +--> ?CO?CALCULATE

?PR?BALANCEPROCESS?BALANCE                     -----    -----      -----    -----      -----    -----
  +--> ?PR?BALTURNONCHECK?BALANCE
  +--> ?PR?CTOTURNONCHECK?BALANCE
  +--> ?PR?BALPROCESS?BALANCE

?PR?BALPROCESS?BALANCE                         -----    -----      -----    -----      02B7H    0002H
  +--> ?PR?_AFEBALCTL?AFE
  +--> ?PR?CTOCHECKVOL?BALANCE

?PR?_AFEBALCTL?AFE                             -----    -----      -----    -----      02B9H    0002H
  +--> ?PR?_AFEWRITEREG?AFE

?PR?CTOCHECKVOL?BALANCE                        0029H.5  0000H.1    -----    -----      -----    -----

?PR?PROTECTPROCESS?PROTECT                     -----    -----      -----    -----      -----    -----
  +--> ?PR?PROTECTOV?PROTECT
  +--> ?PR?PROTECTUV?PROTECT
  +--> ?PR?PROTECTOTC?PROTECT
  +--> ?PR?PROTECTUTC?PROTECT
  +--> ?PR?PROTECTOTD?PROTECT
  +--> ?PR?PROTECTUTD?PROTECT
  +--> ?PR?PROTECTOCC?PROTECT
  +--> ?PR?PROTECTOCD1?PROTECT
  +--> ?PR?PROTECTOCD2?PROTECT

?PR?PROTECTOV?PROTECT                          -----    -----      -----    -----      -----    -----
  +--> ?PR?AFECLRFLG?AFE

?PR?PORSELFTEST?PORSELFTEST                    -----    -----      -----    -----      -----    -----
  +--> ?PR?AFECALCUVOL?CALCULATE
  +--> ?PR?AFECALCUTEMPE?CALCULATE
  +--> ?PR?PORPROTECTOV?PORSELFTEST
  +--> ?PR?PORPROTECTUV?PORSELFTEST
  +--> ?PR?PORPROTECTOTC?PORSELFTEST
  +--> ?PR?PORPROTECTUTC?PORSELFTEST
  +--> ?PR?PORPROTECTOTD?PORSELFTEST
  +--> ?PR?PORPROTECTUTD?PORSELFTEST
  +--> ?PR?GASGAUGEINIT?GASGAUGEV4_12

?PR?GASGAUGEINIT?GASGAUGEV4_12                 -----    -----      -----    -----      02B7H    0002H
  +--> ?PR?GASGAUGEVARIN?GASGAUGEINTER_V4_13
  +--> ?PR?GASGAUGEGETOCV?GASGAUGEV4_12
  +--> ?PR?_GASGAUGEINITSOC?GASGAUGEV4_12
  +--> ?PR?GASGAUGEVAROUT?GASGAUGEINTER_V4_13

?PR?GASGAUGEVARIN?GASGAUGEINTER_V4_13          0029H.5  0000H.1    -----    -----      -----    -----
BL51 BANKED LINKER/LOCATER V6.22                                                      02/06/2025  15:28:46  PAGE 13



?PR?GASGAUGEGETOCV?GASGAUGEV4_12               -----    -----      -----    -----      02B9H    0001H

?PR?_GASGAUGEINITSOC?GASGAUGEV4_12             -----    -----      -----    -----      02B9H    0002H

?PR?GASGAUGEVAROUT?GASGAUGEINTER_V4_13         0029H.5  0000H.1    -----    -----      -----    -----

?PR?LOADCHECK?CHARGERLOAD                      -----    -----      -----    -----      -----    -----
  +--> ?PR?AFELOADCHECKEN?AFE
  +--> ?PR?AFERDSTATUS?AFE
  +--> ?PR?AFELOADCHECKDIS?AFE
  +--> ?PR?AFECLRFLG?AFE

?PR?AFELOADCHECKEN?AFE                         -----    -----      -----    -----      -----    -----
  +--> ?PR?_AFEWRITEREG?AFE

?PR?AFERDSTATUS?AFE                            -----    -----      -----    -----      02B7H    0002H
  +--> ?PR?_AFEREADREG?AFE

?PR?AFELOADCHECKDIS?AFE                        -----    -----      -----    -----      -----    -----
  +--> ?PR?_AFEWRITEREG?AFE

?PR?CHGERCHECK?CHARGERLOAD                     -----    -----      -----    -----      -----    -----
  +--> ?PR?AFECHGERCHECKEN?AFE
  +--> ?PR?AFERDSTATUS?AFE
  +--> ?PR?AFECHGERCHECKDIS?AFE
  +--> ?PR?AFECLRFLG?AFE

?PR?AFECHGERCHECKEN?AFE                        -----    -----      -----    -----      -----    -----
  +--> ?PR?_AFEWRITEREG?AFE

?PR?AFECHGERCHECKDIS?AFE                       -----    -----      -----    -----      -----    -----
  +--> ?PR?_AFEWRITEREG?AFE

?PR?MOSCTRL?MOSCTRL                            -----    -----      -----    -----      -----    -----
  +--> ?PR?MOSSTATUSCHECK?MOSCTRL
  +--> ?PR?_AFEMOSCTL?AFE

?PR?_AFEMOSCTL?AFE                             -----    -----      -----    -----      -----    -----
  +--> ?PR?_AFEWRITEREG?AFE

?PR?PROTECTOCRECOVER?PROTECT                   -----    -----      -----    -----      -----    -----
  +--> ?PR?AFECLRFLG?AFE

?PR?GASGAUGEMANAGE?GASGAUGEV4_12               -----    -----      -----    -----      -----    -----
  +--> ?PR?GASGAUGEVARIN?GASGAUGEINTER_V4_13
  +--> ?PR?CORRECTCHGDFRC?GASGAUGEV4_12
  +--> ?PR?FCCUPDATE?GASGAUGEV4_12
  +--> ?PR?DATAFILTER?GASGAUGEV4_12
  +--> ?PR?GASGAUGEVAROUT?GASGAUGEINTER_V4_13

?PR?CORRECTCHGDFRC?GASGAUGEV4_12               -----    -----      -----    -----      02B7H    0002H
  +--> ?PR?GASGAUGEGETOCV?GASGAUGEV4_12

?PR?FCCUPDATE?GASGAUGEV4_12                    -----    -----      -----    -----      02B7H    0004H
  +--> ?PR?_GETCYCLEGAIN?GASGAUGEV4_12

BL51 BANKED LINKER/LOCATER V6.22                                                      02/06/2025  15:28:46  PAGE 14


?PR?DATAFILTER?GASGAUGEV4_12                   0029H.5  0000H.1    -----    -----      02B7H    0009H
  +--> ?CO?GASGAUGEV4_12

?PR?AFERAMCHECK?AFE                            -----    -----      -----    -----      02B7H    0003H
  +--> ?PR?_AFEREADREG?AFE
  +--> ?PR?AFEINIT?AFE

?PR?E2PROMBKCHECK?EXTE2PROM                    -----    -----      -----    -----      -----    -----
  +--> ?PR?_RTCREADTIME?RTC
  +--> ?PR?_MEMORYCOPY?MCULIB

?PR?ISPPROCESS?BOOTAPP                         -----    -----      -----    -----      -----    -----
  +--> ?PR?AFEWDTDIS?AFE

?PR?AFEWDTDIS?AFE                              -----    -----      -----    -----      -----    -----
  +--> ?PR?_AFEWRITEREG?AFE

?PR?CALIPROCESS?CALIBRATE                      -----    -----      -----    -----      -----    -----
  +--> ?PR?CALIVOLTAGE?CALIBRATE
  +--> ?PR?CALICURRENTGAIN?CALIBRATE
  +--> ?PR?CALICURZERO?CALIBRATE
  +--> ?PR?CALITS1?CALIBRATE
  +--> ?PR?CALITS2?CALIBRATE
  +--> ?PR?CALIRTCTIME?CALIBRATE

?PR?CALIVOLTAGE?CALIBRATE                      -----    -----      -----    -----      02B7H    0002H

?PR?CALITS1?CALIBRATE                          -----    -----      -----    -----      -----    -----
  +--> ?PR?_CALCUTEMP?CALCULATE

?PR?CALITS2?CALIBRATE                          -----    -----      -----    -----      -----    -----
  +--> ?PR?_CALCUTEMP?CALCULATE

?PR?CALIRTCTIME?CALIBRATE                      -----    -----      -----    -----      -----    -----
  +--> ?PR?_RTCMODIFYTIME?RTC

?PR?MCUFLASHPROCESS?MCUFLASH                   0029H.5  0000H.2    -----    -----      02B7H    0002H
  +--> ?PR?_MCUFLASHWRITE?MCUFLASH
  +--> ?PR?_MCUFLASHWRONEBYTE?MCUFLASH

?PR?E2PROMBKPROCESS?EXTE2PROM                  -----    -----      -----    -----      02B7H    0001H
  +--> ?PR?E2PROMERASE?EXTE2PROM
  +--> ?PR?UART0RDE2PROM?EXTE2PROM
  +--> ?PR?UART2RDE2PROM?EXTE2PROM
  +--> ?PR?UART0RDRTC?EXTE2PROM
  +--> ?PR?UART1RDRTC?EXTE2PROM
  +--> ?PR?UART2RDRTC?EXTE2PROM
  +--> ?PR?E2PROMBKRTC?EXTE2PROM
  +--> ?PR?_E2PROMBKDATA?EXTE2PROM

?PR?E2PROMERASE?EXTE2PROM                      -----    -----      -----    -----      02B8H    000AH
  +--> ?PR?_MEMORYSET?MCULIB
  +--> ?PR?_E2PROMWRITE?EXTE2PROM

?PR?_E2PROMWRITE?EXTE2PROM                     0029H.5  0000H.1    -----    -----      02E1H    0006H
  +--> ?PR?_TWIWRITE?TWI
  +--> ?PR?_DELAY1MS?MCULIB
BL51 BANKED LINKER/LOCATER V6.22                                                      02/06/2025  15:28:46  PAGE 15



?PR?UART0RDE2PROM?EXTE2PROM                    -----    -----      -----    -----      -----    -----
  +--> ?PR?_E2PROMREAD?EXTE2PROM
  +--> ?PR?_CRC8CAL?TWI

?PR?UART2RDE2PROM?EXTE2PROM                    -----    -----      -----    -----      -----    -----
  +--> ?PR?_E2PROMREAD?EXTE2PROM
  +--> ?PR?_CRC8CAL?TWI

?PR?UART0RDRTC?EXTE2PROM                       -----    -----      -----    -----      -----    -----
  +--> ?PR?_RTCREADTIME?RTC
  +--> ?PR?_MEMORYCOPY?MCULIB
  +--> ?PR?_CRC8CAL?TWI

?PR?UART1RDRTC?EXTE2PROM                       -----    -----      -----    -----      -----    -----
  +--> ?PR?_RTCREADTIME?RTC
  +--> ?PR?_MEMORYCOPY?MCULIB
  +--> ?PR?_CRC8CAL?TWI

?PR?UART2RDRTC?EXTE2PROM                       -----    -----      -----    -----      -----    -----
  +--> ?PR?_RTCREADTIME?RTC
  +--> ?PR?_MEMORYCOPY?MCULIB
  +--> ?PR?_CRC8CAL?TWI

?PR?E2PROMBKRTC?EXTE2PROM                      -----    -----      -----    -----      02B8H    000AH
  +--> ?PR?_RTCREADTIME?RTC
  +--> ?PR?_MEMORYCOPY?MCULIB
  +--> ?PR?_E2PROMWRITE?EXTE2PROM

?PR?_E2PROMBKDATA?EXTE2PROM                    -----    -----      -----    -----      02B8H    0021H
  +--> ?PR?_MEMORYCOPY?MCULIB
  +--> ?PR?_RTCREADTIME?RTC
  +--> ?PR?_E2PROMWRITE?EXTE2PROM
  +--> ?PR?E2PROMBKBOOT?EXTE2PROM

?PR?E2PROMBKBOOT?EXTE2PROM                     -----    -----      -----    -----      02D9H    0008H
  +--> ?PR?_E2PROMWRITE?EXTE2PROM



SYMBOL TABLE OF MODULE:  .\output\MCUCore_Load (MAIN)

  VALUE           TYPE          NAME
  ----------------------------------

  -------         MODULE        MAIN
  C:0000H         SYMBOL        _ICE_DUMMY_
  D:0080H         PUBLIC        P0
  D:0090H         PUBLIC        P1
  D:00A0H         PUBLIC        P2
  D:00B0H         PUBLIC        P3
  D:00C0H         PUBLIC        P4
  D:0080H         PUBLIC        P5
  B:00A0H.0       PUBLIC        P2_0
  B:00A0H.4       PUBLIC        P2_4
  B:0098H.1       PUBLIC        TI
  C:30A6H         PUBLIC        main
BL51 BANKED LINKER/LOCATER V6.22                                                      02/06/2025  15:28:46  PAGE 16


  D:0099H         PUBLIC        SBUF
  D:00B1H         PUBLIC        RSTSTAT
  B:0098H.4       PUBLIC        REN
  C:7F51H         PUBLIC        _putchar
  -------         PROC          _PUTCHAR
  D:0007H         SYMBOL        c
  C:7F51H         LINE#         13
  C:7F51H         LINE#         14
  C:7F51H         LINE#         15
  C:7F53H         LINE#         16
  C:7F55H         LINE#         17
  C:7F57H         LINE#         18
  C:7F5AH         LINE#         19
  C:7F5CH         LINE#         20
  C:7F5EH         LINE#         21
  C:7F5EH         LINE#         22
  -------         ENDPROC       _PUTCHAR
  -------         PROC          MAIN
  C:30A6H         LINE#         32
  C:30A6H         LINE#         33
  C:30A6H         LINE#         34
  C:30A9H         LINE#         36
  C:30B2H         LINE#         38
  C:30B2H         LINE#         39
  C:30B2H         LINE#         42
  C:30B5H         LINE#         43
  C:30B5H         LINE#         44
  C:30B8H         LINE#         46
  C:30BAH         LINE#         47
  C:30BDH         LINE#         49
  C:30C0H         LINE#         51
  C:30C3H         LINE#         53
  C:30C6H         LINE#         55
  C:30C9H         LINE#         57
  C:30CCH         LINE#         59
  C:30CFH         LINE#         61
  C:30D2H         LINE#         66
  C:30D5H         LINE#         76
  C:30D5H         LINE#         78
  C:30DBH         LINE#         79
  C:30DBH         LINE#         80
  C:30DDH         LINE#         82
  C:30E6H         LINE#         83
  C:3133H         LINE#         84
  C:3180H         LINE#         85
  C:31CDH         LINE#         86
  C:321AH         LINE#         87
  C:3267H         LINE#         88
  C:32D8H         LINE#         89
  C:32E1H         LINE#         90
  C:331AH         LINE#         92
  C:3335H         LINE#         93
  C:3350H         LINE#         95
  C:3352H         LINE#         96
  C:3355H         LINE#         98
  C:3358H         LINE#         100
  C:335BH         LINE#         101
BL51 BANKED LINKER/LOCATER V6.22                                                      02/06/2025  15:28:46  PAGE 17


  C:335EH         LINE#         102
  C:3361H         LINE#         104
  C:3366H         LINE#         105
  C:3366H         LINE#         106
  C:3369H         LINE#         107
  C:3369H         LINE#         109
  C:336CH         LINE#         111
  C:336FH         LINE#         116
  C:336FH         LINE#         118
  C:3372H         LINE#         120
  C:3375H         LINE#         122
  C:3378H         LINE#         124
  C:337BH         LINE#         126
  C:337EH         LINE#         130
  C:3388H         LINE#         131
  C:3390H         LINE#         133
  -------         ENDPROC       MAIN
  -------         ENDMOD        MAIN

  -------         MODULE        INITIAL
  C:0000H         SYMBOL        _ICE_DUMMY_
  D:0080H         PUBLIC        P0
  D:0090H         PUBLIC        P1
  D:00A0H         PUBLIC        P2
  D:00B0H         PUBLIC        P3
  C:7CD1H         PUBLIC        InitIRQ
  D:00C0H         PUBLIC        P4
  D:0080H         PUBLIC        P5
  B:00A8H.7       PUBLIC        EA
  D:00A9H         PUBLIC        IEN1
  D:00E8H         PUBLIC        EXF0
  D:00D8H         PUBLIC        EXF1
  D:00E1H         PUBLIC        P0CR
  D:00E2H         PUBLIC        P1CR
  D:00E3H         PUBLIC        P2CR
  D:00E4H         PUBLIC        P3CR
  D:00BAH         PUBLIC        IENC
  C:7646H         PUBLIC        InitVar
  C:7B18H         PUBLIC        InitGPIO
  B:00A8H.4       PUBLIC        ES0
  B:00A8H.5       PUBLIC        ET3
  D:0086H         PUBLIC        INSCON
  B:0088H.7       PUBLIC        TF3
  C:70A2H         PUBLIC        Initial
  C:5CF1H         PUBLIC        SysParaInit
  D:00E9H         PUBLIC        P0PCR
  D:00EAH         PUBLIC        P1PCR
  D:00EBH         PUBLIC        P2PCR
  D:00ECH         PUBLIC        P3PCR
  -------         PROC          INITVAR
  C:7646H         LINE#         18
  C:7646H         LINE#         19
  C:7646H         LINE#         20
  C:764CH         LINE#         21
  C:7657H         LINE#         22
  C:7661H         LINE#         23
  C:766BH         LINE#         24
BL51 BANKED LINKER/LOCATER V6.22                                                      02/06/2025  15:28:46  PAGE 18


  C:7673H         LINE#         26
  C:7675H         LINE#         27
  C:7677H         LINE#         28
  C:767DH         LINE#         29
  C:767FH         LINE#         30
  C:7681H         LINE#         32
  C:7687H         LINE#         33
  -------         ENDPROC       INITVAR
  -------         PROC          SYSPARAINIT
  C:5CF1H         LINE#         41
  C:5CF1H         LINE#         42
  C:5CF1H         LINE#         43
  C:5CFAH         LINE#         44
  C:5CFAH         LINE#         45
  C:5D06H         LINE#         46
  C:5D0FH         LINE#         47
  C:5D0FH         LINE#         48
  C:5D17H         LINE#         49
  C:5D17H         LINE#         50
  C:5D19H         LINE#         51
  C:5D22H         LINE#         52
  C:5D22H         LINE#         53
  C:5D2FH         LINE#         54
  C:5D36H         LINE#         55
  C:5D38H         LINE#         57
  C:5D38H         LINE#         58
  C:5D3BH         LINE#         60
  C:5D3BH         LINE#         62
  C:5D45H         LINE#         63
  C:5D4FH         LINE#         64
  C:5D5BH         LINE#         65
  C:5D6AH         LINE#         67
  C:5D72H         LINE#         69
  C:5D7BH         LINE#         70
  C:5D7BH         LINE#         71
  C:5D7EH         LINE#         72
  C:5D7FH         LINE#         73
  C:5D8AH         LINE#         74
  C:5D8AH         LINE#         75
  C:5D8DH         LINE#         76
  C:5D8EH         LINE#         78
  C:5D8EH         LINE#         79
  C:5D91H         LINE#         80
  C:5D91H         LINE#         81
  -------         ENDPROC       SYSPARAINIT
  -------         PROC          INITIRQ
  C:7CD1H         LINE#         89
  C:7CD1H         LINE#         90
  C:7CD1H         LINE#         91
  C:7CD3H         LINE#         93
  C:7CD5H         LINE#         102
  C:7CDEH         LINE#         103
  C:7CE0H         LINE#         105
  C:7CE3H         LINE#         106
  C:7CE6H         LINE#         107
  C:7CE9H         LINE#         108
  C:7CECH         LINE#         110
BL51 BANKED LINKER/LOCATER V6.22                                                      02/06/2025  15:28:46  PAGE 19


  C:7CEEH         LINE#         111
  -------         ENDPROC       INITIRQ
  -------         PROC          INITGPIO
  C:7B18H         LINE#         164
  C:7B18H         LINE#         165
  C:7B18H         LINE#         167
  C:7B1BH         LINE#         168
  C:7B1EH         LINE#         169
  C:7B21H         LINE#         171
  C:7B24H         LINE#         172
  C:7B27H         LINE#         173
  C:7B2AH         LINE#         175
  C:7B2DH         LINE#         176
  C:7B30H         LINE#         177
  C:7B33H         LINE#         179
  C:7B36H         LINE#         180
  C:7B39H         LINE#         181
  C:7B3CH         LINE#         185
  C:7B3FH         LINE#         186
  C:7B42H         LINE#         530
  -------         ENDPROC       INITGPIO
  -------         PROC          INITIAL
  C:70A2H         LINE#         538
  C:70A2H         LINE#         539
  C:70A2H         LINE#         540
  C:70A7H         LINE#         542
  C:70AAH         LINE#         546
  C:70ADH         LINE#         548
  C:70B0H         LINE#         550
  C:70B9H         LINE#         553
  C:70BCH         LINE#         564
  C:70BFH         LINE#         566
  C:70C8H         LINE#         568
  C:70CBH         LINE#         569
  C:70D0H         LINE#         570
  C:70D0H         LINE#         571
  C:70D2H         LINE#         572
  C:70D2H         LINE#         573
  C:70D5H         LINE#         575
  C:70D8H         LINE#         576
  C:70D8H         LINE#         577
  C:70DDH         LINE#         578
  C:70DDH         LINE#         579
  C:70DFH         LINE#         580
  C:70DFH         LINE#         582
  C:70E8H         LINE#         583
  C:70E8H         LINE#         584
  C:70EAH         LINE#         585
  C:70EAH         LINE#         586
  C:70EAH         LINE#         588
  C:70EDH         LINE#         589
  -------         ENDPROC       INITIAL
  -------         ENDMOD        INITIAL

  -------         MODULE        INTERRUPTAPP
  C:0000H         SYMBOL        _ICE_DUMMY_
  D:0080H         PUBLIC        P0
BL51 BANKED LINKER/LOCATER V6.22                                                      02/06/2025  15:28:46  PAGE 20


  D:0090H         PUBLIC        P1
  D:00A0H         PUBLIC        P2
  X:049EH         PUBLIC        ucTimer1s
  D:00B0H         PUBLIC        P3
  D:00C0H         PUBLIC        P4
  D:0080H         PUBLIC        P5
  C:102EH         PUBLIC        _InterruptINT4App
  B:002DH.6       PUBLIC        bTimer5msFlg
  X:049FH         PUBLIC        ucTimer50ms
  B:002DH.7       PUBLIC        bTimer1sFlg
  C:7C2DH         PUBLIC        InterruptTimer3App
  B:002EH.0       PUBLIC        bTimer50msFlg
  -------         PROC          _INTERRUPTINT4APP
  D:0007H         SYMBOL        IntSource
  C:102EH         LINE#         24
  C:102EH         LINE#         25
  C:102EH         LINE#         26
  C:1032H         LINE#         27
  C:1032H         LINE#         28
  C:1038H         LINE#         29
  C:1038H         LINE#         30
  C:103DH         LINE#         31
  C:103FH         LINE#         32
  C:103FH         LINE#         33
  C:1040H         LINE#         34
  C:1044H         LINE#         35
  C:1044H         LINE#         36
  C:104AH         LINE#         37
  C:104AH         LINE#         38
  C:104FH         LINE#         39
  C:1051H         LINE#         40
  C:1051H         LINE#         41
  C:1051H         LINE#         42
  -------         ENDPROC       _INTERRUPTINT4APP
  -------         PROC          INTERRUPTTIMER3APP
  C:7C2DH         LINE#         51
  C:7C2DH         LINE#         52
  C:7C2DH         LINE#         54
  C:7C2FH         LINE#         56
  C:7C3AH         LINE#         57
  C:7C3AH         LINE#         58
  C:7C3CH         LINE#         59
  C:7C3EH         LINE#         60
  C:7C3EH         LINE#         62
  C:7C49H         LINE#         63
  C:7C49H         LINE#         64
  C:7C4BH         LINE#         65
  C:7C4DH         LINE#         66
  C:7C4DH         LINE#         68
  C:7C50H         LINE#         69
  -------         ENDPROC       INTERRUPTTIMER3APP
  -------         ENDMOD        INTERRUPTAPP

  -------         MODULE        LED
  C:0000H         SYMBOL        _ICE_DUMMY_
  D:0080H         PUBLIC        P0
  D:0090H         PUBLIC        P1
BL51 BANKED LINKER/LOCATER V6.22                                                      02/06/2025  15:28:46  PAGE 21


  D:00A0H         PUBLIC        P2
  D:00B0H         PUBLIC        P3
  D:00C0H         PUBLIC        P4
  D:0080H         PUBLIC        P5
  C:7749H         PUBLIC        _LedGetDisNum
  B:00A0H.1       PUBLIC        P2_1
  B:00A0H.2       PUBLIC        P2_2
  B:00A0H.3       PUBLIC        P2_3
  X:03FCH         PUBLIC        ucLedChgFlickCnt
  B:00B0H.5       PUBLIC        P3_5
  X:03FDH         PUBLIC        ucLedBleFlickCnt
  X:03FEH         PUBLIC        ucLedTimeCnt
  B:002EH.4       PUBLIC        bLedDisFlg
  B:002EH.5       PUBLIC        bLedDisBleFlg
  C:7E14H         PUBLIC        LedAutoOff
  C:6B5BH         PUBLIC        LedDisplay
  -------         PROC          _LEDGETDISNUM
  D:0006H         SYMBOL        Rsoc
  C:7749H         LINE#         24
  C:7749H         LINE#         25
  C:7749H         LINE#         26
  C:7752H         LINE#         27
  C:7752H         LINE#         28
  C:7755H         LINE#         29
  C:7755H         LINE#         30
  C:775EH         LINE#         31
  C:775EH         LINE#         32
  C:7761H         LINE#         33
  C:7761H         LINE#         34
  C:776AH         LINE#         35
  C:776AH         LINE#         36
  C:776DH         LINE#         37
  C:776DH         LINE#         38
  C:7776H         LINE#         39
  C:7776H         LINE#         40
  C:7779H         LINE#         41
  C:7779H         LINE#         42
  C:7782H         LINE#         43
  C:7782H         LINE#         44
  C:7785H         LINE#         45
  C:7785H         LINE#         47
  C:7785H         LINE#         48
  C:7787H         LINE#         49
  C:7787H         LINE#         50
  -------         ENDPROC       _LEDGETDISNUM
  -------         PROC          LEDAUTOOFF
  C:7E14H         LINE#         59
  C:7E14H         LINE#         60
  C:7E14H         LINE#         61
  C:7E17H         LINE#         62
  C:7E17H         LINE#         63
  C:7E22H         LINE#         64
  C:7E22H         LINE#         65
  C:7E24H         LINE#         66
  C:7E26H         LINE#         67
  C:7E26H         LINE#         68
  C:7E26H         LINE#         69
BL51 BANKED LINKER/LOCATER V6.22                                                      02/06/2025  15:28:46  PAGE 22


  -------         ENDPROC       LEDAUTOOFF
  -------         PROC          LEDDISPLAY
  -------         DO            
  D:0007H         SYMBOL        LedDisNum
  -------         ENDDO         
  C:6B5BH         LINE#         80
  C:6B5BH         LINE#         81
  C:6B5BH         LINE#         84
  C:6B5EH         LINE#         85
  C:6B5EH         LINE#         86
  C:6B69H         LINE#         87
  C:6B69H         LINE#         88
  C:6B6BH         LINE#         89
  C:6B70H         LINE#         90
  C:6B70H         LINE#         91
  C:6B72H         LINE#         93
  C:6B72H         LINE#         94
  C:6B74H         LINE#         95
  C:6B74H         LINE#         97
  C:6B77H         LINE#         98
  C:6B77H         LINE#         99
  C:6B82H         LINE#         100
  C:6B82H         LINE#         101
  C:6B84H         LINE#         103
  C:6B84H         LINE#         104
  C:6B84H         LINE#         106
  C:6B84H         LINE#         108
  C:6B84H         LINE#         110
  C:6B87H         LINE#         111
  C:6B87H         LINE#         112
  C:6B92H         LINE#         113
  C:6B92H         LINE#         114
  C:6B92H         LINE#         116
  C:6B92H         LINE#         117
  C:6B97H         LINE#         118
  C:6B97H         LINE#         120
  C:6B97H         LINE#         121
  C:6B9BH         LINE#         122
  C:6B9BH         LINE#         124
  C:6B9DH         LINE#         125
  C:6B9FH         LINE#         126
  C:6BA3H         LINE#         127
  C:6BA3H         LINE#         129
  C:6BA5H         LINE#         130
  C:6BA7H         LINE#         131
  C:6BA9H         LINE#         132
  C:6BADH         LINE#         133
  C:6BADH         LINE#         135
  C:6BAFH         LINE#         136
  C:6BB1H         LINE#         137
  C:6BB3H         LINE#         138
  C:6BB3H         LINE#         139
  C:6BB3H         LINE#         140
  C:6BB3H         LINE#         142
  C:6BB3H         LINE#         143
  C:6BB3H         LINE#         145
  C:6BB3H         LINE#         147
BL51 BANKED LINKER/LOCATER V6.22                                                      02/06/2025  15:28:46  PAGE 23


  C:6BB3H         LINE#         149
  C:6BB6H         LINE#         150
  -------         ENDPROC       LEDDISPLAY
  -------         ENDMOD        LED

  -------         MODULE        KEYAPP
  C:0000H         SYMBOL        _ICE_DUMMY_
  D:0080H         PUBLIC        P0
  D:0090H         PUBLIC        P1
  D:00A0H         PUBLIC        P2
  D:00B0H         PUBLIC        P3
  D:00C0H         PUBLIC        P4
  D:0080H         PUBLIC        P5
  D:00B7H         PUBLIC        PWM2CON
  C:7A5FH         PUBLIC        KeyProcess
  B:0080H.3       PUBLIC        P0_3
  C:67F0H         PUBLIC        KeySwitchSpeed
  X:03FFH         PUBLIC        ucDsgingSpeed
  -------         PROC          KEYSWITCHSPEED
  C:67F0H         LINE#         20
  C:67F0H         LINE#         21
  C:67F0H         LINE#         22
  C:67F2H         LINE#         23
  C:67F4H         LINE#         24
  C:67F6H         LINE#         25
  C:67F9H         LINE#         26
  C:67F9H         LINE#         27
  C:67FFH         LINE#         28
  C:67FFH         LINE#         29
  C:6801H         LINE#         30
  C:6803H         LINE#         31
  C:6813H         LINE#         32
  C:6816H         LINE#         33
  C:6817H         LINE#         34
  C:681EH         LINE#         35
  C:681EH         LINE#         36
  C:6821H         LINE#         37
  C:6823H         LINE#         38
  C:6830H         LINE#         39
  C:6833H         LINE#         40
  C:6834H         LINE#         42
  C:6834H         LINE#         43
  C:6839H         LINE#         44
  C:683BH         LINE#         45
  C:684BH         LINE#         46
  C:684EH         LINE#         47
  C:684EH         LINE#         48
  C:684FH         LINE#         50
  C:684FH         LINE#         51
  C:6851H         LINE#         52
  C:6853H         LINE#         53
  C:6855H         LINE#         54
  C:6855H         LINE#         55
  -------         ENDPROC       KEYSWITCHSPEED
  -------         PROC          KEYPROCESS
  C:7A5FH         LINE#         64
  C:7A5FH         LINE#         65
BL51 BANKED LINKER/LOCATER V6.22                                                      02/06/2025  15:28:46  PAGE 24


  C:7A5FH         LINE#         66
  C:7A62H         LINE#         67
  C:7A62H         LINE#         68
  C:7A64H         LINE#         69
  C:7A75H         LINE#         70
  C:7A75H         LINE#         71
  C:7A75H         LINE#         72
  C:7A78H         LINE#         73
  C:7A79H         LINE#         75
  C:7A79H         LINE#         76
  C:7A7BH         LINE#         77
  C:7A80H         LINE#         78
  C:7A81H         LINE#         80
  C:7A81H         LINE#         81
  C:7A83H         LINE#         82
  C:7A84H         LINE#         84
  C:7A84H         LINE#         85
  C:7A86H         LINE#         86
  C:7A89H         LINE#         87
  C:7A89H         LINE#         88
  C:7A8BH         LINE#         89
  C:7A8CH         LINE#         91
  C:7A8CH         LINE#         92
  C:7A8EH         LINE#         93
  C:7A8EH         LINE#         94
  C:7A8EH         LINE#         96
  C:7A8EH         LINE#         97
  C:7A8EH         LINE#         98
  C:7A8EH         LINE#         99
  C:7A8EH         LINE#         100
  -------         ENDPROC       KEYPROCESS
  -------         ENDMOD        KEYAPP

  -------         MODULE        LOWPOWER
  C:0000H         SYMBOL        _ICE_DUMMY_
  D:0080H         PUBLIC        P0
  D:0090H         PUBLIC        P1
  X:053CH         PUBLIC        ucSleepTimerCnt
  D:00A0H         PUBLIC        P2
  D:00B0H         PUBLIC        P3
  D:00C0H         PUBLIC        P4
  D:0080H         PUBLIC        P5
  B:00A8H.7       PUBLIC        EA
  B:00C8H.6       PUBLIC        ENTWI
  D:00B7H         PUBLIC        PWM2CON
  B:002CH.6       PUBLIC        bPDFlg
  B:0080H.3       PUBLIC        P0_3
  D:00D8H         PUBLIC        EXF1
  B:00A0H.5       PUBLIC        P2_5
  X:053DH         PUBLIC        ucPDTimerCnt
  C:78EDH         PUBLIC        SystemIntoSleep
  C:5F5CH         PUBLIC        LowPowerCheck
  B:002CH.7       PUBLIC        bPCEnterPDFlg
  C:7709H         PUBLIC        LowPowerProcess
  C:76C9H         PUBLIC        WakeUpProcess
  D:00B1H         PUBLIC        RSTSTAT
  C:7F0BH         PUBLIC        SystemIntoPD
BL51 BANKED LINKER/LOCATER V6.22                                                      02/06/2025  15:28:46  PAGE 25


  B:00A8H.4       PUBLIC        ES0
  B:00A8H.5       PUBLIC        ET3
  X:053EH         PUBLIC        ucResetFlag
  B:002DH.0       PUBLIC        bWakeupFlg
  B:002DH.1       PUBLIC        bSleepFlg
  -------         PROC          WAKEUPPROCESS
  C:76C9H         LINE#         26
  C:76C9H         LINE#         27
  C:76C9H         LINE#         28
  C:76CCH         LINE#         29
  C:76CCH         LINE#         30
  C:76CEH         LINE#         31
  C:76D1H         LINE#         32
  C:76D1H         LINE#         33
  C:76D6H         LINE#         34
  C:76D8H         LINE#         36
  C:76DAH         LINE#         37
  C:76DFH         LINE#         38
  C:76E4H         LINE#         41
  C:76E6H         LINE#         43
  C:76E8H         LINE#         44
  C:76EAH         LINE#         46
  C:76EFH         LINE#         47
  C:76F2H         LINE#         48
  C:76F5H         LINE#         49
  C:76F5H         LINE#         50
  C:76FAH         LINE#         51
  C:76FCH         LINE#         52
  C:7700H         LINE#         53
  C:7704H         LINE#         54
  C:7708H         LINE#         55
  C:7708H         LINE#         56
  -------         ENDPROC       WAKEUPPROCESS
  -------         PROC          SYSTEMINTOPD
  C:7F0BH         LINE#         65
  C:7F0BH         LINE#         66
  C:7F0BH         LINE#         67
  C:7F0BH         LINE#         68
  C:7F0BH         LINE#         69
  C:7F0EH         LINE#         71
  C:7F10H         LINE#         73
  C:7F12H         LINE#         74
  C:7F17H         LINE#         76
  C:7F1AH         LINE#         77
  -------         ENDPROC       SYSTEMINTOPD
  -------         PROC          SYSTEMINTOSLEEP
  C:78EDH         LINE#         87
  C:78EDH         LINE#         88
  C:78EDH         LINE#         90
  C:78EFH         LINE#         91
  C:78F1H         LINE#         93
  C:78F4H         LINE#         94
  C:78F7H         LINE#         95
  C:78FCH         LINE#         96
  C:78FEH         LINE#         97
  C:7901H         LINE#         98
  C:7904H         LINE#         99
BL51 BANKED LINKER/LOCATER V6.22                                                      02/06/2025  15:28:46  PAGE 26


  C:7904H         LINE#         100
  C:7906H         LINE#         101
  C:7908H         LINE#         103
  C:7908H         LINE#         104
  C:790AH         LINE#         105
  C:790AH         LINE#         106
  C:790FH         LINE#         108
  C:7911H         LINE#         110
  C:7913H         LINE#         118
  C:7915H         LINE#         119
  C:7918H         LINE#         120
  C:791DH         LINE#         121
  C:791FH         LINE#         123
  C:7922H         LINE#         124
  -------         ENDPROC       SYSTEMINTOSLEEP
  -------         PROC          LOWPOWERCHECK
  C:5F5CH         LINE#         135
  C:5F5CH         LINE#         136
  C:5F5CH         LINE#         137
  C:5F68H         LINE#         138
  C:5F68H         LINE#         139
  C:5F6AH         LINE#         140
  C:5F6CH         LINE#         141
  C:5F6DH         LINE#         142
  C:5F70H         LINE#         143
  C:5F70H         LINE#         144
  C:5F7FH         LINE#         145
  C:5F7FH         LINE#         146
  C:5F81H         LINE#         147
  C:5F83H         LINE#         148
  C:5F83H         LINE#         149
  C:5F84H         LINE#         150
  C:5F87H         LINE#         151
  C:5F87H         LINE#         152
  C:5F8DH         LINE#         153
  C:5F8DH         LINE#         154
  C:5F90H         LINE#         155
  C:5F90H         LINE#         156
  C:5F9FH         LINE#         157
  C:5F9FH         LINE#         158
  C:5FA1H         LINE#         159
  C:5FA3H         LINE#         160
  C:5FA3H         LINE#         161
  C:5FA4H         LINE#         163
  C:5FA4H         LINE#         164
  C:5FA9H         LINE#         165
  C:5FC1H         LINE#         166
  C:5FC1H         LINE#         167
  C:5FCFH         LINE#         168
  C:5FCFH         LINE#         169
  C:5FD1H         LINE#         170
  C:5FD3H         LINE#         171
  C:5FD3H         LINE#         172
  C:5FD4H         LINE#         174
  C:5FD4H         LINE#         175
  C:5FD9H         LINE#         176
  C:5FD9H         LINE#         177
BL51 BANKED LINKER/LOCATER V6.22                                                      02/06/2025  15:28:46  PAGE 27


  C:5FD9H         LINE#         178
  C:5FDAH         LINE#         180
  C:5FDAH         LINE#         181
  C:5FDFH         LINE#         182
  C:5FE1H         LINE#         183
  C:5FE1H         LINE#         184
  C:5FE2H         LINE#         186
  C:5FE2H         LINE#         187
  C:5FE7H         LINE#         188
  C:5FE9H         LINE#         189
  C:5FE9H         LINE#         190
  -------         ENDPROC       LOWPOWERCHECK
  -------         PROC          LOWPOWERPROCESS
  C:7709H         LINE#         199
  C:7709H         LINE#         200
  C:7709H         LINE#         201
  C:770FH         LINE#         202
  C:770FH         LINE#         203
  C:7711H         LINE#         204
  C:7729H         LINE#         205
  C:7729H         LINE#         206
  C:772BH         LINE#         207
  C:772EH         LINE#         208
  C:772EH         LINE#         209
  C:7730H         LINE#         210
  C:7732H         LINE#         211
  C:7735H         LINE#         212
  C:7735H         LINE#         213
  C:7737H         LINE#         214
  C:773AH         LINE#         215
  C:773DH         LINE#         216
  C:773FH         LINE#         217
  C:7742H         LINE#         218
  C:7742H         LINE#         219
  C:7745H         LINE#         220
  C:7745H         LINE#         222
  C:7748H         LINE#         223
  -------         ENDPROC       LOWPOWERPROCESS
  -------         ENDMOD        LOWPOWER

  -------         MODULE        UARTAPP
  C:0000H         SYMBOL        _ICE_DUMMY_
  D:0080H         PUBLIC        P0
  C:46AEH         PUBLIC        Uart0RdCmdProcess
  D:0090H         PUBLIC        P1
  C:78B6H         PUBLIC        Uart0ReadSubClassID
  D:00A0H         PUBLIC        P2
  D:00B0H         PUBLIC        P3
  D:00C0H         PUBLIC        P4
  B:0028H.3       PUBLIC        bUart0SndAckFlg
  D:0080H         PUBLIC        P5
  B:0028H.4       PUBLIC        bUart1SndAckFlg
  B:0028H.5       PUBLIC        bUart2SndAckFlg
  X:03EFH         PUBLIC        ucSubClassID
  C:5E2EH         PUBLIC        _InterruptUart0AppRx
  C:5B07H         PUBLIC        Uart0WrCmdProcess
  C:59B1H         PUBLIC        InterruptUart0AppTx
BL51 BANKED LINKER/LOCATER V6.22                                                      02/06/2025  15:28:46  PAGE 28


  X:03F0H         PUBLIC        ucUartErrCode
  C:6E26H         PUBLIC        Uart0CaliVoltage
  C:7266H         PUBLIC        Uart0CaliTS1
  C:72AFH         PUBLIC        Uart0CaliTS2
  C:7341H         PUBLIC        Page1WrRdFuncTable
  C:7365H         PUBLIC        Page2WrRdFuncTable
  C:7DECH         PUBLIC        Uart0Check
  D:0099H         PUBLIC        SBUF
  C:532FH         PUBLIC        Uart0CaliCurrent
  C:6DD2H         PUBLIC        Uart0CaliRTC
  X:03F1H         PUBLIC        ucUart0SndLength
  X:03F2H         PUBLIC        ucUart1SndLength
  X:03F3H         PUBLIC        ucUart2SndLength
  D:00B1H         PUBLIC        RSTSTAT
  X:03F4H         PUBLIC        ucUart0TimeoutCnt
  X:03F5H         PUBLIC        ucUart1TimeoutCnt
  X:03F6H         PUBLIC        ucUart2TimeoutCnt
  X:0400H         PUBLIC        ucUart0Buf
  X:04A0H         PUBLIC        ucUart1Buf
  X:0540H         PUBLIC        ucUart2Buf
  B:0028H.6       PUBLIC        bUart0ReadFlg
  B:0028H.7       PUBLIC        bUart1ReadFlg
  B:0029H.0       PUBLIC        bUart2ReadFlg
  C:4547H         PUBLIC        Uart0IapCheckHandshake
  B:0029H.1       PUBLIC        bUart0WriteFlg
  C:68BCH         PUBLIC        _Uart0ReadInfo
  C:7F1DH         PUBLIC        Uart0Handshake
  B:0029H.2       PUBLIC        bUart1WriteFlg
  B:0029H.3       PUBLIC        bUart2WriteFlg
  C:74EFH         PUBLIC        Uart0WriteManufacture
  C:7923H         PUBLIC        Uart0CaliCurOffset
  B:0098H.4       PUBLIC        REN
  B:0029H.4       PUBLIC        bISPFlg
  C:6486H         PUBLIC        _Uart0WriteInfo
  X:03F7H         PUBLIC        ucUart0BufPT
  X:03F8H         PUBLIC        ucUart1BufPT
  X:03F9H         PUBLIC        ucUart2BufPT
  D:009AH         PUBLIC        SADDR
  X:03FAH         PUBLIC        uiReceCheckSum
  -------         PROC          UART0HANDSHAKE
  C:7F1DH         LINE#         110
  C:7F1DH         LINE#         111
  C:7F1DH         LINE#         112
  C:7F23H         LINE#         113
  C:7F23H         LINE#         114
  C:7F28H         LINE#         115
  C:7F29H         LINE#         117
  C:7F29H         LINE#         118
  C:7F2EH         LINE#         119
  C:7F2EH         LINE#         120
  -------         ENDPROC       UART0HANDSHAKE
  -------         PROC          _UART0WRITEINFO
  X:05EEH         SYMBOL        ptr
  -------         DO            
  D:0007H         SYMBOL        i
  -------         ENDDO         
  C:6486H         LINE#         170
BL51 BANKED LINKER/LOCATER V6.22                                                      02/06/2025  15:28:46  PAGE 29


  C:648EH         LINE#         171
  C:648EH         LINE#         174
  C:64AFH         LINE#         175
  C:64AFH         LINE#         176
  C:64BAH         LINE#         177
  C:64BAH         LINE#         178
  C:64BDH         LINE#         179
  C:64D6H         LINE#         180
  C:64E0H         LINE#         181
  C:64E3H         LINE#         182
  C:64E5H         LINE#         183
  C:64EAH         LINE#         185
  C:64EFH         LINE#         186
  C:64F0H         LINE#         188
  C:64F0H         LINE#         189
  C:64F5H         LINE#         190
  C:64F5H         LINE#         191
  -------         ENDPROC       _UART0WRITEINFO
  -------         PROC          _UART0READINFO
  D:0006H         SYMBOL        ptr
  -------         DO            
  D:0005H         SYMBOL        i
  -------         ENDDO         
  C:68BCH         LINE#         263
  C:68BCH         LINE#         264
  C:68BCH         LINE#         267
  C:68C5H         LINE#         268
  C:68C5H         LINE#         269
  C:68C7H         LINE#         270
  C:68C7H         LINE#         271
  C:68D3H         LINE#         272
  C:68D3H         LINE#         273
  C:68D6H         LINE#         274
  C:68E8H         LINE#         275
  C:68EDH         LINE#         276
  C:68F0H         LINE#         277
  C:690CH         LINE#         279
  C:691EH         LINE#         280
  -------         ENDPROC       _UART0READINFO
  -------         PROC          UART0WRITEMANUFACTURE
  C:74EFH         LINE#         346
  C:74EFH         LINE#         347
  C:74EFH         LINE#         348
  C:7510H         LINE#         349
  C:7510H         LINE#         350
  C:7518H         LINE#         351
  C:7518H         LINE#         352
  C:751EH         LINE#         353
  C:7520H         LINE#         354
  C:7524H         LINE#         355
  C:7524H         LINE#         356
  C:7526H         LINE#         357
  C:7526H         LINE#         358
  C:7528H         LINE#         359
  C:752DH         LINE#         360
  C:752EH         LINE#         362
  C:752EH         LINE#         363
BL51 BANKED LINKER/LOCATER V6.22                                                      02/06/2025  15:28:46  PAGE 30


  C:7533H         LINE#         364
  C:7533H         LINE#         365
  -------         ENDPROC       UART0WRITEMANUFACTURE
  -------         PROC          UART0READSUBCLASSID
  C:78B6H         LINE#         437
  C:78B6H         LINE#         438
  C:78B6H         LINE#         439
  C:78D7H         LINE#         440
  C:78D7H         LINE#         441
  C:78DFH         LINE#         443
  C:78E1H         LINE#         444
  C:78E6H         LINE#         445
  C:78E7H         LINE#         447
  C:78E7H         LINE#         448
  C:78ECH         LINE#         449
  C:78ECH         LINE#         450
  -------         ENDPROC       UART0READSUBCLASSID
  -------         PROC          UART0RDCMDPROCESS
  -------         DO            
  X:05F0H         SYMBOL        rdaddr
  -------         ENDDO         
  C:46AEH         LINE#         506
  C:46AEH         LINE#         507
  C:46AEH         LINE#         510
  C:4702H         LINE#         511
  C:4702H         LINE#         512
  C:4702H         LINE#         513
  C:4702H         LINE#         514
  C:4702H         LINE#         515
  C:4702H         LINE#         516
  C:4702H         LINE#         517
  C:4702H         LINE#         518
  C:4702H         LINE#         519
  C:4702H         LINE#         520
  C:4702H         LINE#         521
  C:4702H         LINE#         522
  C:4712H         LINE#         523
  C:4713H         LINE#         525
  C:4713H         LINE#         526
  C:471AH         LINE#         527
  C:471BH         LINE#         529
  C:471BH         LINE#         530
  C:4722H         LINE#         531
  C:4723H         LINE#         533
  C:4723H         LINE#         534
  C:472AH         LINE#         535
  C:472BH         LINE#         537
  C:472BH         LINE#         538
  C:4732H         LINE#         539
  C:4733H         LINE#         541
  C:4733H         LINE#         542
  C:473AH         LINE#         543
  C:473BH         LINE#         545
  C:473BH         LINE#         546
  C:4742H         LINE#         547
  C:4743H         LINE#         549
  C:4743H         LINE#         550
BL51 BANKED LINKER/LOCATER V6.22                                                      02/06/2025  15:28:46  PAGE 31


  C:474AH         LINE#         551
  C:474BH         LINE#         553
  C:474BH         LINE#         554
  C:4752H         LINE#         555
  C:4753H         LINE#         557
  C:4753H         LINE#         558
  C:475AH         LINE#         559
  C:475BH         LINE#         561
  C:475BH         LINE#         562
  C:4762H         LINE#         563
  C:4763H         LINE#         565
  C:4763H         LINE#         566
  C:476AH         LINE#         567
  C:476BH         LINE#         569
  C:476BH         LINE#         570
  C:4772H         LINE#         571
  C:4773H         LINE#         573
  C:4773H         LINE#         574
  C:477AH         LINE#         575
  C:477BH         LINE#         577
  C:477BH         LINE#         578
  C:4782H         LINE#         579
  C:4783H         LINE#         581
  C:4783H         LINE#         582
  C:478CH         LINE#         583
  C:478CH         LINE#         584
  C:478EH         LINE#         585
  C:4794H         LINE#         586
  C:4795H         LINE#         587
  C:47A3H         LINE#         588
  C:47A3H         LINE#         589
  C:47A5H         LINE#         590
  C:47ABH         LINE#         591
  C:47ACH         LINE#         592
  C:47B3H         LINE#         593
  C:47B3H         LINE#         594
  C:47D1H         LINE#         595
  C:47D4H         LINE#         596
  C:47D5H         LINE#         597
  C:47DCH         LINE#         598
  C:47DCH         LINE#         599
  C:47FAH         LINE#         600
  C:47FDH         LINE#         601
  C:47FDH         LINE#         602
  C:47FDH         LINE#         603
  C:47FDH         LINE#         604
  -------         ENDPROC       UART0RDCMDPROCESS
  -------         PROC          UART0CALIVOLTAGE
  C:6E26H         LINE#         830
  C:6E26H         LINE#         831
  C:6E26H         LINE#         832
  C:6E47H         LINE#         833
  C:6E47H         LINE#         834
  C:6E5AH         LINE#         836
  C:6E5DH         LINE#         837
  C:6E5DH         LINE#         838
  C:6E62H         LINE#         839
BL51 BANKED LINKER/LOCATER V6.22                                                      02/06/2025  15:28:46  PAGE 32


  C:6E63H         LINE#         841
  C:6E63H         LINE#         842
  C:6E65H         LINE#         843
  C:6E6CH         LINE#         844
  C:6E71H         LINE#         845
  C:6E71H         LINE#         846
  C:6E72H         LINE#         848
  C:6E72H         LINE#         849
  C:6E77H         LINE#         850
  C:6E77H         LINE#         851
  -------         ENDPROC       UART0CALIVOLTAGE
  -------         PROC          UART0CALICURRENT
  C:532FH         LINE#         923
  C:532FH         LINE#         924
  C:532FH         LINE#         925
  C:5353H         LINE#         926
  C:5353H         LINE#         930
  C:53BBH         LINE#         932
  C:53D1H         LINE#         933
  C:53D1H         LINE#         934
  C:53D6H         LINE#         935
  C:53D7H         LINE#         937
  C:53D7H         LINE#         938
  C:53D9H         LINE#         939
  C:53E0H         LINE#         940
  C:53E5H         LINE#         941
  C:53E5H         LINE#         942
  C:53E6H         LINE#         944
  C:53E6H         LINE#         945
  C:53EBH         LINE#         946
  C:53EBH         LINE#         947
  -------         ENDPROC       UART0CALICURRENT
  -------         PROC          UART0CALICUROFFSET
  C:7923H         LINE#         950
  C:7923H         LINE#         951
  C:7923H         LINE#         952
  C:7944H         LINE#         953
  C:7944H         LINE#         954
  C:7946H         LINE#         955
  C:794DH         LINE#         957
  C:7952H         LINE#         958
  C:7953H         LINE#         960
  C:7953H         LINE#         961
  C:7958H         LINE#         962
  C:7958H         LINE#         963
  -------         ENDPROC       UART0CALICUROFFSET
  -------         PROC          UART0CALITS1
  C:7266H         LINE#         1073
  C:7266H         LINE#         1074
  C:7266H         LINE#         1075
  C:7287H         LINE#         1076
  C:7287H         LINE#         1077
  C:7289H         LINE#         1078
  C:729CH         LINE#         1079
  C:72A3H         LINE#         1081
  C:72A8H         LINE#         1082
  C:72A9H         LINE#         1084
BL51 BANKED LINKER/LOCATER V6.22                                                      02/06/2025  15:28:46  PAGE 33


  C:72A9H         LINE#         1085
  C:72AEH         LINE#         1086
  C:72AEH         LINE#         1087
  -------         ENDPROC       UART0CALITS1
  -------         PROC          UART0CALITS2
  C:72AFH         LINE#         1090
  C:72AFH         LINE#         1091
  C:72AFH         LINE#         1092
  C:72D0H         LINE#         1093
  C:72D0H         LINE#         1094
  C:72D2H         LINE#         1095
  C:72E5H         LINE#         1096
  C:72ECH         LINE#         1098
  C:72F1H         LINE#         1099
  C:72F2H         LINE#         1101
  C:72F2H         LINE#         1102
  C:72F7H         LINE#         1103
  C:72F7H         LINE#         1104
  -------         ENDPROC       UART0CALITS2
  -------         PROC          UART0CALIRTC
  -------         DO            
  D:0007H         SYMBOL        i
  -------         ENDDO         
  C:6DD2H         LINE#         1196
  C:6DD2H         LINE#         1197
  C:6DD2H         LINE#         1200
  C:6DF3H         LINE#         1201
  C:6DF3H         LINE#         1202
  C:6DF4H         LINE#         1203
  C:6DF4H         LINE#         1204
  C:6E0CH         LINE#         1205
  C:6E11H         LINE#         1206
  C:6E13H         LINE#         1207
  C:6E1AH         LINE#         1208
  C:6E1FH         LINE#         1209
  C:6E20H         LINE#         1211
  C:6E20H         LINE#         1212
  C:6E25H         LINE#         1213
  C:6E25H         LINE#         1214
  -------         ENDPROC       UART0CALIRTC
  -------         PROC          UART0WRCMDPROCESS
  -------         DO            
  X:05F2H         SYMBOL        rdaddr
  -------         ENDDO         
  C:5B07H         LINE#         1280
  C:5B07H         LINE#         1281
  C:5B07H         LINE#         1283
  C:5B33H         LINE#         1284
  C:5B33H         LINE#         1285
  C:5B33H         LINE#         1286
  C:5B36H         LINE#         1287
  C:5B37H         LINE#         1288
  C:5B37H         LINE#         1289
  C:5B3AH         LINE#         1290
  C:5B3BH         LINE#         1291
  C:5B3BH         LINE#         1292
  C:5B3EH         LINE#         1293
BL51 BANKED LINKER/LOCATER V6.22                                                      02/06/2025  15:28:46  PAGE 34


  C:5B3FH         LINE#         1294
  C:5B3FH         LINE#         1295
  C:5B42H         LINE#         1296
  C:5B43H         LINE#         1297
  C:5B43H         LINE#         1298
  C:5B46H         LINE#         1299
  C:5B47H         LINE#         1300
  C:5B47H         LINE#         1301
  C:5B4AH         LINE#         1302
  C:5B4BH         LINE#         1303
  C:5B4BH         LINE#         1304
  C:5B4EH         LINE#         1305
  C:5B4FH         LINE#         1307
  C:5B4FH         LINE#         1308
  C:5B52H         LINE#         1309
  C:5B53H         LINE#         1310
  C:5B53H         LINE#         1311
  C:5B71H         LINE#         1312
  C:5B74H         LINE#         1313
  C:5B75H         LINE#         1314
  C:5B75H         LINE#         1315
  C:5B93H         LINE#         1316
  C:5B96H         LINE#         1317
  C:5B97H         LINE#         1319
  C:5B97H         LINE#         1320
  C:5B9EH         LINE#         1321
  C:5B9EH         LINE#         1322
  C:5BA0H         LINE#         1323
  C:5BA2H         LINE#         1324
  C:5BA7H         LINE#         1325
  C:5BA8H         LINE#         1327
  C:5BA8H         LINE#         1328
  C:5BADH         LINE#         1329
  C:5BADH         LINE#         1330
  C:5BADH         LINE#         1331
  C:5BADH         LINE#         1332
  -------         ENDPROC       UART0WRCMDPROCESS
  -------         PROC          UART0IAPCHECKHANDSHAKE
  -------         DO            
  D:0007H         SYMBOL        i
  D:0007H         SYMBOL        databak
  X:05F4H         SYMBOL        checksum
  -------         ENDDO         
  C:4547H         LINE#         1466
  C:4547H         LINE#         1467
  C:4547H         LINE#         1469
  C:454EH         LINE#         1471
  C:4556H         LINE#         1472
  C:4556H         LINE#         1473
  C:455EH         LINE#         1474
  C:455EH         LINE#         1475
  C:4563H         LINE#         1476
  C:4564H         LINE#         1478
  C:4564H         LINE#         1479
  C:456BH         LINE#         1480
  C:456FH         LINE#         1481
  C:456FH         LINE#         1482
BL51 BANKED LINKER/LOCATER V6.22                                                      02/06/2025  15:28:46  PAGE 35


  C:4570H         LINE#         1484
  C:4570H         LINE#         1485
  C:458BH         LINE#         1486
  C:458BH         LINE#         1487
  C:459EH         LINE#         1488
  C:459EH         LINE#         1489
  C:45B6H         LINE#         1490
  C:45B6H         LINE#         1491
  C:45BEH         LINE#         1492
  C:45BEH         LINE#         1493
  C:45C9H         LINE#         1494
  C:45C9H         LINE#         1495
  C:45CEH         LINE#         1496
  C:45CEH         LINE#         1497
  C:45CFH         LINE#         1498
  C:45D7H         LINE#         1499
  C:45D7H         LINE#         1500
  C:45E2H         LINE#         1501
  C:45E2H         LINE#         1502
  C:45E9H         LINE#         1503
  C:45E9H         LINE#         1504
  C:45E9H         LINE#         1505
  C:45EAH         LINE#         1507
  C:45EAH         LINE#         1508
  C:45EFH         LINE#         1509
  C:461EH         LINE#         1510
  C:461EH         LINE#         1511
  C:4625H         LINE#         1512
  C:4625H         LINE#         1514
  C:462CH         LINE#         1515
  C:462CH         LINE#         1516
  C:4630H         LINE#         1517
  C:4632H         LINE#         1519
  C:4632H         LINE#         1520
  C:4634H         LINE#         1521
  C:4639H         LINE#         1522
  C:4639H         LINE#         1524
  C:463EH         LINE#         1525
  C:4644H         LINE#         1527
  C:4649H         LINE#         1528
  C:464FH         LINE#         1529
  C:4652H         LINE#         1531
  C:466BH         LINE#         1532
  C:466BH         LINE#         1533
  C:4680H         LINE#         1534
  C:4683H         LINE#         1536
  C:4697H         LINE#         1537
  C:46A8H         LINE#         1539
  C:46ADH         LINE#         1540
  C:46ADH         LINE#         1541
  C:46ADH         LINE#         1542
  -------         ENDPROC       UART0IAPCHECKHANDSHAKE
  -------         PROC          _INTERRUPTUART0APPRX
  D:0007H         SYMBOL        RxData
  C:5E2EH         LINE#         1729
  C:5E2EH         LINE#         1730
  C:5E2EH         LINE#         1731
BL51 BANKED LINKER/LOCATER V6.22                                                      02/06/2025  15:28:46  PAGE 36


  C:5E3DH         LINE#         1732
  C:5E43H         LINE#         1733
  C:5E49H         LINE#         1734
  C:5E49H         LINE#         1735
  C:5E4BH         LINE#         1736
  C:5E4BH         LINE#         1737
  C:5E53H         LINE#         1738
  C:5E53H         LINE#         1739
  C:5E5DH         LINE#         1740
  C:5E5DH         LINE#         1741
  C:5E61H         LINE#         1742
  C:5E61H         LINE#         1743
  C:5E63H         LINE#         1744
  C:5E65H         LINE#         1745
  C:5E67H         LINE#         1747
  C:5E67H         LINE#         1748
  C:5E69H         LINE#         1749
  C:5E6BH         LINE#         1750
  C:5E6BH         LINE#         1751
  C:5E6DH         LINE#         1752
  C:5E75H         LINE#         1753
  C:5E75H         LINE#         1754
  C:5E7AH         LINE#         1755
  C:5E7AH         LINE#         1756
  C:5E7AH         LINE#         1758
  C:5E7DH         LINE#         1759
  C:5E7DH         LINE#         1760
  C:5E85H         LINE#         1761
  C:5E85H         LINE#         1762
  C:5E88H         LINE#         1763
  C:5E88H         LINE#         1764
  C:5E8AH         LINE#         1765
  C:5E8DH         LINE#         1766
  C:5E8DH         LINE#         1767
  C:5EA6H         LINE#         1768
  C:5EA6H         LINE#         1769
  C:5EA9H         LINE#         1770
  C:5EABH         LINE#         1771
  C:5EB0H         LINE#         1772
  C:5EB0H         LINE#         1773
  C:5EB2H         LINE#         1775
  C:5EB2H         LINE#         1776
  C:5EB5H         LINE#         1777
  C:5EB5H         LINE#         1778
  C:5EB7H         LINE#         1780
  C:5EBCH         LINE#         1781
  C:5EC0H         LINE#         1782
  C:5EC4H         LINE#         1783
  -------         ENDPROC       _INTERRUPTUART0APPRX
  -------         PROC          INTERRUPTUART0APPTX
  C:59B1H         LINE#         1792
  C:59B1H         LINE#         1793
  C:59B1H         LINE#         1794
  C:59C1H         LINE#         1795
  C:59C1H         LINE#         1796
  C:59DAH         LINE#         1797
  C:59DAH         LINE#         1798
BL51 BANKED LINKER/LOCATER V6.22                                                      02/06/2025  15:28:46  PAGE 37


  C:59DCH         LINE#         1799
  C:59DEH         LINE#         1800
  C:59E0H         LINE#         1801
  C:59E4H         LINE#         1802
  C:59E6H         LINE#         1803
  C:59E8H         LINE#         1804
  C:59EAH         LINE#         1805
  C:59ECH         LINE#         1806
  C:59EEH         LINE#         1808
  C:59EEH         LINE#         1809
  C:59F4H         LINE#         1810
  C:5A03H         LINE#         1811
  C:5A03H         LINE#         1812
  C:5A05H         LINE#         1813
  C:5A22H         LINE#         1814
  C:5A22H         LINE#         1815
  C:5A24H         LINE#         1816
  C:5A29H         LINE#         1817
  C:5A2BH         LINE#         1818
  C:5A2FH         LINE#         1819
  C:5A31H         LINE#         1820
  C:5A33H         LINE#         1821
  C:5A35H         LINE#         1822
  C:5A37H         LINE#         1823
  C:5A39H         LINE#         1825
  C:5A39H         LINE#         1826
  C:5A3FH         LINE#         1827
  C:5A4EH         LINE#         1828
  C:5A4EH         LINE#         1830
  C:5A53H         LINE#         1831
  C:5A57H         LINE#         1832
  C:5A5BH         LINE#         1833
  -------         ENDPROC       INTERRUPTUART0APPTX
  -------         PROC          UART0CHECK
  C:7DECH         LINE#         1842
  C:7DECH         LINE#         1843
  C:7DECH         LINE#         1844
  C:7DF7H         LINE#         1845
  C:7DF7H         LINE#         1846
  C:7DF9H         LINE#         1847
  C:7DFDH         LINE#         1848
  C:7DFFH         LINE#         1849
  C:7DFFH         LINE#         1850
  -------         ENDPROC       UART0CHECK
  -------         ENDMOD        UARTAPP

  -------         MODULE        MEMORY
  C:0000H         SYMBOL        _ICE_DUMMY_
  B:0020H.2       PUBLIC        bOCRC_EN
  X:0024H         PUBLIC        E2uiLearnLowTempe
  D:0080H         PUBLIC        P0
  D:0022H         PUBLIC        uiBatStatus
  D:0090H         PUBLIC        P1
  X:001EH         PUBLIC        E2ulCycleThreshold
  D:00A0H         PUBLIC        P2
  D:00B0H         PUBLIC        P3
  B:0025H.6       PUBLIC        bFastDischarge
BL51 BANKED LINKER/LOCATER V6.22                                                      02/06/2025  15:28:46  PAGE 38


  D:00C0H         PUBLIC        P4
  D:0080H         PUBLIC        P5
  B:0023H.0       PUBLIC        bOV
  X:002AH         PUBLIC        E2ucLowPowerDeley
  B:0023H.1       PUBLIC        bUV
  X:00B3H         PUBLIC        E2ulCycleThresholdCount
  B:0025H.5       PUBLIC        bMidDischarge
  B:0020H.6       PUBLIC        bOCPM
  B:0025H.2       PUBLIC        bCHGING
  X:006DH         PUBLIC        E2slOCCCurrent
  X:00C5H         PUBLIC        E2siTS0Offset
  X:0087H         PUBLIC        E2ucLoadRDelay
  X:00C7H         PUBLIC        E2siTS1Offset
  X:0071H         PUBLIC        E2ucOCCDelay
  X:00ABH         PUBLIC        E2ulDfRC
  B:0025H.4       PUBLIC        bSlowDischarge
  B:0021H.3       PUBLIC        bLEDNum0
  B:0021H.4       PUBLIC        bLEDNum1
  X:00BCH         PUBLIC        E2uiAFEOVvol
  X:002FH         PUBLIC        E2ucRamCheckFlg0
  X:006AH         PUBLIC        E2siChgEndCurr
  X:0061H         PUBLIC        E2ucRamCheckFlg1
  B:0025H.3       PUBLIC        bDSGING
  X:0073H         PUBLIC        E2ucRamCheckFlg2
  X:008CH         PUBLIC        E2ucDSG1PWMRatioH
  X:0088H         PUBLIC        E2ucRamCheckFlg3
  X:0064H         PUBLIC        E2uiOVRvol
  X:002CH         PUBLIC        E2siChgBKCur
  X:00B9H         PUBLIC        E2ucDsgEndFlg
  X:008DH         PUBLIC        E2ucRamCheckFlg5
  X:0053H         PUBLIC        E2ucDeviceChem
  X:0098H         PUBLIC        E2ucRamCheckFlg6
  B:0022H.5       PUBLIC        bAFE_SC
  B:0025H.0       PUBLIC        bCHGMOS
  B:0020H.3       PUBLIC        bBAL_EN
  X:001AH         PUBLIC        E2ulFCC
  X:00A1H         PUBLIC        E2ucRamCheckFlg7
  X:008BH         PUBLIC        E2ucDSG1PWMRatioL
  X:00A9H         PUBLIC        E2ucRamCheckFlg8
  X:00BAH         PUBLIC        E2ucRamCheckFlg9
  X:0076H         PUBLIC        E2uiUVRvol
  X:0047H         PUBLIC        E2ucDeviceName
  X:0090H         PUBLIC        E2uiTempOTCR
  X:009BH         PUBLIC        E2uiTempOTDR
  B:0021H.5       PUBLIC        bTempNum
  X:00C3H         PUBLIC        E2siCadcOffset
  X:0097H         PUBLIC        E2ucTempRDelay
  D:0026H         PUBLIC        ucAFEStatus
  X:00AFH         PUBLIC        E2slDsgEndCurr
  X:0094H         PUBLIC        E2uiTempUTCR
  B:0020H.7       PUBLIC        bEnEEPRomBK
  X:00BFH         PUBLIC        E2uiVPackGain
  X:00BEH         PUBLIC        E2ucRamCheckFlgA
  X:00A4H         PUBLIC        E2uiBalanceVolDiff
  X:009FH         PUBLIC        E2uiTempUTDR
  X:00CAH         PUBLIC        E2ucRamCheckFlgB
  B:0025H.1       PUBLIC        bDSGMOS
BL51 BANKED LINKER/LOCATER V6.22                                                      02/06/2025  15:28:46  PAGE 39


  X:01FEH         PUBLIC        E2uiCheckFlag
  X:00A2H         PUBLIC        E2uiBalanceVol
  B:0022H.4       PUBLIC        bAFE_OV
  X:0068H         PUBLIC        E2uiChgEndVol
  X:00AAH         PUBLIC        E2ucSOC
  X:0035H         PUBLIC        E2ucMNFName
  B:0023H.2       PUBLIC        bOCC
  D:0020H         PUBLIC        uiPackConfig
  X:0067H         PUBLIC        E2ucOVRDelay
  X:002EH         PUBLIC        E2ucRTCBKDelay
  X:0041H         PUBLIC        E2ulMNFDate
  B:0020H.5       PUBLIC        bCTO_EN
  X:00B7H         PUBLIC        E2uiLastCCount
  X:0002H         PUBLIC        E2uiVOC
  X:0079H         PUBLIC        E2ucUVRDelay
  X:007AH         PUBLIC        E2uiDsgEndVol
  X:00C9H         PUBLIC        E2ucCalibrated
  B:0026H.4       PUBLIC        bAfeCHG
  X:00C1H         PUBLIC        E2siCadcGain
  B:0026H.2       PUBLIC        bAfeChging
  X:00CBH         PUBLIC        Reserved
  B:0021H.0       PUBLIC        bCellNum1
  X:007DH         PUBLIC        E2slOCD1Current
  B:0022H.6       PUBLIC        bCTO
  B:0022H.0       PUBLIC        bOTC
  B:0021H.1       PUBLIC        bCellNum2
  X:0082H         PUBLIC        E2slOCD2Current
  B:0022H.1       PUBLIC        bOTD
  B:0021H.2       PUBLIC        bCellNum3
  X:0081H         PUBLIC        E2ucOCD1Delay
  X:0086H         PUBLIC        E2ucOCD2Delay
  X:00A6H         PUBLIC        E2siBalCurrent
  B:0024H.2       PUBLIC        bVDQ
  B:0026H.5       PUBLIC        bAfeDSG
  B:0022H.2       PUBLIC        bUTC
  X:0062H         PUBLIC        E2uiOVvol
  X:0028H         PUBLIC        E2siDfilterCur
  B:0026H.3       PUBLIC        bAfeDsging
  B:0022H.3       PUBLIC        bUTD
  X:0000H         PUBLIC        E2uiPackConfigMap
  X:0074H         PUBLIC        E2uiUVvol
  X:0022H         PUBLIC        E2uiCycleCount
  X:008EH         PUBLIC        E2uiTempOTC
  X:0099H         PUBLIC        E2uiTempOTD
  X:0026H         PUBLIC        E2Reserve
  B:0021H.6       PUBLIC        bChgerLock
  X:0096H         PUBLIC        E2ucTempDelay
  B:0026H.0       PUBLIC        bAfeChger
  X:0092H         PUBLIC        E2uiTempUTC
  X:009DH         PUBLIC        E2uiTempUTD
  X:0034H         PUBLIC        E2ucID
  X:00BBH         PUBLIC        E2ucAFEProtectConfig
  X:0032H         PUBLIC        E2uiHWVersion
  X:005FH         PUBLIC        E2uiChemID
  X:002BH         PUBLIC        E2ucChgBKDelay
  X:0066H         PUBLIC        E2ucOVDelay
  D:0024H         PUBLIC        uiPackStatus
BL51 BANKED LINKER/LOCATER V6.22                                                      02/06/2025  15:28:46  PAGE 40


  B:0023H.3       PUBLIC        bOCD1
  B:0023H.4       PUBLIC        bOCD2
  B:0024H.0       PUBLIC        bFC
  B:0020H.4       PUBLIC        bPF_EN
  X:0072H         PUBLIC        E2ucOCCRDelay
  X:0016H         PUBLIC        E2ulDesignCapacity
  B:0024H.1       PUBLIC        bFD
  B:0020H.0       PUBLIC        bSC_EN
  X:0045H         PUBLIC        E2uiSerialNum
  X:0030H         PUBLIC        E2uiSWVersion
  X:00A8H         PUBLIC        E2ucBalanceDelay
  X:0089H         PUBLIC        E2uiDSG1PWMFreq
  X:0078H         PUBLIC        E2ucUVDelay
  X:006CH         PUBLIC        E2ucChgEndDelay
  B:0021H.7       PUBLIC        bLoadLock
  B:0026H.1       PUBLIC        bAfeLoad
  I:00A0H         PUBLIC        STACK
  B:0020H.1       PUBLIC        bOV_EN
  X:007CH         PUBLIC        E2ucDsgEndDelay
  -------         ENDMOD        MEMORY

  -------         MODULE        AFE
  C:0000H         SYMBOL        _ICE_DUMMY_
  X:0200H         PUBLIC        uiVadcVmax
  D:000FH         PUBLIC        uiCellVmin
  D:0080H         PUBLIC        P0
  D:0011H         PUBLIC        uiCellVmax
  D:0090H         PUBLIC        P1
  D:00A0H         PUBLIC        P2
  D:00B0H         PUBLIC        P3
  C:618AH         PUBLIC        AFEInitReg
  X:0202H         PUBLIC        uiTempeMin
  D:00C0H         PUBLIC        P4
  D:0080H         PUBLIC        P5
  X:0204H         PUBLIC        uiTempeMax
  B:002BH.4       PUBLIC        bCADCFlg
  C:7E99H         PUBLIC        AfeADCEn
  C:7804H         PUBLIC        AFEClrFlg
  C:7D7CH         PUBLIC        AFERdStatus
  D:0013H         PUBLIC        ucCellNum
  X:0206H         PUBLIC        Info
  C:7EF8H         PUBLIC        AfeTempADCDis
  X:023CH         PUBLIC        slCadcCurBuf
  B:002BH.5       PUBLIC        bAfeErr
  B:002BH.6       PUBLIC        bVADCFlg
  C:77C7H         PUBLIC        AFERdFlg
  C:7D94H         PUBLIC        _AfeAlarmDis
  C:7E86H         PUBLIC        AfeWDTDis
  B:002BH.7       PUBLIC        bAfeI2CRWErrFlg
  C:7DC2H         PUBLIC        _AFEMosCtl
  C:7EE5H         PUBLIC        AfeTempADCEn
  X:027CH         PUBLIC        ucTempeMiddle
  C:7F2FH         PUBLIC        _AfeAlarmEn
  C:7E73H         PUBLIC        AfeWDTEn
  X:027DH         PUBLIC        slCadcCurrent
  X:0281H         PUBLIC        slCadcCurAverage
  C:7ED2H         PUBLIC        AfeCADCDis
BL51 BANKED LINKER/LOCATER V6.22                                                      02/06/2025  15:28:46  PAGE 41


  C:7E3AH         PUBLIC        AFEChgerCheckDis
  C:7788H         PUBLIC        _AfeBalCtl
  X:0285H         PUBLIC        AFE
  C:7EBFH         PUBLIC        AfeCADCEn
  C:7E27H         PUBLIC        AFEChgerCheckEn
  C:691FH         PUBLIC        AFERamCheck
  C:7E60H         PUBLIC        AFELoadCheckDis
  D:00C8H         PUBLIC        TWICON
  X:02A3H         PUBLIC        REG
  C:7BBBH         PUBLIC        AFEEnterPD
  C:6103H         PUBLIC        AFEInit
  C:7D62H         PUBLIC        AFETwiCheck
  C:7E4DH         PUBLIC        AFELoadCheckEn
  C:671CH         PUBLIC        _AFEReadReg
  X:02B1H         PUBLIC        ucAfeI2CErrDelayCnt
  X:02B2H         PUBLIC        ucCadcCnt
  C:7EACH         PUBLIC        AfeADCDis
  D:0014H         PUBLIC        ucCellNumOffset
  C:5A5CH         PUBLIC        _AFEWriteReg
  B:002CH.0       PUBLIC        bAfeAlarmFlg
  X:02B3H         PUBLIC        uiVadcVmin
  -------         PROC          AFETWICHECK
  C:7D62H         LINE#         43
  C:7D62H         LINE#         44
  C:7D62H         LINE#         45
  C:7D65H         LINE#         46
  C:7D65H         LINE#         47
  C:7D70H         LINE#         48
  C:7D70H         LINE#         49
  C:7D72H         LINE#         50
  C:7D75H         LINE#         51
  C:7D75H         LINE#         52
  C:7D76H         LINE#         54
  C:7D76H         LINE#         55
  C:7D7BH         LINE#         56
  C:7D7BH         LINE#         57
  -------         ENDPROC       AFETWICHECK
  -------         PROC          _AFEWRITEREG
  X:02BEH         SYMBOL        Reg
  X:02BFH         SYMBOL        Length
  X:02C0H         SYMBOL        WrBuf
  -------         DO            
  B:0029H.6       SYMBOL        Result
  X:02C2H         SYMBOL        Times
  X:02C3H         SYMBOL        i
  -------         ENDDO         
  C:5A5CH         LINE#         67
  C:5A6AH         LINE#         68
  C:5A6AH         LINE#         69
  C:5A6CH         LINE#         70
  C:5A6FH         LINE#         73
  C:5A75H         LINE#         74
  C:5A75H         LINE#         75
  C:5A84H         LINE#         76
  C:5A84H         LINE#         77
  C:5A91H         LINE#         78
  C:5A91H         LINE#         80
BL51 BANKED LINKER/LOCATER V6.22                                                      02/06/2025  15:28:46  PAGE 42


  C:5A91H         LINE#         81
  C:5AB8H         LINE#         82
  C:5AB8H         LINE#         88
  C:5ABBH         LINE#         89
  C:5ABBH         LINE#         90
  C:5ABDH         LINE#         91
  C:5ABFH         LINE#         93
  C:5ABFH         LINE#         94
  C:5AC2H         LINE#         95
  C:5AC7H         LINE#         96
  C:5ACAH         LINE#         97
  C:5ACDH         LINE#         98
  C:5ACDH         LINE#         99
  C:5ACFH         LINE#         100
  C:5AD8H         LINE#         101
  C:5AD8H         LINE#         102
  C:5ADAH         LINE#         103
  C:5ADCH         LINE#         105
  C:5ADCH         LINE#         106
  C:5AE1H         LINE#         107
  C:5AE7H         LINE#         108
  C:5AF1H         LINE#         109
  C:5AF1H         LINE#         110
  C:5AF6H         LINE#         111
  C:5AFFH         LINE#         112
  C:5AFFH         LINE#         113
  C:5B04H         LINE#         115
  C:5B06H         LINE#         116
  -------         ENDPROC       _AFEWRITEREG
  -------         PROC          _AFEREADREG
  X:02C1H         SYMBOL        Reg
  X:02C2H         SYMBOL        Length
  X:02C3H         SYMBOL        RdBuf
  -------         DO            
  B:0029H.6       SYMBOL        Result
  X:02C5H         SYMBOL        Times
  -------         ENDDO         
  C:671CH         LINE#         126
  C:672AH         LINE#         127
  C:672AH         LINE#         128
  C:672CH         LINE#         129
  C:672FH         LINE#         131
  C:6732H         LINE#         132
  C:6732H         LINE#         133
  C:673FH         LINE#         134
  C:673FH         LINE#         136
  C:6768H         LINE#         140
  C:676BH         LINE#         141
  C:676BH         LINE#         142
  C:676DH         LINE#         143
  C:676FH         LINE#         145
  C:676FH         LINE#         146
  C:6772H         LINE#         147
  C:6777H         LINE#         148
  C:677AH         LINE#         149
  C:677DH         LINE#         150
  C:677DH         LINE#         151
BL51 BANKED LINKER/LOCATER V6.22                                                      02/06/2025  15:28:46  PAGE 43


  C:677FH         LINE#         152
  C:677FH         LINE#         153
  C:6784H         LINE#         155
  C:6786H         LINE#         156
  -------         ENDPROC       _AFEREADREG
  -------         PROC          AFECLRFLG
  C:7804H         LINE#         165
  C:7804H         LINE#         166
  C:7804H         LINE#         167
  C:7811H         LINE#         168
  C:7811H         LINE#         169
  C:781BH         LINE#         170
  C:781BH         LINE#         171
  C:7822H         LINE#         172
  C:782DH         LINE#         173
  C:7834H         LINE#         174
  C:783FH         LINE#         175
  C:783FH         LINE#         176
  C:783FH         LINE#         177
  -------         ENDPROC       AFECLRFLG
  -------         PROC          AFEINITREG
  -------         DO            
  D:0004H         SYMBOL        TempVar
  -------         ENDDO         
  C:618AH         LINE#         186
  C:618AH         LINE#         187
  C:618AH         LINE#         190
  C:618FH         LINE#         191
  C:6193H         LINE#         192
  C:6196H         LINE#         193
  C:619AH         LINE#         194
  C:619DH         LINE#         195
  C:619FH         LINE#         196
  C:61A3H         LINE#         197
  C:61A7H         LINE#         198
  C:61ABH         LINE#         199
  C:61AFH         LINE#         200
  C:61B2H         LINE#         202
  C:61B5H         LINE#         203
  C:61B5H         LINE#         204
  C:61BCH         LINE#         205
  C:61CEH         LINE#         206
  C:61CEH         LINE#         207
  C:61D1H         LINE#         208
  C:61D1H         LINE#         209
  C:61D8H         LINE#         210
  C:61EAH         LINE#         211
  C:6207H         LINE#         212
  C:620CH         LINE#         213
  C:620FH         LINE#         214
  C:620FH         LINE#         215
  -------         ENDPROC       AFEINITREG
  -------         PROC          AFEINIT
  -------         DO            
  X:02BAH         SYMBOL        RdBuf
  X:02BCH         SYMBOL        i
  B:0029H.5       SYMBOL        Result
BL51 BANKED LINKER/LOCATER V6.22                                                      02/06/2025  15:28:46  PAGE 44


  X:02BDH         SYMBOL        j
  -------         ENDDO         
  C:6103H         LINE#         225
  C:6103H         LINE#         226
  C:6103H         LINE#         229
  C:6105H         LINE#         230
  C:610BH         LINE#         232
  C:6115H         LINE#         233
  C:6115H         LINE#         234
  C:6122H         LINE#         235
  C:6122H         LINE#         236
  C:6132H         LINE#         237
  C:6132H         LINE#         238
  C:613BH         LINE#         240
  C:6169H         LINE#         241
  C:6169H         LINE#         242
  C:6171H         LINE#         243
  C:6171H         LINE#         244
  C:6173H         LINE#         245
  C:6175H         LINE#         246
  C:6175H         LINE#         247
  C:6175H         LINE#         248
  C:617EH         LINE#         249
  C:617EH         LINE#         251
  C:617EH         LINE#         252
  C:6180H         LINE#         253
  C:6180H         LINE#         254
  C:6183H         LINE#         255
  C:6183H         LINE#         256
  C:6185H         LINE#         257
  C:6185H         LINE#         258
  C:6187H         LINE#         259
  C:6189H         LINE#         261
  -------         ENDPROC       AFEINIT
  -------         PROC          AFERDFLG
  C:77C7H         LINE#         272
  C:77C7H         LINE#         273
  C:77C7H         LINE#         274
  C:77D4H         LINE#         275
  C:77D4H         LINE#         276
  C:77DCH         LINE#         277
  C:77DCH         LINE#         278
  C:77DEH         LINE#         279
  C:77DEH         LINE#         281
  C:77E2H         LINE#         282
  C:77E2H         LINE#         283
  C:77E4H         LINE#         284
  C:77E4H         LINE#         286
  C:77EFH         LINE#         287
  C:77EFH         LINE#         288
  C:77F1H         LINE#         289
  C:77F3H         LINE#         290
  C:77F3H         LINE#         291
  C:77F7H         LINE#         292
  C:77F7H         LINE#         293
  C:77F9H         LINE#         294
  C:77F9H         LINE#         296
BL51 BANKED LINKER/LOCATER V6.22                                                      02/06/2025  15:28:46  PAGE 45


  C:7800H         LINE#         297
  C:7800H         LINE#         298
  C:7803H         LINE#         299
  C:7803H         LINE#         300
  C:7803H         LINE#         301
  -------         ENDPROC       AFERDFLG
  -------         PROC          AFERDSTATUS
  -------         DO            
  X:02B7H         SYMBOL        RegTemp
  -------         ENDDO         
  C:7D7CH         LINE#         310
  C:7D7CH         LINE#         311
  C:7D7CH         LINE#         313
  C:7D89H         LINE#         314
  C:7D89H         LINE#         315
  C:7D93H         LINE#         316
  C:7D93H         LINE#         317
  -------         ENDPROC       AFERDSTATUS
  -------         PROC          AFERAMCHECK
  -------         DO            
  X:02B7H         SYMBOL        RdBuf
  X:02B9H         SYMBOL        i
  -------         ENDDO         
  C:691FH         LINE#         326
  C:691FH         LINE#         327
  C:691FH         LINE#         331
  C:692FH         LINE#         332
  C:692FH         LINE#         333
  C:6938H         LINE#         335
  C:6966H         LINE#         336
  C:6966H         LINE#         337
  C:696EH         LINE#         338
  C:696EH         LINE#         339
  C:6973H         LINE#         340
  C:6973H         LINE#         341
  C:6975H         LINE#         342
  C:6975H         LINE#         343
  C:6976H         LINE#         344
  C:6976H         LINE#         345
  C:6976H         LINE#         346
  C:697FH         LINE#         347
  -------         ENDPROC       AFERAMCHECK
  -------         PROC          AFEENTERPD
  C:7BBBH         LINE#         356
  C:7BBBH         LINE#         357
  C:7BBBH         LINE#         358
  C:7BC1H         LINE#         359
  C:7BCEH         LINE#         360
  C:7BCEH         LINE#         361
  C:7BD5H         LINE#         362
  C:7BE0H         LINE#         363
  C:7BE0H         LINE#         364
  -------         ENDPROC       AFEENTERPD
  -------         PROC          _AFEMOSCTL
  D:0007H         SYMBOL        MosStatus
  C:7DC2H         LINE#         373
  C:7DC2H         LINE#         374
BL51 BANKED LINKER/LOCATER V6.22                                                      02/06/2025  15:28:46  PAGE 46


  C:7DC2H         LINE#         375
  C:7DC9H         LINE#         376
  C:7DCBH         LINE#         377
  C:7DD6H         LINE#         378
  -------         ENDPROC       _AFEMOSCTL
  -------         PROC          AFECHGERCHECKEN
  C:7E27H         LINE#         388
  C:7E27H         LINE#         389
  C:7E27H         LINE#         390
  C:7E2EH         LINE#         391
  C:7E39H         LINE#         392
  -------         ENDPROC       AFECHGERCHECKEN
  -------         PROC          AFECHGERCHECKDIS
  C:7E3AH         LINE#         395
  C:7E3AH         LINE#         396
  C:7E3AH         LINE#         397
  C:7E41H         LINE#         398
  C:7E4CH         LINE#         399
  -------         ENDPROC       AFECHGERCHECKDIS
  -------         PROC          AFELOADCHECKEN
  C:7E4DH         LINE#         402
  C:7E4DH         LINE#         403
  C:7E4DH         LINE#         404
  C:7E54H         LINE#         405
  C:7E5FH         LINE#         406
  -------         ENDPROC       AFELOADCHECKEN
  -------         PROC          AFELOADCHECKDIS
  C:7E60H         LINE#         409
  C:7E60H         LINE#         410
  C:7E60H         LINE#         411
  C:7E67H         LINE#         412
  C:7E72H         LINE#         413
  -------         ENDPROC       AFELOADCHECKDIS
  -------         PROC          _AFEBALCTL
  X:02B9H         SYMBOL        BalChTemp
  C:7788H         LINE#         422
  C:7790H         LINE#         423
  C:7790H         LINE#         424
  C:77A4H         LINE#         425
  C:77B1H         LINE#         426
  C:77B1H         LINE#         427
  C:77BBH         LINE#         428
  C:77C6H         LINE#         429
  C:77C6H         LINE#         430
  -------         ENDPROC       _AFEBALCTL
  -------         PROC          AFEWDTEN
  C:7E73H         LINE#         439
  C:7E73H         LINE#         440
  C:7E73H         LINE#         441
  C:7E7AH         LINE#         442
  C:7E85H         LINE#         443
  -------         ENDPROC       AFEWDTEN
  -------         PROC          AFEWDTDIS
  C:7E86H         LINE#         446
  C:7E86H         LINE#         447
  C:7E86H         LINE#         448
  C:7E8DH         LINE#         449
BL51 BANKED LINKER/LOCATER V6.22                                                      02/06/2025  15:28:46  PAGE 47


  C:7E98H         LINE#         450
  -------         ENDPROC       AFEWDTDIS
  -------         PROC          AFEADCEN
  C:7E99H         LINE#         459
  C:7E99H         LINE#         460
  C:7E99H         LINE#         461
  C:7EA0H         LINE#         462
  C:7EABH         LINE#         463
  -------         ENDPROC       AFEADCEN
  -------         PROC          AFEADCDIS
  C:7EACH         LINE#         466
  C:7EACH         LINE#         467
  C:7EACH         LINE#         468
  C:7EB3H         LINE#         469
  C:7EBEH         LINE#         470
  -------         ENDPROC       AFEADCDIS
  -------         PROC          AFECADCEN
  C:7EBFH         LINE#         472
  C:7EBFH         LINE#         473
  C:7EBFH         LINE#         474
  C:7EC6H         LINE#         475
  C:7ED1H         LINE#         476
  -------         ENDPROC       AFECADCEN
  -------         PROC          AFECADCDIS
  C:7ED2H         LINE#         479
  C:7ED2H         LINE#         480
  C:7ED2H         LINE#         481
  C:7ED9H         LINE#         482
  C:7EE4H         LINE#         483
  -------         ENDPROC       AFECADCDIS
  -------         PROC          AFETEMPADCEN
  C:7EE5H         LINE#         485
  C:7EE5H         LINE#         486
  C:7EE5H         LINE#         487
  C:7EECH         LINE#         488
  C:7EF7H         LINE#         489
  -------         ENDPROC       AFETEMPADCEN
  -------         PROC          AFETEMPADCDIS
  C:7EF8H         LINE#         492
  C:7EF8H         LINE#         493
  C:7EF8H         LINE#         494
  C:7EFFH         LINE#         495
  C:7F0AH         LINE#         496
  -------         ENDPROC       AFETEMPADCDIS
  -------         PROC          _AFEALARMEN
  D:0007H         SYMBOL        AlarmFlg
  C:7F2FH         LINE#         505
  C:7F2FH         LINE#         506
  C:7F2FH         LINE#         507
  C:7F35H         LINE#         508
  C:7F40H         LINE#         509
  -------         ENDPROC       _AFEALARMEN
  -------         PROC          _AFEALARMDIS
  D:0007H         SYMBOL        AlarmFlg
  C:7D94H         LINE#         511
  C:7D94H         LINE#         512
  C:7D94H         LINE#         513
BL51 BANKED LINKER/LOCATER V6.22                                                      02/06/2025  15:28:46  PAGE 48


  C:7D9FH         LINE#         514
  C:7DAAH         LINE#         515
  -------         ENDPROC       _AFEALARMDIS
  -------         ENDMOD        AFE

  -------         MODULE        BALANCE
  C:0000H         SYMBOL        _ICE_DUMMY_
  D:0080H         PUBLIC        P0
  D:0090H         PUBLIC        P1
  D:00A0H         PUBLIC        P2
  B:002CH.1       PUBLIC        bBalancingFlg
  D:00B0H         PUBLIC        P3
  D:00C0H         PUBLIC        P4
  B:002CH.2       PUBLIC        bCellOpenDecFlag
  D:0080H         PUBLIC        P5
  C:7F77H         PUBLIC        BalanceProcess
  X:0536H         PUBLIC        ucBalanceStep
  X:0537H         PUBLIC        ucCellOpenDecCnt
  X:0538H         PUBLIC        ucCtoCnt
  B:002CH.3       PUBLIC        bBalanceFlg
  C:7BE1H         PUBLIC        CTOTurnOnCheck
  X:0539H         PUBLIC        ucBalanceTimeCnt
  B:002CH.4       PUBLIC        bBalanceOddFlg
  X:053AH         PUBLIC        uiBalanceChannel
  B:002CH.5       PUBLIC        bCTOValidFlg
  C:4945H         PUBLIC        BalTurnOnCheck
  C:5798H         PUBLIC        BalProcess
  C:7959H         PUBLIC        CTOCheckVol
  -------         PROC          BALTURNONCHECK
  -------         DO            
  D:0005H         SYMBOL        i
  -------         ENDDO         
  C:4945H         LINE#         32
  C:4945H         LINE#         33
  C:4945H         LINE#         36
  C:4951H         LINE#         37
  C:4951H         LINE#         38
  C:4957H         LINE#         39
  C:4957H         LINE#         40
  C:495EH         LINE#         41
  C:498EH         LINE#         44
  C:498EH         LINE#         45
  C:4990H         LINE#         46
  C:4995H         LINE#         47
  C:4996H         LINE#         49
  C:4996H         LINE#         50
  C:49E0H         LINE#         51
  C:49E0H         LINE#         52
  C:49E3H         LINE#         53
  C:49E3H         LINE#         54
  C:49E9H         LINE#         55
  C:49E9H         LINE#         56
  C:4A05H         LINE#         57
  C:4A05H         LINE#         58
  C:4A1BH         LINE#         59
  C:4A1BH         LINE#         60
  C:4A60H         LINE#         61
BL51 BANKED LINKER/LOCATER V6.22                                                      02/06/2025  15:28:46  PAGE 49


  C:4A60H         LINE#         62
  C:4A7BH         LINE#         63
  C:4A7BH         LINE#         64
  C:4A7EH         LINE#         65
  C:4A80H         LINE#         66
  C:4A80H         LINE#         67
  C:4A81H         LINE#         69
  C:4A81H         LINE#         70
  C:4A83H         LINE#         71
  C:4A88H         LINE#         72
  C:4A88H         LINE#         73
  C:4A88H         LINE#         74
  C:4A88H         LINE#         75
  C:4A88H         LINE#         76
  -------         ENDPROC       BALTURNONCHECK
  -------         PROC          CTOCHECKVOL
  -------         DO            
  B:0029H.5       SYMBOL        bResult
  -------         ENDDO         
  C:7959H         LINE#         87
  C:7959H         LINE#         88
  C:7959H         LINE#         89
  C:795BH         LINE#         91
  C:795EH         LINE#         92
  C:795EH         LINE#         93
  C:7961H         LINE#         94
  C:7961H         LINE#         95
  C:7964H         LINE#         96
  C:7964H         LINE#         97
  C:7973H         LINE#         98
  C:7973H         LINE#         99
  C:7975H         LINE#         100
  C:7980H         LINE#         101
  C:7980H         LINE#         102
  C:7982H         LINE#         103
  C:7982H         LINE#         104
  C:7984H         LINE#         106
  C:7984H         LINE#         107
  C:7986H         LINE#         108
  C:798BH         LINE#         109
  C:798BH         LINE#         110
  C:798BH         LINE#         111
  C:798BH         LINE#         128
  C:798BH         LINE#         130
  C:798DH         LINE#         131
  -------         ENDPROC       CTOCHECKVOL
  -------         PROC          BALPROCESS
  -------         DO            
  X:02B7H         SYMBOL        BalChTemp
  -------         ENDDO         
  C:5798H         LINE#         144
  C:5798H         LINE#         145
  C:5798H         LINE#         150
  C:57B6H         LINE#         151
  C:57B6H         LINE#         152
  C:57B8H         LINE#         153
  C:57B8H         LINE#         155
BL51 BANKED LINKER/LOCATER V6.22                                                      02/06/2025  15:28:46  PAGE 50


  C:57D0H         LINE#         156
  C:57D0H         LINE#         157
  C:57D0H         LINE#         158
  C:57D6H         LINE#         159
  C:57D6H         LINE#         160
  C:57D9H         LINE#         161
  C:57D9H         LINE#         162
  C:57ECH         LINE#         163
  C:57EEH         LINE#         165
  C:57EEH         LINE#         166
  C:5801H         LINE#         167
  C:5801H         LINE#         168
  C:580CH         LINE#         169
  C:5812H         LINE#         170
  C:5814H         LINE#         171
  C:5814H         LINE#         172
  C:5815H         LINE#         174
  C:5815H         LINE#         175
  C:581BH         LINE#         176
  C:581CH         LINE#         178
  C:581CH         LINE#         179
  C:5821H         LINE#         180
  C:5821H         LINE#         181
  C:5827H         LINE#         182
  C:582DH         LINE#         183
  C:582FH         LINE#         184
  C:582FH         LINE#         185
  C:5830H         LINE#         187
  C:5830H         LINE#         188
  C:5835H         LINE#         189
  C:5835H         LINE#         190
  C:583BH         LINE#         191
  C:583CH         LINE#         193
  C:583CH         LINE#         194
  C:5842H         LINE#         195
  C:5844H         LINE#         196
  C:5844H         LINE#         197
  C:5845H         LINE#         199
  C:5845H         LINE#         200
  C:584BH         LINE#         201
  C:584DH         LINE#         202
  C:584FH         LINE#         203
  C:5851H         LINE#         204
  C:5851H         LINE#         205
  C:5851H         LINE#         206
  -------         ENDPROC       BALPROCESS
  -------         PROC          CTOTURNONCHECK
  C:7BE1H         LINE#         215
  C:7BE1H         LINE#         216
  C:7BE1H         LINE#         220
  C:7BE7H         LINE#         222
  C:7BE7H         LINE#         223
  C:7BF2H         LINE#         224
  C:7BF2H         LINE#         225
  C:7BF5H         LINE#         226
  C:7BF8H         LINE#         227
  C:7BF8H         LINE#         228
BL51 BANKED LINKER/LOCATER V6.22                                                      02/06/2025  15:28:46  PAGE 51


  C:7BFAH         LINE#         229
  C:7BFCH         LINE#         230
  C:7C06H         LINE#         231
  C:7C06H         LINE#         232
  C:7C06H         LINE#         233
  C:7C06H         LINE#         234
  -------         ENDPROC       CTOTURNONCHECK
  -------         PROC          BALANCEPROCESS
  C:7F77H         LINE#         242
  C:7F77H         LINE#         243
  C:7F77H         LINE#         244
  C:7F7AH         LINE#         246
  C:7F7DH         LINE#         248
  C:7F80H         LINE#         249
  -------         ENDPROC       BALANCEPROCESS
  -------         ENDMOD        BALANCE

  -------         MODULE        CALCULATE
  C:0000H         SYMBOL        _ICE_DUMMY_
  C:5852H         PUBLIC        OffsetCalculate
  D:0080H         PUBLIC        P0
  D:0090H         PUBLIC        P1
  D:00A0H         PUBLIC        P2
  D:00B0H         PUBLIC        P3
  C:380CH         PUBLIC        _CalcuTemp
  D:00C0H         PUBLIC        P4
  D:0080H         PUBLIC        P5
  C:79F8H         PUBLIC        siCurTempOffset
  C:40EFH         PUBLIC        AfeCalcuCurr
  C:4BCBH         PUBLIC        AfeCalcuVol
  C:7389H         PUBLIC        AfeGetTempe
  X:05F6H         PUBLIC        ucChgingCheckCnt
  C:7E00H         PUBLIC        AFEInfoProcess
  X:05F7H         PUBLIC        ucDsgingCheckCnt
  B:00A8H.4       PUBLIC        ES0
  C:71D2H         PUBLIC        AfeGetVol
  C:4F22H         PUBLIC        AfeCalcuTempe
  -------         PROC          _CALCUTEMP
  D:0082H         SYMBOL        getdata
  -------         DO            
  X:02B7H         SYMBOL        i
  X:02B8H         SYMBOL        Temperature
  X:02BAH         SYMBOL        Tempcalcu
  -------         ENDDO         
  C:380CH         LINE#         22
  C:3810H         LINE#         23
  C:3810H         LINE#         31
  C:383EH         LINE#         32
  C:3850H         LINE#         33
  C:3850H         LINE#         34
  C:386DH         LINE#         35
  C:386DH         LINE#         38
  C:3886H         LINE#         39
  C:3886H         LINE#         40
  C:3890H         LINE#         41
  C:3893H         LINE#         42
  C:38ACH         LINE#         43
BL51 BANKED LINKER/LOCATER V6.22                                                      02/06/2025  15:28:46  PAGE 52


  C:38ACH         LINE#         44
  C:38B6H         LINE#         45
  C:38B9H         LINE#         47
  C:38B9H         LINE#         48
  C:38C1H         LINE#         49
  C:38E0H         LINE#         50
  C:38E0H         LINE#         51
  C:38F3H         LINE#         52
  C:38F3H         LINE#         53
  C:3913H         LINE#         54
  C:3913H         LINE#         55
  C:3913H         LINE#         56
  C:3913H         LINE#         57
  C:391BH         LINE#         58
  C:391BH         LINE#         60
  C:391BH         LINE#         61
  C:392EH         LINE#         62
  C:392EH         LINE#         63
  C:394EH         LINE#         64
  C:394EH         LINE#         65
  C:394EH         LINE#         66
  C:394EH         LINE#         67
  C:3956H         LINE#         68
  C:395CH         LINE#         69
  C:395CH         LINE#         70
  C:3964H         LINE#         72
  C:39F3H         LINE#         73
  C:39F3H         LINE#         74
  C:39FBH         LINE#         75
  -------         ENDPROC       _CALCUTEMP
  -------         PROC          AFEGETVOL
  -------         DO            
  X:02C0H         SYMBOL        i
  B:0029H.5       SYMBOL        Result
  -------         ENDDO         
  C:71D2H         LINE#         84
  C:71D2H         LINE#         85
  C:71D2H         LINE#         87
  C:71D4H         LINE#         89
  C:71F1H         LINE#         90
  C:71F1H         LINE#         91
  C:720CH         LINE#         92
  C:720CH         LINE#         93
  C:720EH         LINE#         94
  C:7211H         LINE#         95
  C:7211H         LINE#         96
  C:7219H         LINE#         98
  C:721BH         LINE#         99
  -------         ENDPROC       AFEGETVOL
  -------         PROC          AFEGETTEMPE
  -------         DO            
  B:0029H.5       SYMBOL        Result
  -------         ENDDO         
  C:7389H         LINE#         101
  C:7389H         LINE#         102
  C:7389H         LINE#         103
  C:738BH         LINE#         105
BL51 BANKED LINKER/LOCATER V6.22                                                      02/06/2025  15:28:46  PAGE 53


  C:7398H         LINE#         106
  C:7398H         LINE#         107
  C:739AH         LINE#         108
  C:739AH         LINE#         109
  C:73A7H         LINE#         110
  C:73A7H         LINE#         111
  C:73A9H         LINE#         112
  C:73A9H         LINE#         114
  C:73B6H         LINE#         115
  C:73B6H         LINE#         116
  C:73B8H         LINE#         117
  C:73B8H         LINE#         118
  C:73BFH         LINE#         119
  C:73BFH         LINE#         120
  C:73CCH         LINE#         121
  C:73CCH         LINE#         122
  C:73CEH         LINE#         123
  C:73CEH         LINE#         124
  C:73CEH         LINE#         126
  C:73D0H         LINE#         127
  -------         ENDPROC       AFEGETTEMPE
  -------         PROC          AFECALCUTEMPE
  -------         DO            
  D:0006H         SYMBOL        TempeData
  -------         ENDDO         
  C:4F22H         LINE#         136
  C:4F22H         LINE#         137
  C:4F22H         LINE#         140
  C:4F2AH         LINE#         141
  C:4F2AH         LINE#         142
  C:4F41H         LINE#         144
  C:4F43H         LINE#         152
  C:4F4AH         LINE#         154
  C:4F4CH         LINE#         162
  C:4F6BH         LINE#         164
  C:4F6DH         LINE#         172
  C:4F74H         LINE#         175
  C:4F76H         LINE#         184
  C:4F7DH         LINE#         185
  C:4F7DH         LINE#         186
  C:4F9CH         LINE#         188
  C:4F9EH         LINE#         196
  C:4FA5H         LINE#         198
  C:4FA7H         LINE#         206
  C:4FA7H         LINE#         208
  C:4FB7H         LINE#         209
  C:4FBFH         LINE#         210
  C:4FC2H         LINE#         211
  C:4FC2H         LINE#         212
  C:4FD9H         LINE#         214
  C:4FDBH         LINE#         222
  C:4FE2H         LINE#         224
  C:4FE4H         LINE#         233
  C:4FF1H         LINE#         234
  C:4FF1H         LINE#         235
  C:4FF6H         LINE#         236
  C:4FF7H         LINE#         238
BL51 BANKED LINKER/LOCATER V6.22                                                      02/06/2025  15:28:46  PAGE 54


  C:4FF7H         LINE#         239
  C:4FFFH         LINE#         240
  C:4FFFH         LINE#         241
  C:4FFFH         LINE#         242
  C:4FFFH         LINE#         243
  -------         ENDPROC       AFECALCUTEMPE
  -------         PROC          AFECALCUVOL
  -------         DO            
  X:02B7H         SYMBOL        i
  X:02B8H         SYMBOL        TempPackVol
  X:02BCH         SYMBOL        TempCellVol
  -------         ENDDO         
  C:4BCBH         LINE#         253
  C:4BCBH         LINE#         254
  C:4BCBH         LINE#         256
  C:4BDFH         LINE#         257
  C:4BE6H         LINE#         258
  C:4BF0H         LINE#         260
  C:4BF8H         LINE#         261
  C:4BF8H         LINE#         262
  C:4C19H         LINE#         263
  C:4C19H         LINE#         264
  C:4C50H         LINE#         266
  C:4C67H         LINE#         267
  C:4C67H         LINE#         268
  C:4C75H         LINE#         269
  C:4C75H         LINE#         270
  C:4C8CH         LINE#         271
  C:4C8CH         LINE#         272
  C:4C9AH         LINE#         273
  C:4C9AH         LINE#         275
  C:4C9DH         LINE#         276
  C:4C9DH         LINE#         278
  C:4C9FH         LINE#         286
  C:4CB9H         LINE#         288
  C:4CBBH         LINE#         296
  C:4CD0H         LINE#         297
  C:4CD0H         LINE#         298
  C:4CD9H         LINE#         300
  C:4CDCH         LINE#         301
  C:4CDCH         LINE#         302
  C:4CE6H         LINE#         303
  C:4CF0H         LINE#         306
  C:4CF2H         LINE#         314
  C:4D00H         LINE#         316
  C:4D02H         LINE#         324
  C:4D02H         LINE#         325
  C:4D02H         LINE#         326
  -------         ENDPROC       AFECALCUVOL
  -------         PROC          OFFSETCALCULATE
  -------         DO            
  X:02BCH         SYMBOL        siCadcTempOffset
  X:02BEH         SYMBOL        i
  -------         ENDDO         
  C:5852H         LINE#         347
  C:5852H         LINE#         348
  C:5852H         LINE#         349
BL51 BANKED LINKER/LOCATER V6.22                                                      02/06/2025  15:28:46  PAGE 55


  C:5859H         LINE#         352
  C:5868H         LINE#         353
  C:5868H         LINE#         354
  C:58D4H         LINE#         355
  C:58D4H         LINE#         356
  C:58F1H         LINE#         357
  C:58F3H         LINE#         358
  C:58F3H         LINE#         359
  C:58FCH         LINE#         360
  C:5904H         LINE#         361
  -------         ENDPROC       OFFSETCALCULATE
  -------         PROC          AFECALCUCURR
  -------         DO            
  X:02B7H         SYMBOL        i
  X:02B8H         SYMBOL        Tempdata
  -------         ENDDO         
  C:40EFH         LINE#         369
  C:40EFH         LINE#         370
  C:40EFH         LINE#         372
  C:40F9H         LINE#         374
  C:4104H         LINE#         376
  C:4110H         LINE#         377
  C:4110H         LINE#         378
  C:4119H         LINE#         379
  C:4119H         LINE#         380
  C:4168H         LINE#         382
  C:4182H         LINE#         383
  C:418DH         LINE#         384
  C:418DH         LINE#         385
  C:418FH         LINE#         386
  C:418FH         LINE#         387
  C:419EH         LINE#         388
  C:419EH         LINE#         389
  C:41BCH         LINE#         390
  C:41C4H         LINE#         391
  C:41D9H         LINE#         393
  C:41DBH         LINE#         394
  C:41DDH         LINE#         395
  C:41FDH         LINE#         396
  C:41FDH         LINE#         397
  C:4208H         LINE#         398
  C:4208H         LINE#         399
  C:420BH         LINE#         400
  C:420DH         LINE#         402
  C:420FH         LINE#         410
  C:421BH         LINE#         412
  C:421DH         LINE#         420
  C:421DH         LINE#         421
  C:421EH         LINE#         422
  C:4238H         LINE#         423
  C:4238H         LINE#         424
  C:4242H         LINE#         425
  C:4242H         LINE#         426
  C:4245H         LINE#         427
  C:4247H         LINE#         428
  C:4250H         LINE#         430
  C:4252H         LINE#         438
BL51 BANKED LINKER/LOCATER V6.22                                                      02/06/2025  15:28:46  PAGE 56


  C:425EH         LINE#         440
  C:4260H         LINE#         448
  C:4260H         LINE#         449
  C:4261H         LINE#         451
  C:4261H         LINE#         453
  C:4263H         LINE#         461
  C:426DH         LINE#         463
  C:426FH         LINE#         471
  C:426FH         LINE#         472
  -------         ENDPROC       AFECALCUCURR
  -------         PROC          AFEINFOPROCESS
  C:7E00H         LINE#         481
  C:7E00H         LINE#         482
  C:7E00H         LINE#         483
  C:7E03H         LINE#         485
  C:7E05H         LINE#         486
  C:7E08H         LINE#         487
  C:7E0BH         LINE#         489
  C:7E0EH         LINE#         490
  C:7E0EH         LINE#         491
  C:7E10H         LINE#         492
  C:7E13H         LINE#         493
  C:7E13H         LINE#         494
  -------         ENDPROC       AFEINFOPROCESS
  -------         ENDMOD        CALCULATE

  -------         MODULE        CALIBRATE
  C:0000H         SYMBOL        _ICE_DUMMY_
  D:0080H         PUBLIC        P0
  D:0090H         PUBLIC        P1
  D:00A0H         PUBLIC        P2
  D:00B0H         PUBLIC        P3
  D:00C0H         PUBLIC        P4
  D:0080H         PUBLIC        P5
  X:05D6H         PUBLIC        slExtCur
  C:7F41H         PUBLIC        CaliCurZero
  X:05DAH         PUBLIC        ucExtcaliSwitch1
  C:6643H         PUBLIC        CaliVoltage
  C:7534H         PUBLIC        CaliTS1
  C:7579H         PUBLIC        CaliTS2
  X:05DBH         PUBLIC        uiExtTemp1
  X:05DDH         PUBLIC        uiExtTemp2
  C:6EC9H         PUBLIC        CaliProcess
  C:7840H         PUBLIC        CaliCurrentGain
  X:05DFH         PUBLIC        ulExtVPack
  X:05E1H         PUBLIC        ucExtRTC
  C:75BEH         PUBLIC        CaliRTCTime
  B:002FH.4       PUBLIC        bCaliFlg
  -------         PROC          CALIVOLTAGE
  -------         DO            
  D:0007H         SYMBOL        i
  X:02B7H         SYMBOL        VPackTemp
  -------         ENDDO         
  C:6643H         LINE#         26
  C:6643H         LINE#         27
  C:6643H         LINE#         29
  C:664AH         LINE#         31
BL51 BANKED LINKER/LOCATER V6.22                                                      02/06/2025  15:28:46  PAGE 57


  C:6662H         LINE#         32
  C:6662H         LINE#         33
  C:667CH         LINE#         34
  C:667FH         LINE#         36
  C:66AFH         LINE#         37
  -------         ENDPROC       CALIVOLTAGE
  -------         PROC          CALICURRENTGAIN
  -------         DO            
  D:0006H         SYMBOL        TempGain
  -------         ENDDO         
  C:7840H         LINE#         46
  C:7840H         LINE#         47
  C:7840H         LINE#         50
  C:786EH         LINE#         51
  C:7872H         LINE#         52
  C:7872H         LINE#         53
  C:787AH         LINE#         54
  C:787AH         LINE#         55
  -------         ENDPROC       CALICURRENTGAIN
  -------         PROC          CALICURZERO
  C:7F41H         LINE#         64
  C:7F41H         LINE#         65
  C:7F41H         LINE#         66
  C:7F50H         LINE#         67
  -------         ENDPROC       CALICURZERO
  -------         PROC          CALITS1
  -------         DO            
  D:0006H         SYMBOL        Tempe
  -------         ENDDO         
  C:7534H         LINE#         76
  C:7534H         LINE#         77
  C:7534H         LINE#         80
  C:754CH         LINE#         81
  C:7570H         LINE#         82
  C:7570H         LINE#         83
  C:7578H         LINE#         84
  C:7578H         LINE#         85
  -------         ENDPROC       CALITS1
  -------         PROC          CALITS2
  -------         DO            
  D:0006H         SYMBOL        Tempe
  -------         ENDDO         
  C:7579H         LINE#         87
  C:7579H         LINE#         88
  C:7579H         LINE#         91
  C:7591H         LINE#         92
  C:75B5H         LINE#         93
  C:75B5H         LINE#         94
  C:75BDH         LINE#         95
  C:75BDH         LINE#         96
  -------         ENDPROC       CALITS2
  -------         PROC          CALIRTCTIME
  C:75BEH         LINE#         106
  C:75BEH         LINE#         107
  C:75BEH         LINE#         108
  C:75C6H         LINE#         109
  C:75CEH         LINE#         110
BL51 BANKED LINKER/LOCATER V6.22                                                      02/06/2025  15:28:46  PAGE 58


  C:75D6H         LINE#         111
  C:75DEH         LINE#         112
  C:75E6H         LINE#         113
  C:75EEH         LINE#         114
  C:75F6H         LINE#         116
  C:75FDH         LINE#         118
  C:75FFH         LINE#         119
  C:7601H         LINE#         120
  -------         ENDPROC       CALIRTCTIME
  -------         PROC          CALIPROCESS
  C:6EC9H         LINE#         131
  C:6EC9H         LINE#         132
  C:6EC9H         LINE#         133
  C:6ECCH         LINE#         134
  C:6ECCH         LINE#         135
  C:6ECEH         LINE#         137
  C:6ED5H         LINE#         138
  C:6ED5H         LINE#         139
  C:6ED8H         LINE#         140
  C:6ED8H         LINE#         142
  C:6EDFH         LINE#         143
  C:6EDFH         LINE#         144
  C:6EE2H         LINE#         145
  C:6EE2H         LINE#         147
  C:6EE9H         LINE#         148
  C:6EE9H         LINE#         149
  C:6EECH         LINE#         150
  C:6EECH         LINE#         152
  C:6EF3H         LINE#         153
  C:6EF3H         LINE#         154
  C:6EF6H         LINE#         155
  C:6EF6H         LINE#         157
  C:6EFDH         LINE#         158
  C:6EFDH         LINE#         159
  C:6F00H         LINE#         160
  C:6F00H         LINE#         162
  C:6F07H         LINE#         163
  C:6F07H         LINE#         164
  C:6F0AH         LINE#         165
  C:6F0AH         LINE#         167
  C:6F0FH         LINE#         168
  C:6F11H         LINE#         169
  C:6F17H         LINE#         170
  C:6F17H         LINE#         171
  -------         ENDPROC       CALIPROCESS
  -------         ENDMOD        CALIBRATE

  -------         MODULE        CHARGERLOAD
  C:0000H         SYMBOL        _ICE_DUMMY_
  D:0080H         PUBLIC        P0
  D:0090H         PUBLIC        P1
  D:00A0H         PUBLIC        P2
  D:00B0H         PUBLIC        P3
  D:00C0H         PUBLIC        P4
  D:0080H         PUBLIC        P5
  X:05F8H         PUBLIC        ucChgerRCnt
  B:002DH.2       PUBLIC        bChgerChkingFlg
BL51 BANKED LINKER/LOCATER V6.22                                                      02/06/2025  15:28:46  PAGE 59


  C:72F8H         PUBLIC        ChgerCheck
  X:05F9H         PUBLIC        ucLoadRCnt
  B:002DH.3       PUBLIC        bLoadChkingFlg
  B:002DH.4       PUBLIC        bChgerStartCheckFlg
  C:7054H         PUBLIC        LoadCheck
  B:002DH.5       PUBLIC        bLoadStartCheckFlg
  -------         PROC          LOADCHECK
  C:7054H         LINE#         26
  C:7054H         LINE#         27
  C:7054H         LINE#         28
  C:7057H         LINE#         29
  C:7057H         LINE#         30
  C:7059H         LINE#         31
  C:705BH         LINE#         32
  C:7060H         LINE#         33
  C:7063H         LINE#         34
  C:7064H         LINE#         35
  C:7067H         LINE#         36
  C:7067H         LINE#         37
  C:706AH         LINE#         38
  C:706DH         LINE#         39
  C:706DH         LINE#         40
  C:7089H         LINE#         41
  C:7089H         LINE#         42
  C:708BH         LINE#         43
  C:708DH         LINE#         44
  C:7090H         LINE#         45
  C:7093H         LINE#         46
  C:7093H         LINE#         47
  C:7095H         LINE#         48
  C:7095H         LINE#         49
  C:7097H         LINE#         50
  C:7099H         LINE#         51
  C:709CH         LINE#         52
  C:709CH         LINE#         53
  C:709EH         LINE#         54
  C:70A1H         LINE#         55
  C:70A1H         LINE#         56
  C:70A1H         LINE#         57
  C:70A1H         LINE#         58
  C:70A1H         LINE#         59
  -------         ENDPROC       LOADCHECK
  -------         PROC          CHGERCHECK
  C:72F8H         LINE#         68
  C:72F8H         LINE#         69
  C:72F8H         LINE#         70
  C:72FBH         LINE#         71
  C:72FBH         LINE#         72
  C:72FDH         LINE#         73
  C:72FFH         LINE#         74
  C:7304H         LINE#         75
  C:7307H         LINE#         76
  C:7308H         LINE#         77
  C:730BH         LINE#         78
  C:730BH         LINE#         79
  C:730EH         LINE#         80
  C:7311H         LINE#         81
BL51 BANKED LINKER/LOCATER V6.22                                                      02/06/2025  15:28:46  PAGE 60


  C:7311H         LINE#         82
  C:732DH         LINE#         83
  C:732DH         LINE#         84
  C:732FH         LINE#         85
  C:7331H         LINE#         86
  C:7334H         LINE#         87
  C:7337H         LINE#         88
  C:7337H         LINE#         89
  C:7339H         LINE#         90
  C:733BH         LINE#         91
  C:733EH         LINE#         92
  C:733EH         LINE#         93
  C:7340H         LINE#         94
  C:7340H         LINE#         95
  C:7340H         LINE#         96
  C:7340H         LINE#         97
  -------         ENDPROC       CHGERCHECK
  -------         ENDMOD        CHARGERLOAD

  -------         MODULE        EXTE2PROM
  C:0000H         SYMBOL        _ICE_DUMMY_
  C:6787H         PUBLIC        Uart0RdE2PRom
  C:64F6H         PUBLIC        Uart1RdE2PRom
  D:0080H         PUBLIC        P0
  C:6565H         PUBLIC        Uart2RdE2PRom
  D:0090H         PUBLIC        P1
  D:00A0H         PUBLIC        P2
  C:3F3CH         PUBLIC        _E2PRomBKData
  D:00B0H         PUBLIC        P3
  D:00C0H         PUBLIC        P4
  D:0080H         PUBLIC        P5
  C:69E1H         PUBLIC        _E2PRomWrite
  C:6393H         PUBLIC        E2PRomInit
  C:7CEFH         PUBLIC        E2PRomTwiCheck
  X:03DAH         PUBLIC        ucRTCBKTime1
  B:00A0H.4       PUBLIC        REN1
  B:0090H.4       PUBLIC        REN2
  X:03DBH         PUBLIC        uiRTCBKTime2
  C:7688H         PUBLIC        E2PRomBKBoot
  B:0027H.0       PUBLIC        bE2PErase
  X:03DDH         PUBLIC        uiE2PDataAddr
  B:0027H.1       PUBLIC        bE2PRErr
  B:0027H.2       PUBLIC        bE2PProcessFlg
  X:03DFH         PUBLIC        bUart0E2PRdData
  X:03E0H         PUBLIC        bUart1E2PRdData
  X:03E1H         PUBLIC        bUart2E2PRdData
  I:001EH         PUBLIC        ucUpDataLimitTime
  D:0099H         PUBLIC        SBUF
  X:03E2H         PUBLIC        uiCHGValidTime
  D:00B1H         PUBLIC        RSTSTAT
  X:03E4H         PUBLIC        ucE2PTwiRWErrDelayCnt
  D:0086H         PUBLIC        INSCON
  B:0027H.3       PUBLIC        bE2PTwiRWErrFlg
  B:0027H.4       PUBLIC        bE2PBKChgStart
  X:03E5H         PUBLIC        ucRTCBuf
  D:00A1H         PUBLIC        SBUF1
  B:0027H.5       PUBLIC        bE2PBKRtc
BL51 BANKED LINKER/LOCATER V6.22                                                      02/06/2025  15:28:46  PAGE 61


  D:0091H         PUBLIC        SBUF2
  X:03ECH         PUBLIC        bUart0RTCRdTime
  B:0027H.6       PUBLIC        bE2PBKDsgEndValid
  B:0098H.4       PUBLIC        REN
  X:03EDH         PUBLIC        bUart1RTCRdTime
  C:50D7H         PUBLIC        E2PRomBKCheck
  X:03EEH         PUBLIC        bUart2RTCRdTime
  C:5905H         PUBLIC        E2PRomBKProcess
  C:66B0H         PUBLIC        E2PRomErase
  C:74A9H         PUBLIC        Uart0RdRTC
  C:70EEH         PUBLIC        E2PRomBKRTC
  C:713AH         PUBLIC        Uart1RdRTC
  B:0027H.7       PUBLIC        bE2PBKDsgEnd
  C:7186H         PUBLIC        Uart2RdRTC
  B:0028H.0       PUBLIC        bChgToDsgFlg
  B:0028H.1       PUBLIC        bDsgToChgFlg
  B:0028H.2       PUBLIC        bE2PBKChgStop
  C:6A40H         PUBLIC        _E2PRomRead
  -------         PROC          E2PROMTWICHECK
  C:7CEFH         LINE#         43
  C:7CEFH         LINE#         44
  C:7CEFH         LINE#         45
  C:7CF2H         LINE#         46
  C:7CF2H         LINE#         47
  C:7CF5H         LINE#         48
  C:7CF5H         LINE#         49
  C:7D00H         LINE#         50
  C:7D00H         LINE#         51
  C:7D02H         LINE#         52
  C:7D05H         LINE#         53
  C:7D05H         LINE#         54
  C:7D06H         LINE#         56
  C:7D06H         LINE#         57
  C:7D0BH         LINE#         58
  C:7D0BH         LINE#         59
  C:7D0BH         LINE#         60
  -------         ENDPROC       E2PROMTWICHECK
  -------         PROC          _E2PROMWRITE
  X:02E1H         SYMBOL        WrAddr
  X:02E3H         SYMBOL        Length
  X:02E4H         SYMBOL        WrBuf
  -------         DO            
  B:0029H.5       SYMBOL        Result
  X:02E6H         SYMBOL        i
  -------         ENDDO         
  C:69E1H         LINE#         69
  C:69F2H         LINE#         70
  C:69F2H         LINE#         71
  C:69F4H         LINE#         74
  C:69F7H         LINE#         75
  C:69F7H         LINE#         76
  C:69FAH         LINE#         77
  C:69FAH         LINE#         79
  C:6A23H         LINE#         80
  C:6A23H         LINE#         81
  C:6A25H         LINE#         82
  C:6A27H         LINE#         83
BL51 BANKED LINKER/LOCATER V6.22                                                      02/06/2025  15:28:46  PAGE 62


  C:6A27H         LINE#         91
  C:6A2CH         LINE#         92
  C:6A38H         LINE#         93
  C:6A38H         LINE#         94
  C:6A3DH         LINE#         96
  C:6A3FH         LINE#         97
  -------         ENDPROC       _E2PROMWRITE
  -------         PROC          _E2PROMREAD
  X:02C3H         SYMBOL        RdAddr
  X:02C5H         SYMBOL        Length
  X:02C6H         SYMBOL        RdBuf
  -------         DO            
  B:0029H.6       SYMBOL        Result
  X:02C8H         SYMBOL        i
  -------         ENDDO         
  C:6A40H         LINE#         106
  C:6A51H         LINE#         107
  C:6A51H         LINE#         108
  C:6A53H         LINE#         111
  C:6A56H         LINE#         112
  C:6A56H         LINE#         113
  C:6A59H         LINE#         114
  C:6A59H         LINE#         116
  C:6A82H         LINE#         117
  C:6A82H         LINE#         118
  C:6A84H         LINE#         119
  C:6A86H         LINE#         120
  C:6A86H         LINE#         128
  C:6A8BH         LINE#         129
  C:6A97H         LINE#         130
  C:6A97H         LINE#         131
  C:6A9CH         LINE#         133
  C:6A9EH         LINE#         134
  -------         ENDPROC       _E2PROMREAD
  -------         PROC          E2PROMERASE
  -------         DO            
  X:02B8H         SYMBOL        i
  X:02BAH         SYMBOL        WrBuf
  -------         ENDDO         
  C:66B0H         LINE#         144
  C:66B0H         LINE#         145
  C:66B0H         LINE#         149
  C:66BBH         LINE#         151
  C:66D9H         LINE#         152
  C:66D9H         LINE#         153
  C:66DCH         LINE#         154
  C:66FBH         LINE#         155
  C:6707H         LINE#         157
  C:6714H         LINE#         158
  C:671BH         LINE#         159
  -------         ENDPROC       E2PROMERASE
  -------         PROC          E2PROMINIT
  -------         DO            
  B:0029H.5       SYMBOL        Result
  X:02B7H         SYMBOL        RdBuf
  -------         ENDDO         
  C:6393H         LINE#         168
BL51 BANKED LINKER/LOCATER V6.22                                                      02/06/2025  15:28:46  PAGE 63


  C:6393H         LINE#         169
  C:6393H         LINE#         170
  C:6395H         LINE#         174
  C:63A4H         LINE#         176
  C:63B2H         LINE#         177
  C:63C0H         LINE#         179
  C:63CCH         LINE#         180
  C:63CCH         LINE#         181
  C:63E1H         LINE#         182
  C:63E3H         LINE#         183
  C:63EFH         LINE#         184
  C:63EFH         LINE#         185
  C:6404H         LINE#         186
  C:6406H         LINE#         188
  C:6406H         LINE#         189
  C:640DH         LINE#         190
  C:640DH         LINE#         192
  C:640FH         LINE#         193
  -------         ENDPROC       E2PROMINIT
  -------         PROC          E2PROMBKRTC
  -------         DO            
  X:02B8H         SYMBOL        WrBuf
  D:0007H         SYMBOL        i
  X:02C1H         SYMBOL        checksum
  -------         ENDDO         
  C:70EEH         LINE#         202
  C:70EEH         LINE#         203
  C:70EEH         LINE#         205
  C:70F3H         LINE#         207
  C:70FAH         LINE#         208
  C:7107H         LINE#         209
  C:7109H         LINE#         210
  C:7109H         LINE#         211
  C:711BH         LINE#         212
  C:7120H         LINE#         213
  C:7128H         LINE#         214
  C:712CH         LINE#         216
  C:7139H         LINE#         217
  -------         ENDPROC       E2PROMBKRTC
  -------         PROC          E2PROMBKBOOT
  -------         DO            
  X:02D9H         SYMBOL        WrBuf
  -------         ENDDO         
  C:7688H         LINE#         226
  C:7688H         LINE#         227
  C:7688H         LINE#         230
  C:7695H         LINE#         231
  C:769AH         LINE#         232
  C:76A3H         LINE#         234
  C:76ABH         LINE#         235
  C:76B3H         LINE#         236
  C:76BBH         LINE#         238
  C:76C8H         LINE#         239
  -------         ENDPROC       E2PROMBKBOOT
  -------         PROC          _E2PROMBKDATA
  X:02B8H         SYMBOL        BKType
  -------         DO            
BL51 BANKED LINKER/LOCATER V6.22                                                      02/06/2025  15:28:46  PAGE 64


  X:02B9H         SYMBOL        WrBuf
  -------         ENDDO         
  C:3F3CH         LINE#         248
  C:3F41H         LINE#         249
  C:3F41H         LINE#         252
  C:3F45H         LINE#         253
  C:3F45H         LINE#         254
  C:3F52H         LINE#         255
  C:3F5DH         LINE#         256
  C:3F5FH         LINE#         258
  C:3F5FH         LINE#         259
  C:3F66H         LINE#         260
  C:3F73H         LINE#         261
  C:3F7EH         LINE#         262
  C:3F7EH         LINE#         264
  C:3F8BH         LINE#         265
  C:3F8EH         LINE#         266
  C:3F9BH         LINE#         267
  C:3F9EH         LINE#         268
  C:3FAEH         LINE#         269
  C:3FBEH         LINE#         270
  C:3FCEH         LINE#         271
  C:3FD9H         LINE#         272
  C:3FE9H         LINE#         273
  C:3FF9H         LINE#         274
  C:4009H         LINE#         275
  C:4014H         LINE#         276
  C:402BH         LINE#         277
  C:403BH         LINE#         278
  C:4048H         LINE#         279
  C:404BH         LINE#         280
  C:405BH         LINE#         281
  C:406BH         LINE#         282
  C:407BH         LINE#         283
  C:4086H         LINE#         284
  C:4093H         LINE#         285
  C:4096H         LINE#         286
  C:40A3H         LINE#         287
  C:40A6H         LINE#         288
  C:40AEH         LINE#         289
  C:40B2H         LINE#         291
  C:40C3H         LINE#         293
  C:40CDH         LINE#         294
  C:40E4H         LINE#         295
  C:40E4H         LINE#         296
  C:40EBH         LINE#         297
  C:40EBH         LINE#         299
  C:40EEH         LINE#         300
  -------         ENDPROC       _E2PROMBKDATA
  -------         PROC          UART0RDE2PROM
  -------         DO            
  D:0006H         SYMBOL        RdAddr
  -------         ENDDO         
  C:6787H         LINE#         309
  C:6787H         LINE#         310
  C:6787H         LINE#         313
  C:67B2H         LINE#         314
BL51 BANKED LINKER/LOCATER V6.22                                                      02/06/2025  15:28:46  PAGE 65


  C:67BEH         LINE#         316
  C:67DDH         LINE#         317
  C:67EFH         LINE#         318
  -------         ENDPROC       UART0RDE2PROM
  -------         PROC          UART1RDE2PROM
  -------         DO            
  D:0006H         SYMBOL        RdAddr
  -------         ENDDO         
  C:64F6H         LINE#         326
  C:64F6H         LINE#         327
  C:64F6H         LINE#         330
  C:6521H         LINE#         331
  C:652DH         LINE#         333
  C:654CH         LINE#         334
  C:6564H         LINE#         335
  -------         ENDPROC       UART1RDE2PROM
  -------         PROC          UART2RDE2PROM
  -------         DO            
  D:0006H         SYMBOL        RdAddr
  -------         ENDDO         
  C:6565H         LINE#         343
  C:6565H         LINE#         344
  C:6565H         LINE#         347
  C:6590H         LINE#         348
  C:659CH         LINE#         350
  C:65BBH         LINE#         351
  C:65D3H         LINE#         352
  -------         ENDPROC       UART2RDE2PROM
  -------         PROC          UART0RDRTC
  C:74A9H         LINE#         361
  C:74A9H         LINE#         362
  C:74A9H         LINE#         363
  C:74B0H         LINE#         364
  C:74BDH         LINE#         366
  C:74DCH         LINE#         367
  C:74EEH         LINE#         368
  -------         ENDPROC       UART0RDRTC
  -------         PROC          UART1RDRTC
  C:713AH         LINE#         377
  C:713AH         LINE#         378
  C:713AH         LINE#         379
  C:7141H         LINE#         380
  C:714EH         LINE#         382
  C:716DH         LINE#         383
  C:7185H         LINE#         384
  -------         ENDPROC       UART1RDRTC
  -------         PROC          UART2RDRTC
  C:7186H         LINE#         392
  C:7186H         LINE#         393
  C:7186H         LINE#         394
  C:718DH         LINE#         395
  C:719AH         LINE#         397
  C:71B9H         LINE#         398
  C:71D1H         LINE#         399
  -------         ENDPROC       UART2RDRTC
  -------         PROC          E2PROMBKPROCESS
  -------         DO            
BL51 BANKED LINKER/LOCATER V6.22                                                      02/06/2025  15:28:46  PAGE 66


  X:02B7H         SYMBOL        BKType
  -------         ENDDO         
  C:5905H         LINE#         407
  C:5905H         LINE#         408
  C:5905H         LINE#         411
  C:5911H         LINE#         412
  C:5911H         LINE#         413
  C:5913H         LINE#         417
  C:5916H         LINE#         418
  C:5916H         LINE#         419
  C:5918H         LINE#         420
  C:591BH         LINE#         421
  C:591BH         LINE#         423
  C:592AH         LINE#         424
  C:592AH         LINE#         425
  C:592DH         LINE#         426
  C:592DH         LINE#         427
  C:5932H         LINE#         428
  C:5935H         LINE#         429
  C:5935H         LINE#         430
  C:593BH         LINE#         431
  C:593BH         LINE#         432
  C:593DH         LINE#         433
  C:5940H         LINE#         434
  C:5940H         LINE#         435
  C:5946H         LINE#         436
  C:5946H         LINE#         437
  C:5948H         LINE#         438
  C:594BH         LINE#         439
  C:594BH         LINE#         441
  C:594BH         LINE#         443
  C:595AH         LINE#         444
  C:595AH         LINE#         445
  C:595DH         LINE#         446
  C:595DH         LINE#         447
  C:5962H         LINE#         448
  C:5965H         LINE#         449
  C:5965H         LINE#         450
  C:596BH         LINE#         451
  C:596BH         LINE#         452
  C:596DH         LINE#         453
  C:5970H         LINE#         454
  C:5970H         LINE#         455
  C:5976H         LINE#         456
  C:5976H         LINE#         457
  C:5978H         LINE#         458
  C:597BH         LINE#         459
  C:597BH         LINE#         460
  C:597BH         LINE#         462
  C:597EH         LINE#         463
  C:597EH         LINE#         464
  C:5980H         LINE#         465
  C:5983H         LINE#         466
  C:5983H         LINE#         468
  C:5986H         LINE#         469
  C:5986H         LINE#         470
  C:5988H         LINE#         471
BL51 BANKED LINKER/LOCATER V6.22                                                      02/06/2025  15:28:46  PAGE 67


  C:598EH         LINE#         472
  C:5992H         LINE#         473
  C:5992H         LINE#         475
  C:5995H         LINE#         476
  C:5995H         LINE#         477
  C:5997H         LINE#         478
  C:599DH         LINE#         479
  C:59A1H         LINE#         480
  C:59A1H         LINE#         482
  C:59A4H         LINE#         483
  C:59A4H         LINE#         484
  C:59A6H         LINE#         485
  C:59ACH         LINE#         486
  C:59B0H         LINE#         487
  C:59B0H         LINE#         488
  C:59B0H         LINE#         489
  -------         ENDPROC       E2PROMBKPROCESS
  -------         PROC          E2PROMBKCHECK
  C:50D7H         LINE#         498
  C:50D7H         LINE#         499
  C:50D7H         LINE#         500
  C:50DDH         LINE#         501
  C:50DDH         LINE#         505
  C:50ECH         LINE#         506
  C:50ECH         LINE#         507
  C:50EEH         LINE#         508
  C:50F5H         LINE#         509
  C:50F5H         LINE#         511
  C:510AH         LINE#         512
  C:510AH         LINE#         513
  C:5111H         LINE#         514
  C:5113H         LINE#         515
  C:5115H         LINE#         516
  C:5115H         LINE#         518
  C:5118H         LINE#         519
  C:5118H         LINE#         520
  C:511AH         LINE#         521
  C:511DH         LINE#         522
  C:511DH         LINE#         523
  C:511FH         LINE#         524
  C:5121H         LINE#         525
  C:5123H         LINE#         526
  C:5123H         LINE#         527
  C:5129H         LINE#         528
  C:5129H         LINE#         529
  C:512BH         LINE#         530
  C:512DH         LINE#         531
  C:512FH         LINE#         532
  C:5131H         LINE#         533
  C:5134H         LINE#         534
  C:5134H         LINE#         535
  C:5136H         LINE#         536
  C:5136H         LINE#         537
  C:5136H         LINE#         539
  C:5153H         LINE#         540
  C:5153H         LINE#         541
  C:515DH         LINE#         542
BL51 BANKED LINKER/LOCATER V6.22                                                      02/06/2025  15:28:46  PAGE 68


  C:515DH         LINE#         543
  C:5164H         LINE#         544
  C:5171H         LINE#         545
  C:5171H         LINE#         547
  C:5192H         LINE#         548
  C:5192H         LINE#         549
  C:5199H         LINE#         550
  C:519BH         LINE#         551
  C:519DH         LINE#         552
  C:519FH         LINE#         553
  C:51A1H         LINE#         554
  C:51A1H         LINE#         555
  C:51A2H         LINE#         557
  C:51A2H         LINE#         558
  C:51A9H         LINE#         559
  C:51A9H         LINE#         560
  C:51A9H         LINE#         561
  -------         ENDPROC       E2PROMBKCHECK
  -------         ENDMOD        EXTE2PROM

  -------         MODULE        INTERRUPT
  C:0000H         SYMBOL        _ICE_DUMMY_
  D:0080H         PUBLIC        P0
  D:0090H         PUBLIC        P1
  D:00A0H         PUBLIC        P2
  D:00B0H         PUBLIC        P3
  D:00C0H         PUBLIC        P4
  D:0080H         PUBLIC        P5
  C:1003H         PUBLIC        InterruptTimer3
  D:0086H         PUBLIC        INSCON
  B:0088H.7       PUBLIC        TF3
  B:00D8H.0       PUBLIC        IF40
  C:65D4H         PUBLIC        InterruptINT4
  B:00D8H.1       PUBLIC        IF41
  B:00D8H.2       PUBLIC        IF42
  B:00D8H.3       PUBLIC        IF43
  B:00D8H.4       PUBLIC        IF44
  B:00D8H.5       PUBLIC        IF45
  B:00D8H.6       PUBLIC        IF46
  B:00D8H.7       PUBLIC        IF47
  -------         PROC          INTERRUPTINT4
  C:65D4H         LINE#         18
  C:65E1H         LINE#         20
  C:65E3H         LINE#         21
  C:65E6H         LINE#         23
  C:65E9H         LINE#         24
  C:65E9H         LINE#         25
  C:65EBH         LINE#         26
  C:65F0H         LINE#         27
  C:65F0H         LINE#         28
  C:65F3H         LINE#         29
  C:65F3H         LINE#         30
  C:65F5H         LINE#         31
  C:65FAH         LINE#         32
  C:65FAH         LINE#         33
  C:65FDH         LINE#         34
  C:65FDH         LINE#         35
BL51 BANKED LINKER/LOCATER V6.22                                                      02/06/2025  15:28:46  PAGE 69


  C:65FFH         LINE#         36
  C:6604H         LINE#         37
  C:6604H         LINE#         38
  C:6607H         LINE#         39
  C:6607H         LINE#         40
  C:6609H         LINE#         41
  C:660EH         LINE#         42
  C:660EH         LINE#         43
  C:6611H         LINE#         44
  C:6611H         LINE#         45
  C:6613H         LINE#         46
  C:6618H         LINE#         47
  C:6618H         LINE#         48
  C:661BH         LINE#         49
  C:661BH         LINE#         50
  C:661DH         LINE#         51
  C:6622H         LINE#         52
  C:6622H         LINE#         53
  C:6625H         LINE#         54
  C:6625H         LINE#         55
  C:6627H         LINE#         56
  C:662CH         LINE#         57
  C:662CH         LINE#         58
  C:662FH         LINE#         59
  C:662FH         LINE#         60
  C:6631H         LINE#         61
  C:6636H         LINE#         62
  C:6636H         LINE#         64
  C:6638H         LINE#         65
  -------         ENDPROC       INTERRUPTINT4
  -------         PROC          INTERRUPTTIMER3
  C:1003H         LINE#         74
  C:100BH         LINE#         76
  C:100DH         LINE#         78
  C:1010H         LINE#         79
  C:1012H         LINE#         80
  C:1015H         LINE#         82
  C:1018H         LINE#         84
  C:101AH         LINE#         85
  -------         ENDPROC       INTERRUPTTIMER3
  -------         ENDMOD        INTERRUPT

  -------         MODULE        KEYSCAN
  C:0000H         SYMBOL        _ICE_DUMMY_
  D:0080H         PUBLIC        P0
  D:0090H         PUBLIC        P1
  D:00A0H         PUBLIC        P2
  D:00B0H         PUBLIC        P3
  D:00C0H         PUBLIC        P4
  D:0008H         PUBLIC        ucKeyValue
  D:0080H         PUBLIC        P5
  D:0009H         PUBLIC        ucKeyValueBK
  B:00B0H.0       PUBLIC        P3_0
  B:00A0H.7       PUBLIC        P2_7
  D:000AH         PUBLIC        uiKeyValidCnt
  D:000CH         PUBLIC        ucKeyOldValue
  B:002FH.5       PUBLIC        bKeyFlg
BL51 BANKED LINKER/LOCATER V6.22                                                      02/06/2025  15:28:46  PAGE 70


  C:5BAEH         PUBLIC        KeyScan
  D:000DH         PUBLIC        uiKeyInvalidCnt
  -------         PROC          KEYSCAN
  -------         DO            
  C:5C43H         SYMBOL        scanend
  -------         ENDDO         
  C:5BAEH         LINE#         33
  C:5BAEH         LINE#         34
  C:5BAEH         LINE#         35
  C:5BB4H         LINE#         36
  C:5BB4H         LINE#         37
  C:5BB7H         LINE#         46
  C:5BBAH         LINE#         47
  C:5BBAH         LINE#         48
  C:5BBDH         LINE#         49
  C:5BBFH         LINE#         50
  C:5BC2H         LINE#         51
  C:5BC2H         LINE#         52
  C:5BC5H         LINE#         53
  C:5BC5H         LINE#         69
  C:5BCBH         LINE#         70
  C:5BCBH         LINE#         71
  C:5BD3H         LINE#         72
  C:5BDEH         LINE#         73
  C:5BDEH         LINE#         74
  C:5BE8H         LINE#         75
  C:5BE8H         LINE#         76
  C:5BF2H         LINE#         77
  C:5BF2H         LINE#         78
  C:5BF8H         LINE#         79
  C:5BFAH         LINE#         81
  C:5BFAH         LINE#         82
  C:5BFDH         LINE#         83
  C:5BFDH         LINE#         84
  C:5BFFH         LINE#         85
  C:5C01H         LINE#         86
  C:5C01H         LINE#         91
  C:5C01H         LINE#         93
  C:5C01H         LINE#         94
  C:5C03H         LINE#         95
  C:5C03H         LINE#         96
  C:5C03H         LINE#         98
  C:5C03H         LINE#         99
  C:5C09H         LINE#         100
  C:5C09H         LINE#         101
  C:5C0EH         LINE#         102
  C:5C16H         LINE#         103
  C:5C1EH         LINE#         104
  C:5C1EH         LINE#         105
  C:5C24H         LINE#         106
  C:5C26H         LINE#         107
  C:5C27H         LINE#         108
  C:5C31H         LINE#         109
  C:5C31H         LINE#         110
  C:5C37H         LINE#         111
  C:5C3DH         LINE#         112
  C:5C3FH         LINE#         113
BL51 BANKED LINKER/LOCATER V6.22                                                      02/06/2025  15:28:46  PAGE 71


  C:5C3FH         LINE#         114
  C:5C40H         LINE#         116
  C:5C40H         LINE#         117
  C:5C43H         LINE#         118
  C:5C43H         LINE#         119
  C:5C48H         LINE#         120
  C:5C4CH         LINE#         121
  C:5C4FH         LINE#         122
  C:5C4FH         LINE#         123
  C:5C4FH         LINE#         124
  C:5C4FH         LINE#         125
  -------         ENDPROC       KEYSCAN
  -------         ENDMOD        KEYSCAN

  -------         MODULE        MCUFLASH
  C:0000H         SYMBOL        _ICE_DUMMY_
  D:00F3H         PUBLIC        IB_CON2
  D:0080H         PUBLIC        P0
  D:00F4H         PUBLIC        IB_CON3
  D:0090H         PUBLIC        P1
  D:00F5H         PUBLIC        IB_CON4
  D:00A0H         PUBLIC        P2
  D:00F6H         PUBLIC        IB_CON5
  D:00B0H         PUBLIC        P3
  D:00C0H         PUBLIC        P4
  X:05FAH         PUBLIC        bMcuFlashWrWaitCnt
  D:0080H         PUBLIC        P5
  B:00A8H.7       PUBLIC        EA
  D:00FCH         PUBLIC        IB_DATA
  C:7B6DH         PUBLIC        _McuFlashCheckFlg
  C:6A9FH         PUBLIC        _McuFlashRead
  C:798EH         PUBLIC        _McuFlashWrOneByte
  B:002EH.1       PUBLIC        bMcuFlashErr
  C:5EC5H         PUBLIC        _McuFlashWrite
  X:05FBH         PUBLIC        ucMcuFlashWrValid
  D:00FBH         PUBLIC        IB_OFFSET
  D:00B1H         PUBLIC        RSTSTAT
  D:00A7H         PUBLIC        FLASHCON
  C:6077H         PUBLIC        _McuFlashWrSector
  C:7DD7H         PUBLIC        McuFlashWrWaitCheck
  B:002EH.2       PUBLIC        bMcuFlashWrFlg
  C:7C07H         PUBLIC        _McuFlashBlankCheck
  C:6C6DH         PUBLIC        _McuFlashDataCheck
  D:00F7H         PUBLIC        XPAGE
  B:002EH.3       PUBLIC        bMcuFlashWrWaitFlg
  C:526EH         PUBLIC        McuFlashProcess
  D:00F2H         PUBLIC        IB_CON1
  -------         PROC          _MCUFLASHWRONEBYTE
  D:0002H         SYMBOL        McuFlashAddr
  D:0005H         SYMBOL        WrData
  C:798EH         LINE#         24
  C:7992H         LINE#         25
  C:7992H         LINE#         26
  C:7994H         LINE#         27
  C:7997H         LINE#         29
  C:799AH         LINE#         30
  C:799EH         LINE#         31
BL51 BANKED LINKER/LOCATER V6.22                                                      02/06/2025  15:28:46  PAGE 72


  C:79A2H         LINE#         33
  C:79A5H         LINE#         34
  C:79A8H         LINE#         35
  C:79ABH         LINE#         36
  C:79AEH         LINE#         37
  C:79B5H         LINE#         38
  C:79B5H         LINE#         39
  C:79B8H         LINE#         40
  C:79B9H         LINE#         41
  C:79BAH         LINE#         42
  C:79BBH         LINE#         43
  C:79BCH         LINE#         44
  C:79BDH         LINE#         45
  C:79BDH         LINE#         47
  C:79C0H         LINE#         48
  C:79C2H         LINE#         49
  -------         ENDPROC       _MCUFLASHWRONEBYTE
  -------         PROC          _MCUFLASHBLANKCHECK
  D:0006H         SYMBOL        McuFlashAddr
  -------         DO            
  B:002AH.0       SYMBOL        Result
  D:0004H         SYMBOL        i
  -------         ENDDO         
  C:7C07H         LINE#         58
  C:7C07H         LINE#         59
  C:7C07H         LINE#         60
  C:7C09H         LINE#         63
  C:7C0CH         LINE#         64
  C:7C0CH         LINE#         65
  C:7C19H         LINE#         66
  C:7C19H         LINE#         67
  C:7C1BH         LINE#         68
  C:7C1DH         LINE#         69
  C:7C1DH         LINE#         70
  C:7C2AH         LINE#         72
  C:7C2CH         LINE#         73
  -------         ENDPROC       _MCUFLASHBLANKCHECK
  -------         PROC          _MCUFLASHDATACHECK
  X:02BDH         SYMBOL        McuFlashAddr
  D:0004H         SYMBOL        XramAddr
  -------         DO            
  B:002AH.0       SYMBOL        Result
  D:0006H         SYMBOL        ptr
  X:02BFH         SYMBOL        i
  -------         ENDDO         
  C:6C6DH         LINE#         82
  C:6C75H         LINE#         83
  C:6C75H         LINE#         84
  C:6C77H         LINE#         85
  C:6C7BH         LINE#         88
  C:6C8EH         LINE#         89
  C:6C8EH         LINE#         90
  C:6CB4H         LINE#         91
  C:6CB4H         LINE#         92
  C:6CB6H         LINE#         93
  C:6CB8H         LINE#         94
  C:6CB8H         LINE#         95
BL51 BANKED LINKER/LOCATER V6.22                                                      02/06/2025  15:28:46  PAGE 73


  C:6CC4H         LINE#         97
  C:6CC6H         LINE#         98
  -------         ENDPROC       _MCUFLASHDATACHECK
  -------         PROC          _MCUFLASHWRSECTOR
  X:02BDH         SYMBOL        McuFlashAddr
  D:0004H         SYMBOL        XramAddr
  -------         DO            
  B:002AH.0       SYMBOL        Result
  D:0004H         SYMBOL        i
  X:02BFH         SYMBOL        ptr
  -------         ENDDO         
  C:6077H         LINE#         107
  C:607FH         LINE#         108
  C:607FH         LINE#         109
  C:6081H         LINE#         111
  C:6089H         LINE#         113
  C:608CH         LINE#         114
  C:608CH         LINE#         115
  C:6097H         LINE#         116
  C:609DH         LINE#         117
  C:60ACH         LINE#         118
  C:60AFH         LINE#         119
  C:60B2H         LINE#         120
  C:60B2H         LINE#         121
  C:60B5H         LINE#         122
  C:60B9H         LINE#         123
  C:60B9H         LINE#         124
  C:60BCH         LINE#         125
  C:60C4H         LINE#         126
  C:60C4H         LINE#         127
  C:60C7H         LINE#         128
  C:60D7H         LINE#         129
  C:60D7H         LINE#         130
  C:60DAH         LINE#         131
  C:60DBH         LINE#         132
  C:60DCH         LINE#         133
  C:60DDH         LINE#         134
  C:60DEH         LINE#         135
  C:60DFH         LINE#         136
  C:60E1H         LINE#         137
  C:60E3H         LINE#         139
  C:60E3H         LINE#         140
  C:60E5H         LINE#         141
  C:60E7H         LINE#         142
  C:60E7H         LINE#         143
  C:60E7H         LINE#         145
  C:60E7H         LINE#         146
  C:60E9H         LINE#         147
  C:60EBH         LINE#         148
  C:60EBH         LINE#         149
  C:60EBH         LINE#         151
  C:60EBH         LINE#         152
  C:60EDH         LINE#         153
  C:60EFH         LINE#         154
  C:60EFH         LINE#         155
  C:60EFH         LINE#         157
  C:60EFH         LINE#         158
BL51 BANKED LINKER/LOCATER V6.22                                                      02/06/2025  15:28:46  PAGE 74


  C:60F1H         LINE#         159
  C:60F3H         LINE#         160
  C:60F3H         LINE#         161
  C:6100H         LINE#         163
  C:6102H         LINE#         164
  -------         ENDPROC       _MCUFLASHWRSECTOR
  -------         PROC          _MCUFLASHWRITE
  X:02B9H         SYMBOL        McuFlashAddr
  X:02BBH         SYMBOL        XramAddr
  -------         DO            
  B:0029H.7       SYMBOL        Result
  -------         ENDDO         
  C:5EC5H         LINE#         177
  C:5ED3H         LINE#         178
  C:5ED3H         LINE#         179
  C:5ED5H         LINE#         181
  C:5ED8H         LINE#         182
  C:5EDAH         LINE#         183
  C:5EDDH         LINE#         185
  C:5EE6H         LINE#         186
  C:5EE9H         LINE#         187
  C:5EECH         LINE#         188
  C:5EECH         LINE#         189
  C:5EEFH         LINE#         190
  C:5EF3H         LINE#         191
  C:5EF3H         LINE#         192
  C:5EF6H         LINE#         193
  C:5EFEH         LINE#         194
  C:5EFEH         LINE#         195
  C:5F01H         LINE#         196
  C:5F0AH         LINE#         197
  C:5F0AH         LINE#         198
  C:5F0DH         LINE#         199
  C:5F0EH         LINE#         200
  C:5F0FH         LINE#         201
  C:5F10H         LINE#         202
  C:5F11H         LINE#         203
  C:5F12H         LINE#         205
  C:5F1FH         LINE#         206
  C:5F1FH         LINE#         207
  C:5F32H         LINE#         208
  C:5F32H         LINE#         209
  C:5F45H         LINE#         210
  C:5F45H         LINE#         211
  C:5F47H         LINE#         212
  C:5F47H         LINE#         213
  C:5F47H         LINE#         214
  C:5F47H         LINE#         215
  C:5F47H         LINE#         216
  C:5F47H         LINE#         217
  C:5F47H         LINE#         218
  C:5F47H         LINE#         220
  C:5F4AH         LINE#         221
  C:5F4CH         LINE#         222
  C:5F4EH         LINE#         223
  C:5F50H         LINE#         224
  C:5F52H         LINE#         226
BL51 BANKED LINKER/LOCATER V6.22                                                      02/06/2025  15:28:46  PAGE 75


  C:5F55H         LINE#         227
  C:5F57H         LINE#         228
  C:5F59H         LINE#         230
  C:5F5BH         LINE#         231
  -------         ENDPROC       _MCUFLASHWRITE
  -------         PROC          MCUFLASHPROCESS
  -------         DO            
  B:0029H.5       SYMBOL        McuFlashBk1WrFailFlg
  B:0029H.6       SYMBOL        McuFlashBk2WrFailFlg
  X:02B7H         SYMBOL        VoltageMin
  -------         ENDDO         
  C:526EH         LINE#         244
  C:526EH         LINE#         245
  C:526EH         LINE#         246
  C:5272H         LINE#         249
  C:5278H         LINE#         250
  C:5278H         LINE#         251
  C:527AH         LINE#         253
  C:5280H         LINE#         254
  C:5287H         LINE#         255
  C:5287H         LINE#         256
  C:5291H         LINE#         257
  C:5293H         LINE#         259
  C:5293H         LINE#         260
  C:529DH         LINE#         261
  C:529DH         LINE#         263
  C:52C0H         LINE#         264
  C:52C0H         LINE#         265
  C:52C9H         LINE#         266
  C:52C9H         LINE#         267
  C:52D3H         LINE#         268
  C:52D3H         LINE#         269
  C:52D5H         LINE#         270
  C:52DDH         LINE#         271
  C:52E5H         LINE#         272
  C:52ECH         LINE#         273
  C:52ECH         LINE#         274
  C:52ECH         LINE#         276
  C:52F7H         LINE#         277
  C:52F7H         LINE#         278
  C:5302H         LINE#         279
  C:5302H         LINE#         280
  C:5304H         LINE#         281
  C:530CH         LINE#         282
  C:5314H         LINE#         283
  C:531BH         LINE#         284
  C:531BH         LINE#         285
  C:531BH         LINE#         286
  C:531DH         LINE#         288
  C:531DH         LINE#         289
  C:531FH         LINE#         290
  C:5321H         LINE#         291
  C:5321H         LINE#         292
  C:5326H         LINE#         294
  C:532CH         LINE#         295
  C:532CH         LINE#         296
  C:532EH         LINE#         297
BL51 BANKED LINKER/LOCATER V6.22                                                      02/06/2025  15:28:46  PAGE 76


  C:532EH         LINE#         298
  C:532EH         LINE#         299
  -------         ENDPROC       MCUFLASHPROCESS
  -------         PROC          _MCUFLASHREAD
  X:02B7H         SYMBOL        SourceAddr
  D:0004H         SYMBOL        TargetAddr
  X:02B9H         SYMBOL        Length
  -------         DO            
  D:0006H         SYMBOL        i
  B:0029H.5       SYMBOL        Result
  D:0015H         SYMBOL        TargetAddr1
  -------         ENDDO         
  C:6A9FH         LINE#         308
  C:6AADH         LINE#         309
  C:6AADH         LINE#         311
  C:6AAFH         LINE#         312
  C:6AB7H         LINE#         314
  C:6AB9H         LINE#         315
  C:6ABCH         LINE#         316
  C:6ABFH         LINE#         317
  C:6ACFH         LINE#         318
  C:6ACFH         LINE#         319
  C:6AE7H         LINE#         320
  C:6AEFH         LINE#         321
  C:6AF6H         LINE#         322
  C:6AF9H         LINE#         323
  C:6AFBH         LINE#         325
  C:6AFDH         LINE#         326
  -------         ENDPROC       _MCUFLASHREAD
  -------         PROC          MCUFLASHWRWAITCHECK
  C:7DD7H         LINE#         335
  C:7DD7H         LINE#         336
  C:7DD7H         LINE#         337
  C:7DDAH         LINE#         338
  C:7DDAH         LINE#         339
  C:7DE5H         LINE#         340
  C:7DE5H         LINE#         341
  C:7DE7H         LINE#         342
  C:7DE9H         LINE#         343
  C:7DEBH         LINE#         344
  C:7DEBH         LINE#         345
  C:7DEBH         LINE#         346
  -------         ENDPROC       MCUFLASHWRWAITCHECK
  -------         PROC          _MCUFLASHCHECKFLG
  D:0006H         SYMBOL        McuFlashAddr
  -------         DO            
  B:0029H.5       SYMBOL        Result
  -------         ENDDO         
  C:7B6DH         LINE#         355
  C:7B6DH         LINE#         356
  C:7B6DH         LINE#         357
  C:7B6FH         LINE#         359
  C:7B72H         LINE#         360
  C:7B8CH         LINE#         361
  C:7B8CH         LINE#         362
  C:7B8EH         LINE#         363
  C:7B8EH         LINE#         364
BL51 BANKED LINKER/LOCATER V6.22                                                      02/06/2025  15:28:46  PAGE 77


  C:7B91H         LINE#         366
  C:7B93H         LINE#         367
  -------         ENDPROC       _MCUFLASHCHECKFLG
  -------         ENDMOD        MCUFLASH

  -------         MODULE        MCULIB
  C:0000H         SYMBOL        _ICE_DUMMY_
  D:0080H         PUBLIC        P0
  D:0090H         PUBLIC        P1
  D:00A0H         PUBLIC        P2
  D:00B0H         PUBLIC        P3
  D:00C0H         PUBLIC        P4
  C:73D1H         PUBLIC        _Delay1ms
  D:009DH         PUBLIC        SBRTH
  D:0080H         PUBLIC        P5
  B:00A8H.7       PUBLIC        EA
  D:00C7H         PUBLIC        PWM0CON
  D:00B6H         PUBLIC        PWM1CON
  D:00B7H         PUBLIC        PWM2CON
  D:009CH         PUBLIC        SBRTL
  C:7A8FH         PUBLIC        _McuTimer3Set
  D:00A8H         PUBLIC        IEN0
  D:00A9H         PUBLIC        IEN1
  D:00E8H         PUBLIC        EXF0
  D:008EH         PUBLIC        SUSLO
  C:7A2CH         PUBLIC        _MemoryCopy
  C:7B43H         PUBLIC        _MemorySet
  D:0087H         PUBLIC        PCON
  D:00CFH         PUBLIC        PWM0DH
  D:00A5H         PUBLIC        PWM1DH
  D:00BFH         PUBLIC        PWM2DH
  D:0098H         PUBLIC        SCON
  D:0088H         PUBLIC        TCON
  D:00CEH         PUBLIC        PWM0DL
  D:00A4H         PUBLIC        PWM1DL
  D:00BEH         PUBLIC        PWM2DL
  D:00B2H         PUBLIC        CLKCON
  D:00CDH         PUBLIC        PWM0PH
  D:00AFH         PUBLIC        PWM1PH
  D:00BDH         PUBLIC        PWM2PH
  D:00CCH         PUBLIC        PWM0PL
  D:00AEH         PUBLIC        PWM1PL
  C:7F5FH         PUBLIC        McuIntoIdle
  C:7C51H         PUBLIC        _McuClockSet
  D:00BCH         PUBLIC        PWM2PL
  D:0086H         PUBLIC        INSCON
  D:008DH         PUBLIC        TH3
  D:008CH         PUBLIC        TL3
  C:7F6BH         PUBLIC        McuIntoPD
  B:0088H.2       PUBLIC        TR3
  C:6856H         PUBLIC        RamCheckProcess
  D:0088H         PUBLIC        T3CON
  C:7AECH         PUBLIC        SystemResetProcess
  C:6210H         PUBLIC        _McuPWM0Set
  C:6291H         PUBLIC        _McuPWM1Set
  C:6312H         PUBLIC        _McuPWM2Set
  -------         PROC          _MCUTIMER3SET
BL51 BANKED LINKER/LOCATER V6.22                                                      02/06/2025  15:28:46  PAGE 78


  X:02B7H         SYMBOL        ClkSource
  D:0004H         SYMBOL        XmS
  -------         DO            
  D:0006H         SYMBOL        TempVal
  -------         ENDDO         
  C:7A8FH         LINE#         20
  C:7A94H         LINE#         21
  C:7A94H         LINE#         24
  C:7A97H         LINE#         67
  C:7A9AH         LINE#         68
  C:7AB5H         LINE#         70
  C:7AB7H         LINE#         71
  C:7AB9H         LINE#         72
  C:7ABBH         LINE#         74
  C:7ABEH         LINE#         75
  -------         ENDPROC       _MCUTIMER3SET
  -------         PROC          _MCUCLOCKSET
  X:02B7H         SYMBOL        SysClock
  -------         DO            
  D:0007H         SYMBOL        ea
  -------         ENDDO         
  C:7C51H         LINE#         84
  C:7C56H         LINE#         85
  C:7C56H         LINE#         88
  C:7C5BH         LINE#         89
  C:7C5DH         LINE#         91
  C:7C60H         LINE#         93
  C:7C61H         LINE#         94
  C:7C62H         LINE#         95
  C:7C63H         LINE#         96
  C:7C64H         LINE#         97
  C:7C65H         LINE#         98
  C:7C66H         LINE#         99
  C:7C67H         LINE#         100
  C:7C68H         LINE#         102
  C:7C6BH         LINE#         104
  C:7C6EH         LINE#         106
  C:7C72H         LINE#         107
  -------         ENDPROC       _MCUCLOCKSET
  -------         PROC          _MCUPWM0SET
  X:05E8H         SYMBOL        PwmFreq
  X:05EAH         SYMBOL        DutyRatio
  C:6210H         LINE#         116
  C:621BH         LINE#         117
  C:621BH         LINE#         118
  C:621EH         LINE#         119
  C:6238H         LINE#         120
  C:6257H         LINE#         121
  C:6275H         LINE#         122
  C:6290H         LINE#         123
  -------         ENDPROC       _MCUPWM0SET
  -------         PROC          _MCUPWM1SET
  X:05EBH         SYMBOL        PwmFreq
  X:05EDH         SYMBOL        DutyRatio
  C:6291H         LINE#         125
  C:629CH         LINE#         126
  C:629CH         LINE#         127
BL51 BANKED LINKER/LOCATER V6.22                                                      02/06/2025  15:28:46  PAGE 79


  C:629FH         LINE#         128
  C:62B9H         LINE#         129
  C:62D8H         LINE#         130
  C:62F6H         LINE#         131
  C:6311H         LINE#         132
  -------         ENDPROC       _MCUPWM1SET
  -------         PROC          _MCUPWM2SET
  X:02BCH         SYMBOL        PwmFreq
  X:02BEH         SYMBOL        DutyRatio
  C:6312H         LINE#         134
  C:631DH         LINE#         135
  C:631DH         LINE#         136
  C:6320H         LINE#         137
  C:633AH         LINE#         138
  C:6359H         LINE#         139
  C:6377H         LINE#         140
  C:6392H         LINE#         141
  -------         ENDPROC       _MCUPWM2SET
  -------         PROC          _DELAY1MS
  D:0007H         SYMBOL        Xms
  -------         DO            
  D:0006H         SYMBOL        i
  D:0002H         SYMBOL        j
  D:0004H         SYMBOL        Tcnt
  -------         ENDDO         
  C:73D1H         LINE#         154
  C:73D1H         LINE#         155
  C:73D1H         LINE#         159
  C:73D7H         LINE#         160
  C:73D7H         LINE#         161
  C:73DBH         LINE#         162
  C:73DDH         LINE#         163
  C:73E5H         LINE#         164
  C:73E5H         LINE#         165
  C:73E9H         LINE#         166
  C:73EBH         LINE#         167
  C:73F3H         LINE#         168
  C:73F3H         LINE#         169
  C:73F7H         LINE#         170
  C:73F9H         LINE#         172
  C:73F9H         LINE#         173
  C:73FDH         LINE#         174
  C:73FDH         LINE#         177
  C:7404H         LINE#         178
  C:7404H         LINE#         179
  C:740EH         LINE#         180
  C:740EH         LINE#         181
  C:7415H         LINE#         182
  C:7418H         LINE#         183
  -------         ENDPROC       _DELAY1MS
  -------         PROC          RAMCHECKPROCESS
  C:6856H         LINE#         220
  C:6856H         LINE#         221
  C:6856H         LINE#         222
  C:68B8H         LINE#         234
  C:68B8H         LINE#         235
  C:68BAH         LINE#         236
BL51 BANKED LINKER/LOCATER V6.22                                                      02/06/2025  15:28:46  PAGE 80


  C:68BAH         LINE#         238
  C:68BAH         LINE#         239
  C:68BBH         LINE#         240
  C:68BBH         LINE#         241
  -------         ENDPROC       RAMCHECKPROCESS
  -------         PROC          _MEMORYSET
  X:02C3H         SYMBOL        pt
  D:0005H         SYMBOL        setval
  D:0003H         SYMBOL        length
  -------         DO            
  D:0007H         SYMBOL        i
  -------         ENDDO         
  C:7B43H         LINE#         252
  C:7B4BH         LINE#         253
  C:7B4BH         LINE#         255
  C:7B52H         LINE#         256
  C:7B52H         LINE#         257
  C:7B5FH         LINE#         258
  C:7B69H         LINE#         259
  C:7B6CH         LINE#         260
  -------         ENDPROC       _MEMORYSET
  -------         PROC          _MEMORYCOPY
  X:02D9H         SYMBOL        source
  D:0004H         SYMBOL        target
  D:0003H         SYMBOL        length
  -------         DO            
  D:0007H         SYMBOL        i
  -------         ENDDO         
  C:7A2CH         LINE#         271
  C:7A34H         LINE#         272
  C:7A34H         LINE#         274
  C:7A3BH         LINE#         275
  C:7A3BH         LINE#         276
  C:7A4CH         LINE#         277
  C:7A51H         LINE#         278
  C:7A5BH         LINE#         279
  C:7A5EH         LINE#         280
  -------         ENDPROC       _MEMORYCOPY
  -------         PROC          MCUINTOIDLE
  C:7F5FH         LINE#         289
  C:7F5FH         LINE#         290
  C:7F5FH         LINE#         291
  C:7F62H         LINE#         292
  C:7F65H         LINE#         293
  C:7F66H         LINE#         294
  C:7F67H         LINE#         295
  C:7F68H         LINE#         296
  C:7F69H         LINE#         297
  C:7F6AH         LINE#         298
  -------         ENDPROC       MCUINTOIDLE
  -------         PROC          MCUINTOPD
  C:7F6BH         LINE#         300
  C:7F6BH         LINE#         301
  C:7F6BH         LINE#         302
  C:7F6EH         LINE#         303
  C:7F71H         LINE#         304
  C:7F72H         LINE#         305
BL51 BANKED LINKER/LOCATER V6.22                                                      02/06/2025  15:28:46  PAGE 81


  C:7F73H         LINE#         306
  C:7F74H         LINE#         307
  C:7F75H         LINE#         308
  C:7F76H         LINE#         309
  -------         ENDPROC       MCUINTOPD
  -------         PROC          SYSTEMRESETPROCESS
  C:7AECH         LINE#         318
  C:7AECH         LINE#         319
  C:7AECH         LINE#         320
  C:7B03H         LINE#         322
  C:7B03H         LINE#         323
  C:7B05H         LINE#         324
  C:7B08H         LINE#         325
  C:7B0AH         LINE#         326
  C:7B0CH         LINE#         327
  C:7B0EH         LINE#         329
  C:7B10H         LINE#         330
  C:7B12H         LINE#         331
  C:7B14H         LINE#         333
  C:7B17H         LINE#         334
  C:7B17H         LINE#         335
  -------         ENDPROC       SYSTEMRESETPROCESS
  -------         ENDMOD        MCULIB

  -------         MODULE        MOSCTRL
  C:0000H         SYMBOL        _ICE_DUMMY_
  D:0080H         PUBLIC        P0
  D:0090H         PUBLIC        P1
  D:00A0H         PUBLIC        P2
  D:00B0H         PUBLIC        P3
  D:00C0H         PUBLIC        P4
  D:0080H         PUBLIC        P5
  C:721CH         PUBLIC        MosStatusCheck
  C:7ABFH         PUBLIC        MosCtrl
  B:002EH.6       PUBLIC        bCHGMOSBk
  B:002EH.7       PUBLIC        bDSGMOSBk
  -------         PROC          MOSSTATUSCHECK
  C:721CH         LINE#         20
  C:721CH         LINE#         21
  C:721CH         LINE#         22
  C:721EH         LINE#         23
  C:7220H         LINE#         25
  C:7226H         LINE#         26
  C:7226H         LINE#         27
  C:7228H         LINE#         28
  C:7228H         LINE#         30
  C:723AH         LINE#         31
  C:723AH         LINE#         32
  C:723CH         LINE#         33
  C:723CH         LINE#         35
  C:723FH         LINE#         36
  C:723FH         LINE#         37
  C:724BH         LINE#         38
  C:724BH         LINE#         39
  C:724DH         LINE#         40
  C:724DH         LINE#         41
  C:724DH         LINE#         43
BL51 BANKED LINKER/LOCATER V6.22                                                      02/06/2025  15:28:46  PAGE 82


  C:7250H         LINE#         44
  C:7250H         LINE#         45
  C:7253H         LINE#         46
  C:7253H         LINE#         47
  C:7255H         LINE#         48
  C:7255H         LINE#         49
  C:7255H         LINE#         51
  C:725EH         LINE#         52
  C:725EH         LINE#         53
  C:7260H         LINE#         54
  C:7260H         LINE#         56
  C:7263H         LINE#         57
  C:7263H         LINE#         58
  C:7265H         LINE#         59
  C:7265H         LINE#         60
  -------         ENDPROC       MOSSTATUSCHECK
  -------         PROC          MOSCTRL
  C:7ABFH         LINE#         70
  C:7ABFH         LINE#         71
  C:7ABFH         LINE#         72
  C:7AC2H         LINE#         74
  C:7AD2H         LINE#         75
  C:7AD2H         LINE#         76
  C:7AD6H         LINE#         77
  C:7ADAH         LINE#         79
  C:7AEBH         LINE#         80
  C:7AEBH         LINE#         81
  -------         ENDPROC       MOSCTRL
  -------         ENDMOD        MOSCTRL

  -------         MODULE        PORSELFTEST
  C:0000H         SYMBOL        _ICE_DUMMY_
  D:0080H         PUBLIC        P0
  C:6F18H         PUBLIC        PorProtectOTC
  D:0090H         PUBLIC        P1
  C:6FB6H         PUBLIC        PorProtectOTD
  D:00A0H         PUBLIC        P2
  D:00B0H         PUBLIC        P3
  D:00C0H         PUBLIC        P4
  D:0080H         PUBLIC        P5
  C:6F67H         PUBLIC        PorProtectUTC
  C:7005H         PUBLIC        PorProtectUTD
  C:7419H         PUBLIC        PorProtectOV
  C:7461H         PUBLIC        PorProtectUV
  X:053FH         PUBLIC        ucPorSelfTestDelayCnt
  B:002FH.6       PUBLIC        bPorSelfTestFlg
  C:787BH         PUBLIC        PorSelfTest
  -------         PROC          PORPROTECTOV
  C:7419H         LINE#         20
  C:7419H         LINE#         21
  C:7419H         LINE#         22
  C:741CH         LINE#         23
  C:741CH         LINE#         24
  C:742BH         LINE#         25
  C:742BH         LINE#         26
  C:7440H         LINE#         27
  C:7440H         LINE#         28
BL51 BANKED LINKER/LOCATER V6.22                                                      02/06/2025  15:28:46  PAGE 83


  C:7442H         LINE#         29
  C:7449H         LINE#         30
  C:7449H         LINE#         31
  C:744AH         LINE#         32
  C:7459H         LINE#         33
  C:7459H         LINE#         34
  C:7460H         LINE#         35
  C:7460H         LINE#         36
  C:7460H         LINE#         37
  -------         ENDPROC       PORPROTECTOV
  -------         PROC          PORPROTECTUV
  C:7461H         LINE#         46
  C:7461H         LINE#         47
  C:7461H         LINE#         48
  C:7464H         LINE#         49
  C:7464H         LINE#         50
  C:7473H         LINE#         51
  C:7473H         LINE#         52
  C:7488H         LINE#         53
  C:7488H         LINE#         54
  C:748AH         LINE#         55
  C:7491H         LINE#         56
  C:7491H         LINE#         57
  C:7492H         LINE#         58
  C:74A1H         LINE#         59
  C:74A1H         LINE#         60
  C:74A8H         LINE#         61
  C:74A8H         LINE#         62
  C:74A8H         LINE#         63
  -------         ENDPROC       PORPROTECTUV
  -------         PROC          PORPROTECTOTC
  C:6F18H         LINE#         72
  C:6F18H         LINE#         73
  C:6F18H         LINE#         74
  C:6F1BH         LINE#         75
  C:6F1BH         LINE#         76
  C:6F31H         LINE#         77
  C:6F31H         LINE#         78
  C:6F46H         LINE#         79
  C:6F46H         LINE#         80
  C:6F48H         LINE#         81
  C:6F4FH         LINE#         82
  C:6F4FH         LINE#         83
  C:6F50H         LINE#         84
  C:6F5FH         LINE#         85
  C:6F5FH         LINE#         86
  C:6F66H         LINE#         87
  C:6F66H         LINE#         88
  C:6F66H         LINE#         89
  -------         ENDPROC       PORPROTECTOTC
  -------         PROC          PORPROTECTUTC
  C:6F67H         LINE#         98
  C:6F67H         LINE#         99
  C:6F67H         LINE#         100
  C:6F6AH         LINE#         101
  C:6F6AH         LINE#         102
  C:6F80H         LINE#         103
BL51 BANKED LINKER/LOCATER V6.22                                                      02/06/2025  15:28:46  PAGE 84


  C:6F80H         LINE#         104
  C:6F95H         LINE#         105
  C:6F95H         LINE#         106
  C:6F97H         LINE#         107
  C:6F9EH         LINE#         108
  C:6F9EH         LINE#         109
  C:6F9FH         LINE#         110
  C:6FAEH         LINE#         111
  C:6FAEH         LINE#         112
  C:6FB5H         LINE#         113
  C:6FB5H         LINE#         114
  C:6FB5H         LINE#         115
  -------         ENDPROC       PORPROTECTUTC
  -------         PROC          PORPROTECTOTD
  C:6FB6H         LINE#         124
  C:6FB6H         LINE#         125
  C:6FB6H         LINE#         126
  C:6FB9H         LINE#         127
  C:6FB9H         LINE#         128
  C:6FCFH         LINE#         129
  C:6FCFH         LINE#         130
  C:6FE4H         LINE#         131
  C:6FE4H         LINE#         132
  C:6FE6H         LINE#         133
  C:6FEDH         LINE#         134
  C:6FEDH         LINE#         135
  C:6FEEH         LINE#         136
  C:6FFDH         LINE#         137
  C:6FFDH         LINE#         138
  C:7004H         LINE#         139
  C:7004H         LINE#         140
  C:7004H         LINE#         141
  -------         ENDPROC       PORPROTECTOTD
  -------         PROC          PORPROTECTUTD
  C:7005H         LINE#         150
  C:7005H         LINE#         151
  C:7005H         LINE#         152
  C:7008H         LINE#         153
  C:7008H         LINE#         154
  C:701EH         LINE#         155
  C:701EH         LINE#         156
  C:7033H         LINE#         157
  C:7033H         LINE#         158
  C:7035H         LINE#         159
  C:703CH         LINE#         160
  C:703CH         LINE#         161
  C:703DH         LINE#         162
  C:704CH         LINE#         163
  C:704CH         LINE#         164
  C:7053H         LINE#         165
  C:7053H         LINE#         166
  C:7053H         LINE#         167
  -------         ENDPROC       PORPROTECTUTD
  -------         PROC          PORSELFTEST
  C:787BH         LINE#         176
  C:787BH         LINE#         177
  C:787BH         LINE#         178
BL51 BANKED LINKER/LOCATER V6.22                                                      02/06/2025  15:28:46  PAGE 85


  C:787EH         LINE#         179
  C:787EH         LINE#         180
  C:7881H         LINE#         181
  C:7884H         LINE#         182
  C:7887H         LINE#         183
  C:788AH         LINE#         185
  C:788DH         LINE#         186
  C:7890H         LINE#         187
  C:7893H         LINE#         188
  C:7896H         LINE#         190
  C:78A1H         LINE#         191
  C:78A1H         LINE#         192
  C:78A3H         LINE#         193
  C:78AFH         LINE#         194
  C:78AFH         LINE#         195
  C:78B1H         LINE#         196
  C:78B2H         LINE#         198
  C:78B2H         LINE#         199
  C:78B5H         LINE#         200
  C:78B5H         LINE#         201
  C:78B5H         LINE#         202
  C:78B5H         LINE#         203
  -------         ENDPROC       PORSELFTEST
  -------         ENDMOD        PORSELFTEST

  -------         MODULE        PROTECT
  C:0000H         SYMBOL        _ICE_DUMMY_
  D:0080H         PUBLIC        P0
  D:0090H         PUBLIC        P1
  X:03B8H         PUBLIC        uiOCD1DelayCnt
  D:00A0H         PUBLIC        P2
  X:03BAH         PUBLIC        uiOCD2DelayCnt
  D:00B0H         PUBLIC        P3
  D:00C0H         PUBLIC        P4
  D:0080H         PUBLIC        P5
  C:51AAH         PUBLIC        ProtectOV
  C:53ECH         PUBLIC        ProtectUV
  B:002FH.0       PUBLIC        bOVLock
  B:002FH.1       PUBLIC        bUVLock
  X:03BCH         PUBLIC        uiOVDelayCnt
  X:03BEH         PUBLIC        uiUVDelayCnt
  X:03C0H         PUBLIC        uiOTCRDelayCnt
  X:03C2H         PUBLIC        uiOTDRDelayCnt
  X:03C4H         PUBLIC        uiUTCRDelayCnt
  X:03C6H         PUBLIC        uiUTDRDelayCnt
  C:6CC7H         PUBLIC        ProtectOCC
  C:7C93H         PUBLIC        ProtectProcess
  C:54A8H         PUBLIC        ProtectOTC
  C:5620H         PUBLIC        ProtectOTD
  X:03C8H         PUBLIC        uiOCCRcnt
  X:03CAH         PUBLIC        uiOCCDelayCnt
  X:03CCH         PUBLIC        uiOCDRcnt
  C:5564H         PUBLIC        ProtectUTC
  C:56DCH         PUBLIC        ProtectUTD
  C:6410H         PUBLIC        ProtectOCRecover
  X:03CEH         PUBLIC        uiOTCDelayCnt
  X:03D0H         PUBLIC        uiOTDDelayCnt
BL51 BANKED LINKER/LOCATER V6.22                                                      02/06/2025  15:28:46  PAGE 86


  X:03D2H         PUBLIC        uiUTCDelayCnt
  X:03D4H         PUBLIC        uiUTDDelayCnt
  C:6D20H         PUBLIC        ProtectOCD1
  C:6D79H         PUBLIC        ProtectOCD2
  X:03D6H         PUBLIC        uiOVRDelayCnt
  X:03D8H         PUBLIC        uiUVRDelayCnt
  -------         PROC          PROTECTOV
  C:51AAH         LINE#         39
  C:51AAH         LINE#         40
  C:51AAH         LINE#         41
  C:51B0H         LINE#         42
  C:51B0H         LINE#         43
  C:51BFH         LINE#         44
  C:51BFH         LINE#         45
  C:51E0H         LINE#         46
  C:51E0H         LINE#         47
  C:51E2H         LINE#         48
  C:51E4H         LINE#         49
  C:51EBH         LINE#         50
  C:51F1H         LINE#         51
  C:51F1H         LINE#         52
  C:51F2H         LINE#         53
  C:5201H         LINE#         54
  C:5201H         LINE#         55
  C:5208H         LINE#         56
  C:5208H         LINE#         57
  C:5209H         LINE#         58
  C:520CH         LINE#         59
  C:520CH         LINE#         60
  C:521BH         LINE#         61
  C:521BH         LINE#         62
  C:5239H         LINE#         63
  C:5239H         LINE#         64
  C:523CH         LINE#         65
  C:523CH         LINE#         66
  C:523EH         LINE#         67
  C:5240H         LINE#         68
  C:5242H         LINE#         70
  C:5242H         LINE#         71
  C:5244H         LINE#         72
  C:5246H         LINE#         73
  C:5249H         LINE#         74
  C:5249H         LINE#         75
  C:5250H         LINE#         76
  C:5256H         LINE#         77
  C:5256H         LINE#         78
  C:5257H         LINE#         79
  C:5266H         LINE#         80
  C:5266H         LINE#         81
  C:526DH         LINE#         82
  C:526DH         LINE#         83
  C:526DH         LINE#         84
  -------         ENDPROC       PROTECTOV
  -------         PROC          PROTECTUV
  C:53ECH         LINE#         92
  C:53ECH         LINE#         93
  C:53ECH         LINE#         94
BL51 BANKED LINKER/LOCATER V6.22                                                      02/06/2025  15:28:46  PAGE 87


  C:53EFH         LINE#         95
  C:53EFH         LINE#         96
  C:53FEH         LINE#         97
  C:53FEH         LINE#         98
  C:541FH         LINE#         99
  C:541FH         LINE#         100
  C:5421H         LINE#         101
  C:5423H         LINE#         102
  C:542AH         LINE#         103
  C:5430H         LINE#         104
  C:5430H         LINE#         105
  C:5431H         LINE#         106
  C:5440H         LINE#         107
  C:5440H         LINE#         108
  C:5447H         LINE#         109
  C:5447H         LINE#         110
  C:5448H         LINE#         111
  C:544BH         LINE#         112
  C:544BH         LINE#         113
  C:545AH         LINE#         114
  C:545AH         LINE#         115
  C:5478H         LINE#         116
  C:5478H         LINE#         117
  C:547BH         LINE#         118
  C:547BH         LINE#         119
  C:547DH         LINE#         120
  C:547FH         LINE#         121
  C:5481H         LINE#         123
  C:5481H         LINE#         124
  C:5483H         LINE#         125
  C:5483H         LINE#         126
  C:548AH         LINE#         127
  C:5490H         LINE#         128
  C:5490H         LINE#         129
  C:5491H         LINE#         130
  C:54A0H         LINE#         131
  C:54A0H         LINE#         132
  C:54A7H         LINE#         133
  C:54A7H         LINE#         134
  C:54A7H         LINE#         135
  -------         ENDPROC       PROTECTUV
  -------         PROC          PROTECTOTC
  C:54A8H         LINE#         143
  C:54A8H         LINE#         144
  C:54A8H         LINE#         145
  C:54ABH         LINE#         146
  C:54ABH         LINE#         147
  C:54C1H         LINE#         148
  C:54C1H         LINE#         149
  C:54E2H         LINE#         150
  C:54E2H         LINE#         151
  C:54E4H         LINE#         152
  C:54EBH         LINE#         153
  C:54F1H         LINE#         154
  C:54F1H         LINE#         155
  C:54F2H         LINE#         156
  C:5501H         LINE#         157
BL51 BANKED LINKER/LOCATER V6.22                                                      02/06/2025  15:28:46  PAGE 88


  C:5501H         LINE#         158
  C:5508H         LINE#         159
  C:5508H         LINE#         160
  C:5509H         LINE#         162
  C:5509H         LINE#         163
  C:551FH         LINE#         164
  C:551FH         LINE#         165
  C:553DH         LINE#         166
  C:553DH         LINE#         167
  C:553FH         LINE#         168
  C:5546H         LINE#         169
  C:554CH         LINE#         170
  C:554CH         LINE#         171
  C:554DH         LINE#         172
  C:555CH         LINE#         173
  C:555CH         LINE#         174
  C:5563H         LINE#         175
  C:5563H         LINE#         176
  C:5563H         LINE#         177
  -------         ENDPROC       PROTECTOTC
  -------         PROC          PROTECTUTC
  C:5564H         LINE#         186
  C:5564H         LINE#         187
  C:5564H         LINE#         188
  C:5567H         LINE#         189
  C:5567H         LINE#         190
  C:557DH         LINE#         191
  C:557DH         LINE#         192
  C:559EH         LINE#         193
  C:559EH         LINE#         194
  C:55A0H         LINE#         195
  C:55A7H         LINE#         196
  C:55ADH         LINE#         197
  C:55ADH         LINE#         198
  C:55AEH         LINE#         199
  C:55BDH         LINE#         200
  C:55BDH         LINE#         201
  C:55C4H         LINE#         202
  C:55C4H         LINE#         203
  C:55C5H         LINE#         205
  C:55C5H         LINE#         206
  C:55DBH         LINE#         207
  C:55DBH         LINE#         208
  C:55F9H         LINE#         209
  C:55F9H         LINE#         210
  C:55FBH         LINE#         211
  C:5602H         LINE#         212
  C:5608H         LINE#         213
  C:5608H         LINE#         214
  C:5609H         LINE#         215
  C:5618H         LINE#         216
  C:5618H         LINE#         217
  C:561FH         LINE#         218
  C:561FH         LINE#         219
  C:561FH         LINE#         220
  -------         ENDPROC       PROTECTUTC
  -------         PROC          PROTECTOTD
BL51 BANKED LINKER/LOCATER V6.22                                                      02/06/2025  15:28:46  PAGE 89


  C:5620H         LINE#         229
  C:5620H         LINE#         230
  C:5620H         LINE#         231
  C:5623H         LINE#         232
  C:5623H         LINE#         233
  C:5639H         LINE#         234
  C:5639H         LINE#         235
  C:565AH         LINE#         236
  C:565AH         LINE#         237
  C:565CH         LINE#         238
  C:5663H         LINE#         239
  C:5669H         LINE#         240
  C:5669H         LINE#         241
  C:566AH         LINE#         242
  C:5679H         LINE#         243
  C:5679H         LINE#         244
  C:5680H         LINE#         245
  C:5680H         LINE#         246
  C:5681H         LINE#         248
  C:5681H         LINE#         249
  C:5697H         LINE#         250
  C:5697H         LINE#         251
  C:56B5H         LINE#         252
  C:56B5H         LINE#         253
  C:56B7H         LINE#         254
  C:56BEH         LINE#         255
  C:56C4H         LINE#         256
  C:56C4H         LINE#         257
  C:56C5H         LINE#         258
  C:56D4H         LINE#         259
  C:56D4H         LINE#         260
  C:56DBH         LINE#         261
  C:56DBH         LINE#         262
  C:56DBH         LINE#         263
  -------         ENDPROC       PROTECTOTD
  -------         PROC          PROTECTUTD
  C:56DCH         LINE#         272
  C:56DCH         LINE#         273
  C:56DCH         LINE#         274
  C:56DFH         LINE#         275
  C:56DFH         LINE#         276
  C:56F5H         LINE#         277
  C:56F5H         LINE#         278
  C:5716H         LINE#         279
  C:5716H         LINE#         280
  C:5718H         LINE#         281
  C:571FH         LINE#         282
  C:5725H         LINE#         283
  C:5725H         LINE#         284
  C:5726H         LINE#         285
  C:5735H         LINE#         286
  C:5735H         LINE#         287
  C:573CH         LINE#         288
  C:573CH         LINE#         289
  C:573DH         LINE#         291
  C:573DH         LINE#         292
  C:5753H         LINE#         293
BL51 BANKED LINKER/LOCATER V6.22                                                      02/06/2025  15:28:46  PAGE 90


  C:5753H         LINE#         294
  C:5771H         LINE#         295
  C:5771H         LINE#         296
  C:5773H         LINE#         297
  C:577AH         LINE#         298
  C:5780H         LINE#         299
  C:5780H         LINE#         300
  C:5781H         LINE#         301
  C:5790H         LINE#         302
  C:5790H         LINE#         303
  C:5797H         LINE#         304
  C:5797H         LINE#         305
  C:5797H         LINE#         306
  -------         ENDPROC       PROTECTUTD
  -------         PROC          PROTECTOCC
  C:6CC7H         LINE#         316
  C:6CC7H         LINE#         317
  C:6CC7H         LINE#         318
  C:6CCAH         LINE#         319
  C:6CCAH         LINE#         320
  C:6CDCH         LINE#         321
  C:6CDCH         LINE#         322
  C:6CFAH         LINE#         323
  C:6CFAH         LINE#         324
  C:6CFCH         LINE#         325
  C:6CFEH         LINE#         326
  C:6D05H         LINE#         327
  C:6D05H         LINE#         328
  C:6D06H         LINE#         329
  C:6D09H         LINE#         330
  C:6D09H         LINE#         331
  C:6D18H         LINE#         332
  C:6D18H         LINE#         333
  C:6D1FH         LINE#         334
  C:6D1FH         LINE#         335
  C:6D1FH         LINE#         336
  C:6D1FH         LINE#         337
  -------         ENDPROC       PROTECTOCC
  -------         PROC          PROTECTOCD1
  C:6D20H         LINE#         346
  C:6D20H         LINE#         347
  C:6D20H         LINE#         348
  C:6D23H         LINE#         349
  C:6D23H         LINE#         350
  C:6D35H         LINE#         351
  C:6D35H         LINE#         352
  C:6D53H         LINE#         353
  C:6D53H         LINE#         354
  C:6D5AH         LINE#         355
  C:6D5CH         LINE#         356
  C:6D5EH         LINE#         357
  C:6D5EH         LINE#         358
  C:6D5FH         LINE#         359
  C:6D62H         LINE#         360
  C:6D62H         LINE#         361
  C:6D71H         LINE#         362
  C:6D71H         LINE#         363
BL51 BANKED LINKER/LOCATER V6.22                                                      02/06/2025  15:28:46  PAGE 91


  C:6D78H         LINE#         364
  C:6D78H         LINE#         365
  C:6D78H         LINE#         366
  C:6D78H         LINE#         367
  -------         ENDPROC       PROTECTOCD1
  -------         PROC          PROTECTOCD2
  C:6D79H         LINE#         376
  C:6D79H         LINE#         377
  C:6D79H         LINE#         378
  C:6D7CH         LINE#         379
  C:6D7CH         LINE#         380
  C:6D8EH         LINE#         381
  C:6D8EH         LINE#         382
  C:6DACH         LINE#         383
  C:6DACH         LINE#         384
  C:6DB3H         LINE#         385
  C:6DB5H         LINE#         386
  C:6DB7H         LINE#         387
  C:6DB7H         LINE#         388
  C:6DB8H         LINE#         389
  C:6DBBH         LINE#         390
  C:6DBBH         LINE#         391
  C:6DCAH         LINE#         392
  C:6DCAH         LINE#         393
  C:6DD1H         LINE#         394
  C:6DD1H         LINE#         395
  C:6DD1H         LINE#         396
  C:6DD1H         LINE#         397
  -------         ENDPROC       PROTECTOCD2
  -------         PROC          PROTECTPROCESS
  C:7C93H         LINE#         406
  C:7C93H         LINE#         407
  C:7C93H         LINE#         408
  C:7C96H         LINE#         409
  C:7C96H         LINE#         410
  C:7C99H         LINE#         411
  C:7C9CH         LINE#         413
  C:7C9FH         LINE#         414
  C:7CA2H         LINE#         415
  C:7CA5H         LINE#         416
  C:7CA8H         LINE#         418
  C:7CABH         LINE#         419
  C:7CAEH         LINE#         420
  C:7CB1H         LINE#         421
  C:7CB1H         LINE#         422
  -------         ENDPROC       PROTECTPROCESS
  -------         PROC          PROTECTOCRECOVER
  C:6410H         LINE#         431
  C:6410H         LINE#         432
  C:6410H         LINE#         433
  C:6413H         LINE#         434
  C:6413H         LINE#         435
  C:641CH         LINE#         436
  C:641CH         LINE#         437
  C:643AH         LINE#         438
  C:643AH         LINE#         439
  C:643FH         LINE#         440
BL51 BANKED LINKER/LOCATER V6.22                                                      02/06/2025  15:28:46  PAGE 92


  C:6445H         LINE#         441
  C:6447H         LINE#         442
  C:6449H         LINE#         443
  C:644BH         LINE#         444
  C:644DH         LINE#         445
  C:6450H         LINE#         446
  C:6450H         LINE#         447
  C:6452H         LINE#         448
  C:6455H         LINE#         449
  C:6455H         LINE#         450
  C:6455H         LINE#         451
  C:6455H         LINE#         453
  C:6458H         LINE#         454
  C:6458H         LINE#         455
  C:6476H         LINE#         456
  C:6476H         LINE#         457
  C:647DH         LINE#         458
  C:647FH         LINE#         459
  C:6483H         LINE#         460
  C:6485H         LINE#         461
  C:6485H         LINE#         462
  C:6485H         LINE#         463
  C:6485H         LINE#         464
  -------         ENDPROC       PROTECTOCRECOVER
  -------         ENDMOD        PROTECT

  -------         MODULE        RTC
  C:0000H         SYMBOL        _ICE_DUMMY_
  D:0080H         PUBLIC        P0
  D:0090H         PUBLIC        P1
  C:7D0CH         PUBLIC        RTCTwiCheck
  D:00A0H         PUBLIC        P2
  D:00B0H         PUBLIC        P3
  D:00C0H         PUBLIC        P4
  D:0080H         PUBLIC        P5
  C:5FEAH         PUBLIC        _RTCInitTime
  B:002FH.2       PUBLIC        bRTCTwiRWErr
  C:6C12H         PUBLIC        _RTCRead
  C:5D92H         PUBLIC        _RTCModifyTime
  X:0496H         PUBLIC        ucRTCTwiRWErrDelayCnt
  X:0497H         PUBLIC        RTC
  B:002FH.3       PUBLIC        bRTCErr
  C:6BB7H         PUBLIC        _RTCWrite
  C:3BC1H         PUBLIC        _RTCReadTime
  -------         PROC          RTCTWICHECK
  C:7D0CH         LINE#         23
  C:7D0CH         LINE#         24
  C:7D0CH         LINE#         25
  C:7D0FH         LINE#         26
  C:7D0FH         LINE#         27
  C:7D12H         LINE#         28
  C:7D12H         LINE#         29
  C:7D1DH         LINE#         30
  C:7D1DH         LINE#         31
  C:7D1FH         LINE#         32
  C:7D22H         LINE#         33
  C:7D22H         LINE#         34
BL51 BANKED LINKER/LOCATER V6.22                                                      02/06/2025  15:28:46  PAGE 93


  C:7D23H         LINE#         36
  C:7D23H         LINE#         37
  C:7D28H         LINE#         38
  C:7D28H         LINE#         39
  C:7D28H         LINE#         40
  -------         ENDPROC       RTCTWICHECK
  -------         PROC          _RTCWRITE
  X:02EEH         SYMBOL        WrAddr
  X:02EFH         SYMBOL        Length
  X:02F0H         SYMBOL        WrBuf
  -------         DO            
  B:002AH.0       SYMBOL        Result
  X:02F2H         SYMBOL        i
  -------         ENDDO         
  C:6BB7H         LINE#         49
  C:6BC5H         LINE#         50
  C:6BC5H         LINE#         51
  C:6BC7H         LINE#         54
  C:6BCAH         LINE#         55
  C:6BCAH         LINE#         56
  C:6BCDH         LINE#         57
  C:6BCDH         LINE#         59
  C:6BF5H         LINE#         60
  C:6BF5H         LINE#         61
  C:6BF7H         LINE#         62
  C:6BF9H         LINE#         63
  C:6BF9H         LINE#         71
  C:6BFEH         LINE#         72
  C:6C0AH         LINE#         73
  C:6C0AH         LINE#         74
  C:6C0FH         LINE#         76
  C:6C11H         LINE#         77
  -------         ENDPROC       _RTCWRITE
  -------         PROC          _RTCREAD
  X:02E4H         SYMBOL        RdAddr
  X:02E5H         SYMBOL        Length
  X:02E6H         SYMBOL        RdBuf
  -------         DO            
  B:0029H.7       SYMBOL        Result
  X:02E8H         SYMBOL        i
  -------         ENDDO         
  C:6C12H         LINE#         86
  C:6C20H         LINE#         87
  C:6C20H         LINE#         88
  C:6C22H         LINE#         91
  C:6C25H         LINE#         92
  C:6C25H         LINE#         93
  C:6C28H         LINE#         94
  C:6C28H         LINE#         96
  C:6C50H         LINE#         97
  C:6C50H         LINE#         98
  C:6C52H         LINE#         99
  C:6C54H         LINE#         100
  C:6C54H         LINE#         108
  C:6C59H         LINE#         109
  C:6C65H         LINE#         110
  C:6C65H         LINE#         111
BL51 BANKED LINKER/LOCATER V6.22                                                      02/06/2025  15:28:46  PAGE 94


  C:6C6AH         LINE#         113
  C:6C6CH         LINE#         114
  -------         ENDPROC       _RTCREAD
  -------         PROC          _RTCREADTIME
  X:02D9H         SYMBOL        RtcRdVal
  -------         DO            
  X:02DBH         SYMBOL        rtcbuf
  B:0029H.6       SYMBOL        Result
  -------         ENDDO         
  C:3BC1H         LINE#         122
  C:3BC9H         LINE#         123
  C:3BC9H         LINE#         125
  C:3BCBH         LINE#         127
  C:3BDBH         LINE#         128
  C:3BDBH         LINE#         129
  C:3BE5H         LINE#         130
  C:3BE5H         LINE#         131
  C:3C92H         LINE#         139
  C:3C92H         LINE#         140
  C:3CA3H         LINE#         141
  C:3CADH         LINE#         142
  C:3CBEH         LINE#         143
  C:3CCAH         LINE#         144
  C:3CDDH         LINE#         145
  C:3CEBH         LINE#         146
  C:3CFEH         LINE#         148
  C:3D07H         LINE#         149
  C:3D09H         LINE#         151
  C:3D09H         LINE#         152
  C:3D1CH         LINE#         153
  C:3D26H         LINE#         154
  C:3D33H         LINE#         155
  C:3D3FH         LINE#         156
  C:3D4FH         LINE#         157
  C:3D5FH         LINE#         158
  C:3D6FH         LINE#         160
  C:3D71H         LINE#         161
  C:3D71H         LINE#         162
  C:3D73H         LINE#         164
  C:3D73H         LINE#         165
  C:3D80H         LINE#         166
  C:3D80H         LINE#         167
  C:3D80H         LINE#         169
  C:3D82H         LINE#         170
  -------         ENDPROC       _RTCREADTIME
  -------         PROC          _RTCMODIFYTIME
  X:02E4H         SYMBOL        RtcMdyVal
  -------         DO            
  B:0029H.7       SYMBOL        Result
  X:02E6H         SYMBOL        rtcdata
  X:02E7H         SYMBOL        rtctemp
  -------         ENDDO         
  C:5D92H         LINE#         179
  C:5D9AH         LINE#         180
  C:5D9AH         LINE#         181
  C:5D9CH         LINE#         185
  C:5DA0H         LINE#         186
BL51 BANKED LINKER/LOCATER V6.22                                                      02/06/2025  15:28:46  PAGE 95


  C:5DADH         LINE#         188
  C:5DBEH         LINE#         189
  C:5DC8H         LINE#         190
  C:5DDDH         LINE#         191
  C:5DE9H         LINE#         192
  C:5DFDH         LINE#         193
  C:5E0BH         LINE#         194
  C:5E1EH         LINE#         196
  C:5E2BH         LINE#         198
  C:5E2DH         LINE#         199
  -------         ENDPROC       _RTCMODIFYTIME
  -------         PROC          _RTCINITTIME
  X:02B7H         SYMBOL        RtcInitVal
  -------         DO            
  B:0029H.5       SYMBOL        Result
  X:02B9H         SYMBOL        rtcbuf
  D:0007H         SYMBOL        i
  X:02C2H         SYMBOL        checksum
  -------         ENDDO         
  C:5FEAH         LINE#         208
  C:5FF2H         LINE#         209
  C:5FF2H         LINE#         210
  C:5FF4H         LINE#         213
  C:5FF9H         LINE#         215
  C:6003H         LINE#         217
  C:6010H         LINE#         218
  C:6012H         LINE#         219
  C:6012H         LINE#         220
  C:6024H         LINE#         221
  C:6029H         LINE#         223
  C:603BH         LINE#         224
  C:603BH         LINE#         225
  C:6040H         LINE#         226
  C:6042H         LINE#         227
  C:6046H         LINE#         228
  C:604AH         LINE#         229
  C:604EH         LINE#         230
  C:6052H         LINE#         231
  C:6056H         LINE#         232
  C:6056H         LINE#         234
  C:6067H         LINE#         235
  C:6074H         LINE#         237
  C:6076H         LINE#         238
  -------         ENDPROC       _RTCINITTIME
  -------         ENDMOD        RTC

  -------         MODULE        TWI
  C:0000H         SYMBOL        _ICE_DUMMY_
  D:0080H         PUBLIC        P0
  D:0090H         PUBLIC        P1
  D:00A0H         PUBLIC        P2
  D:00B0H         PUBLIC        P3
  D:00C0H         PUBLIC        P4
  D:0080H         PUBLIC        P5
  D:008AH         PUBLIC        TWIBR
  D:00C6H         PUBLIC        TWICR
  D:0089H         PUBLIC        TWTFREE
BL51 BANKED LINKER/LOCATER V6.22                                                      02/06/2025  15:28:46  PAGE 96


  C:3D83H         PUBLIC        _TwiRead
  D:00B1H         PUBLIC        RSTSTAT
  C:7D46H         PUBLIC        _CRC8cal
  D:00E6H         PUBLIC        TWITOUT
  C:47FEH         PUBLIC        _TwiWrite
  C:7DABH         PUBLIC        TwiInit
  D:008DH         PUBLIC        TWIDAT
  D:00C8H         PUBLIC        TWICON
  D:00D1H         PUBLIC        TWISTA
  C:7B94H         PUBLIC        _TWICheckStatus
  C:4E22H         PUBLIC        CRC8Table
  -------         PROC          _CRC8CAL
  D:0001H         SYMBOL        p
  D:0005H         SYMBOL        counter
  -------         DO            
  D:0007H         SYMBOL        crc8
  -------         ENDDO         
  C:7D46H         LINE#         38
  C:7D46H         LINE#         39
  C:7D46H         LINE#         40
  C:7D48H         LINE#         42
  C:7D4EH         LINE#         43
  C:7D4EH         LINE#         44
  C:7D57H         LINE#         45
  C:7D5EH         LINE#         46
  C:7D61H         LINE#         47
  C:7D61H         LINE#         48
  -------         ENDPROC       _CRC8CAL
  -------         PROC          _TWICHECKSTATUS
  D:0007H         SYMBOL        Status
  -------         DO            
  B:002AH.2       SYMBOL        Result
  D:0004H         SYMBOL        timeoutcount
  -------         ENDDO         
  C:7B94H         LINE#         59
  C:7B94H         LINE#         60
  C:7B94H         LINE#         61
  C:7B96H         LINE#         62
  C:7B9AH         LINE#         64
  C:7B9FH         LINE#         65
  C:7B9FH         LINE#         66
  C:7BA2H         LINE#         67
  C:7BA6H         LINE#         68
  C:7BA6H         LINE#         69
  C:7BABH         LINE#         70
  C:7BADH         LINE#         72
  C:7BADH         LINE#         73
  C:7BADH         LINE#         74
  C:7BADH         LINE#         75
  C:7BAFH         LINE#         76
  C:7BB6H         LINE#         77
  C:7BB6H         LINE#         78
  C:7BB8H         LINE#         79
  C:7BB8H         LINE#         81
  C:7BBAH         LINE#         82
  -------         ENDPROC       _TWICHECKSTATUS
  -------         PROC          _TWIWRITE
BL51 BANKED LINKER/LOCATER V6.22                                                      02/06/2025  15:28:46  PAGE 97


  X:02F3H         SYMBOL        SlaveID
  X:02F4H         SYMBOL        WrAddr
  X:02F6H         SYMBOL        AddrType
  X:02F7H         SYMBOL        Length
  X:02F8H         SYMBOL        CrcFlg
  X:02F9H         SYMBOL        WrBuf
  -------         DO            
  D:0006H         SYMBOL        i
  X:02FBH         SYMBOL        TempBuf
  B:002AH.1       SYMBOL        Result
  X:02FFH         SYMBOL        timeoutcount
  C:491FH         SYMBOL        WrErr
  -------         ENDDO         
  C:47FEH         LINE#         98
  C:480EH         LINE#         99
  C:480EH         LINE#         102
  C:4810H         LINE#         103
  C:481AH         LINE#         105
  C:481FH         LINE#         106
  C:4822H         LINE#         107
  C:4832H         LINE#         108
  C:4842H         LINE#         110
  C:484EH         LINE#         111
  C:484EH         LINE#         112
  C:4857H         LINE#         113
  C:485AH         LINE#         114
  C:4868H         LINE#         115
  C:4868H         LINE#         116
  C:486AH         LINE#         117
  C:486DH         LINE#         118
  C:486DH         LINE#         120
  C:4873H         LINE#         121
  C:4876H         LINE#         122
  C:487DH         LINE#         123
  C:487DH         LINE#         124
  C:487FH         LINE#         125
  C:4882H         LINE#         126
  C:4882H         LINE#         128
  C:4889H         LINE#         129
  C:4889H         LINE#         130
  C:488FH         LINE#         131
  C:4892H         LINE#         132
  C:4899H         LINE#         133
  C:4899H         LINE#         134
  C:489BH         LINE#         135
  C:489EH         LINE#         136
  C:489EH         LINE#         137
  C:489EH         LINE#         139
  C:48A6H         LINE#         140
  C:48A9H         LINE#         141
  C:48B0H         LINE#         142
  C:48B0H         LINE#         143
  C:48B2H         LINE#         144
  C:48B4H         LINE#         145
  C:48B4H         LINE#         147
  C:48BCH         LINE#         148
  C:48BCH         LINE#         149
BL51 BANKED LINKER/LOCATER V6.22                                                      02/06/2025  15:28:46  PAGE 98


  C:48C8H         LINE#         150
  C:48CBH         LINE#         151
  C:48D2H         LINE#         152
  C:48D2H         LINE#         153
  C:48D4H         LINE#         154
  C:48D6H         LINE#         155
  C:48D6H         LINE#         157
  C:48DCH         LINE#         158
  C:48DFH         LINE#         159
  C:48E6H         LINE#         160
  C:48E6H         LINE#         161
  C:48E8H         LINE#         162
  C:48EAH         LINE#         163
  C:48EAH         LINE#         164
  C:48EAH         LINE#         166
  C:48EAH         LINE#         167
  C:48F6H         LINE#         168
  C:48F6H         LINE#         169
  C:4904H         LINE#         170
  C:4907H         LINE#         171
  C:490EH         LINE#         172
  C:490EH         LINE#         173
  C:4910H         LINE#         174
  C:4912H         LINE#         175
  C:4912H         LINE#         176
  C:491CH         LINE#         177
  C:491FH         LINE#         178
  C:491FH         LINE#         179
  C:491FH         LINE#         180
  C:4922H         LINE#         181
  C:4927H         LINE#         182
  C:4927H         LINE#         183
  C:492AH         LINE#         184
  C:4934H         LINE#         185
  C:4934H         LINE#         186
  C:493EH         LINE#         187
  C:4940H         LINE#         189
  C:4940H         LINE#         190
  C:4940H         LINE#         191
  C:4940H         LINE#         192
  C:4942H         LINE#         193
  C:4942H         LINE#         195
  C:4944H         LINE#         196
  -------         ENDPROC       _TWIWRITE
  -------         PROC          _TWIREAD
  D:0002H         SYMBOL        SlaveID
  X:02EAH         SYMBOL        RdAddr
  D:0003H         SYMBOL        AddrType
  X:02EDH         SYMBOL        Length
  X:02EEH         SYMBOL        CrcFlg
  X:02EFH         SYMBOL        RdBuf
  -------         DO            
  B:002AH.0       SYMBOL        Result
  X:02F1H         SYMBOL        i
  X:02F2H         SYMBOL        TempBuf
  X:0320H         SYMBOL        RdCrc
  X:0321H         SYMBOL        timeoutcount
BL51 BANKED LINKER/LOCATER V6.22                                                      02/06/2025  15:28:46  PAGE 99


  C:3F16H         SYMBOL        RdErr
  -------         ENDDO         
  C:3D83H         LINE#         210
  C:3D8DH         LINE#         211
  C:3D8DH         LINE#         212
  C:3D8FH         LINE#         215
  C:3D94H         LINE#         216
  C:3D9CH         LINE#         218
  C:3DA1H         LINE#         219
  C:3DA4H         LINE#         221
  C:3DA9H         LINE#         223
  C:3DB5H         LINE#         224
  C:3DB5H         LINE#         225
  C:3DBEH         LINE#         226
  C:3DC1H         LINE#         227
  C:3DCFH         LINE#         228
  C:3DCFH         LINE#         229
  C:3DD1H         LINE#         230
  C:3DD4H         LINE#         231
  C:3DD4H         LINE#         233
  C:3DD6H         LINE#         234
  C:3DD9H         LINE#         235
  C:3DE0H         LINE#         236
  C:3DE0H         LINE#         237
  C:3DE2H         LINE#         238
  C:3DE5H         LINE#         239
  C:3DE5H         LINE#         241
  C:3DE9H         LINE#         242
  C:3DE9H         LINE#         243
  C:3DEFH         LINE#         244
  C:3DF2H         LINE#         245
  C:3DF9H         LINE#         246
  C:3DF9H         LINE#         247
  C:3DFBH         LINE#         248
  C:3DFEH         LINE#         249
  C:3DFEH         LINE#         250
  C:3DFEH         LINE#         252
  C:3E06H         LINE#         253
  C:3E09H         LINE#         254
  C:3E10H         LINE#         255
  C:3E10H         LINE#         256
  C:3E12H         LINE#         257
  C:3E15H         LINE#         258
  C:3E15H         LINE#         271
  C:3E18H         LINE#         272
  C:3E26H         LINE#         273
  C:3E26H         LINE#         274
  C:3E28H         LINE#         275
  C:3E2BH         LINE#         276
  C:3E2BH         LINE#         278
  C:3E30H         LINE#         279
  C:3E33H         LINE#         280
  C:3E3AH         LINE#         281
  C:3E3AH         LINE#         282
  C:3E3CH         LINE#         283
  C:3E3FH         LINE#         284
  C:3E3FH         LINE#         286
BL51 BANKED LINKER/LOCATER V6.22                                                      02/06/2025  15:28:46  PAGE 100


  C:3E52H         LINE#         287
  C:3E52H         LINE#         288
  C:3E58H         LINE#         289
  C:3E58H         LINE#         290
  C:3E5DH         LINE#         291
  C:3E5DH         LINE#         292
  C:3E60H         LINE#         293
  C:3E65H         LINE#         294
  C:3E67H         LINE#         296
  C:3E67H         LINE#         297
  C:3E6AH         LINE#         298
  C:3E6FH         LINE#         299
  C:3E6FH         LINE#         300
  C:3E7DH         LINE#         301
  C:3E87H         LINE#         302
  C:3E89H         LINE#         304
  C:3E89H         LINE#         305
  C:3E8CH         LINE#         306
  C:3E91H         LINE#         307
  C:3EA1H         LINE#         308
  C:3EA1H         LINE#         309
  C:3EA9H         LINE#         311
  C:3EB1H         LINE#         312
  C:3EB1H         LINE#         313
  C:3EB4H         LINE#         314
  C:3EB9H         LINE#         315
  C:3EBFH         LINE#         316
  C:3ED6H         LINE#         317
  C:3ED6H         LINE#         318
  C:3EE9H         LINE#         319
  C:3EE9H         LINE#         320
  C:3F02H         LINE#         321
  C:3F0CH         LINE#         322
  C:3F14H         LINE#         323
  C:3F14H         LINE#         325
  C:3F14H         LINE#         326
  C:3F16H         LINE#         327
  C:3F16H         LINE#         328
  C:3F16H         LINE#         329
  C:3F16H         LINE#         330
  C:3F16H         LINE#         331
  C:3F19H         LINE#         332
  C:3F1EH         LINE#         333
  C:3F1EH         LINE#         334
  C:3F21H         LINE#         335
  C:3F2BH         LINE#         336
  C:3F2BH         LINE#         337
  C:3F35H         LINE#         338
  C:3F37H         LINE#         340
  C:3F37H         LINE#         341
  C:3F37H         LINE#         342
  C:3F37H         LINE#         343
  C:3F39H         LINE#         344
  C:3F39H         LINE#         346
  C:3F3BH         LINE#         347
  -------         ENDPROC       _TWIREAD
  -------         PROC          TWIINIT
BL51 BANKED LINKER/LOCATER V6.22                                                      02/06/2025  15:28:46  PAGE 101


  C:7DABH         LINE#         367
  C:7DABH         LINE#         368
  C:7DABH         LINE#         369
  C:7DAEH         LINE#         370
  C:7DB1H         LINE#         371
  C:7DB3H         LINE#         372
  C:7DB6H         LINE#         373
  C:7DB9H         LINE#         397
  C:7DBCH         LINE#         398
  C:7DBFH         LINE#         399
  C:7DC1H         LINE#         400
  -------         ENDPROC       TWIINIT
  -------         ENDMOD        TWI

  -------         MODULE        UART
  C:0000H         SYMBOL        _ICE_DUMMY_
  D:0080H         PUBLIC        P0
  D:0090H         PUBLIC        P1
  D:00A0H         PUBLIC        P2
  D:00B0H         PUBLIC        P3
  D:00C4H         PUBLIC        UART0CR
  D:00C0H         PUBLIC        P4
  C:6980H         PUBLIC        UART0Init
  D:009DH         PUBLIC        SBRTH
  D:0080H         PUBLIC        P5
  D:009CH         PUBLIC        SBRTL
  B:0098H.0       PUBLIC        RI
  B:0098H.1       PUBLIC        TI
  D:0099H         PUBLIC        SBUF
  D:0087H         PUBLIC        PCON
  D:0098H         PUBLIC        SCON
  C:7CB2H         PUBLIC        InterruptUART0
  D:0086H         PUBLIC        INSCON
  D:009BH         PUBLIC        SADEN
  D:009AH         PUBLIC        SADDR
  D:009EH         PUBLIC        SFINE
  -------         PROC          UART0INIT
  -------         DO            
  X:02B7H         SYMBOL        TempVal
  -------         ENDDO         
  C:6980H         LINE#         19
  C:6980H         LINE#         20
  C:6980H         LINE#         22
  C:6983H         LINE#         84
  C:6983H         LINE#         86
  C:6986H         LINE#         87
  C:6989H         LINE#         92
  C:6993H         LINE#         93
  C:6999H         LINE#         94
  C:699CH         LINE#         95
  C:69D7H         LINE#         97
  C:69DAH         LINE#         98
  C:69DDH         LINE#         99
  C:69E0H         LINE#         100
  C:69E0H         LINE#         101
  -------         ENDPROC       UART0INIT
  -------         PROC          INTERRUPTUART0
BL51 BANKED LINKER/LOCATER V6.22                                                      02/06/2025  15:28:46  PAGE 102


  -------         DO            
  X:02B6H         SYMBOL        RxData
  -------         ENDDO         
  C:7CB2H         LINE#         110
  C:7CB8H         LINE#         114
  C:7CBAH         LINE#         115
  C:7CBDH         LINE#         117
  C:7CC0H         LINE#         118
  C:7CC0H         LINE#         119
  C:7CC2H         LINE#         120
  C:7CC8H         LINE#         122
  C:7CC8H         LINE#         124
  C:7CC8H         LINE#         125
  C:7CC8H         LINE#         129
  C:7CC8H         LINE#         131
  C:7CCAH         LINE#         132
  -------         ENDPROC       INTERRUPTUART0
  -------         ENDMOD        UART

  -------         MODULE        THERMISTOR
  C:0000H         SYMBOL        _ICE_DUMMY_
  D:0080H         PUBLIC        P0
  D:0090H         PUBLIC        P1
  D:00A0H         PUBLIC        P2
  D:00B0H         PUBLIC        P3
  D:00C0H         PUBLIC        P4
  D:0080H         PUBLIC        P5
  C:4A89H         PUBLIC        NTC103AT
  -------         ENDMOD        THERMISTOR

  -------         MODULE        TWIIO
  C:0000H         SYMBOL        _ICE_DUMMY_
  D:0080H         PUBLIC        P0
  D:0090H         PUBLIC        P1
  D:00A0H         PUBLIC        P2
  D:00B0H         PUBLIC        P3
  D:00C0H         PUBLIC        P4
  D:0080H         PUBLIC        P5
  -------         ENDMOD        TWIIO

  -------         MODULE        ?C_STARTUP
  C:7C73H         SEGMENT       ?C_C51STARTUP
  C:1000H         PUBLIC        ?C_STARTUP
  N:00B2H         SYMBOL        CLKCON
  D:0083H         SYMBOL        DPH
  D:0082H         SYMBOL        DPL
  C:7C79H         SYMBOL        FOR_EACH_IDATA
  C:7C83H         SYMBOL        FOR_EACH_XDATA
  D:0081H         SYMBOL        SP
  C:7C73H         SYMBOL        STARTUP1
  C:1000H         LINE#         12
  C:7C73H         LINE#         18
  C:7C76H         LINE#         19
  C:7C77H         LINE#         22
  C:7C79H         LINE#         24
  C:7C7BH         LINE#         25
  C:7C7CH         LINE#         26
BL51 BANKED LINKER/LOCATER V6.22                                                      02/06/2025  15:28:46  PAGE 103


  C:7C7FH         LINE#         28
  C:7C80H         LINE#         29
  C:7C83H         LINE#         31
  C:7C84H         LINE#         32
  C:7C85H         LINE#         33
  C:7C87H         LINE#         34
  C:7C89H         LINE#         35
  C:7C8CH         LINE#         36
  C:7C8FH         LINE#         37
  C:7C90H         LINE#         38
  -------         ENDMOD        ?C_STARTUP

  -------         MODULE        GASGAUGEINTER_V4_13
  C:0000H         SYMBOL        _ICE_DUMMY_
  D:0080H         PUBLIC        P0
  D:0090H         PUBLIC        P1
  X:0323H         PUBLIC        E2uiDsgCorrectVol
  D:00A0H         PUBLIC        P2
  D:00B0H         PUBLIC        P3
  D:00C0H         PUBLIC        P4
  D:0080H         PUBLIC        P5
  B:00A8H.7       PUBLIC        EA
  X:0325H         PUBLIC        Info_uiRSOC
  X:0327H         PUBLIC        E2ulIdleSocTimes
  X:032BH         PUBLIC        Info_uiRsocCnt
  X:032DH         PUBLIC        E2ulChgerEndVol
  X:0331H         PUBLIC        E2ucChgCurRatio
  X:0332H         PUBLIC        Info_uiSocDecTime
  X:0334H         PUBLIC        Info_ulTempDsgFcc
  X:0338H         PUBLIC        E2ui_CYCLECOUNTA_B
  X:033AH         PUBLIC        E2ui_CYCLECOUNTB_B
  X:033CH         PUBLIC        E2uiTempFCC_K1
  X:033EH         PUBLIC        E2uiTempFCC_K2
  X:0340H         PUBLIC        E2uiChgEndTemp
  X:0342H         PUBLIC        E2ucFccUpdatePercent
  X:0343H         PUBLIC        Info_ulFCC
  X:0347H         PUBLIC        E2ui_CYCLECOUNTA_K
  X:0349H         PUBLIC        E2ui_CYCLECOUNTB_K
  X:034BH         PUBLIC        E2ucChgCorrectSOC
  X:034CH         PUBLIC        E2ucInitSocDif
  X:034DH         PUBLIC        Info_ulVoltage
  X:0351H         PUBLIC        E2uiDsgEndTemp
  X:0353H         PUBLIC        E2ulLoadEndVol
  X:0357H         PUBLIC        E2ucDsgCorrectSOC
  X:0358H         PUBLIC        Info_ulDfilterRC
  X:035CH         PUBLIC        E2uiUpdateCycleCount
  X:035EH         PUBLIC        E2ucDsgVolDet
  D:001AH         PUBLIC        uiCellVminG
  X:035FH         PUBLIC        slAdcCur2
  D:001CH         PUBLIC        uiCellVmaxG
  X:0363H         PUBLIC        E2ucChgerEndDelay
  X:0364H         PUBLIC        Info_uiCycleCount
  X:0366H         PUBLIC        E2slDsgAdjMaxCurr
  X:036AH         PUBLIC        E2ucDsgAdjLowFlg
  X:036BH         PUBLIC        E2ucInitUpSoc
  X:036CH         PUBLIC        E2uiDsgAdjLowTemp
  X:036EH         PUBLIC        E2ucChgChangeSocRatio
BL51 BANKED LINKER/LOCATER V6.22                                                      02/06/2025  15:28:46  PAGE 104


  X:036FH         PUBLIC        E2ucDsgAdjLowSoc
  X:0370H         PUBLIC        E2uiTempFCC_B
  X:0372H         PUBLIC        siCurCompens
  X:0374H         PUBLIC        Info_uiTemp
  X:0376H         PUBLIC        Info_ulRC
  X:037AH         PUBLIC        E2ucChgChangeSocDif
  C:39FCH         PUBLIC        GasGaugeVarIn
  X:037BH         PUBLIC        Info_slCurr
  C:6E78H         PUBLIC        GasGaugeVarOut
  X:037FH         PUBLIC        E2uiChgCorrectVol
  X:0381H         PUBLIC        E2ui_CYCLECOUNTA
  X:0383H         PUBLIC        E2ui_CYCLECOUNTB
  X:0385H         PUBLIC        E2ui_CYCLECOUNTC
  X:0387H         PUBLIC        E2ucChgAdjRatio
  X:0388H         PUBLIC        E2ucChg100Ratio
  X:0389H         PUBLIC        E2ucFullDsgDelay
  -------         PROC          GASGAUGEVARIN
  -------         DO            
  B:0029H.5       SYMBOL        eabak
  -------         ENDDO         
  C:39FCH         LINE#         114
  C:39FCH         LINE#         115
  C:39FCH         LINE#         118
  C:3A00H         LINE#         119
  C:3A02H         LINE#         120
  C:3A11H         LINE#         121
  C:3A1DH         LINE#         122
  C:3A29H         LINE#         123
  C:3A38H         LINE#         124
  C:3A44H         LINE#         125
  C:3A53H         LINE#         126
  C:3A64H         LINE#         127
  C:3A6AH         LINE#         128
  C:3A70H         LINE#         130
  C:3A7AH         LINE#         131
  C:3A81H         LINE#         133
  C:3A85H         LINE#         135
  C:3A8BH         LINE#         136
  C:3A91H         LINE#         137
  C:3A99H         LINE#         138
  C:3AA3H         LINE#         139
  C:3AA8H         LINE#         140
  C:3AADH         LINE#         141
  C:3AB3H         LINE#         142
  C:3ABDH         LINE#         143
  C:3AC4H         LINE#         144
  C:3ACEH         LINE#         145
  C:3AD4H         LINE#         146
  C:3AE8H         LINE#         147
  C:3AEEH         LINE#         148
  C:3AF4H         LINE#         150
  C:3B03H         LINE#         151
  C:3B09H         LINE#         152
  C:3B21H         LINE#         153
  C:3B35H         LINE#         154
  C:3B3BH         LINE#         155
  C:3B41H         LINE#         157
BL51 BANKED LINKER/LOCATER V6.22                                                      02/06/2025  15:28:46  PAGE 105


  C:3B47H         LINE#         158
  C:3B4DH         LINE#         159
  C:3B53H         LINE#         161
  C:3B5DH         LINE#         163
  C:3B63H         LINE#         164
  C:3B6DH         LINE#         165
  C:3B77H         LINE#         167
  C:3B80H         LINE#         168
  C:3B89H         LINE#         169
  C:3B92H         LINE#         170
  C:3B9BH         LINE#         171
  C:3BA4H         LINE#         172
  C:3BADH         LINE#         173
  C:3BB7H         LINE#         174
  C:3BC0H         LINE#         203
  -------         ENDPROC       GASGAUGEVARIN
  -------         PROC          GASGAUGEVAROUT
  -------         DO            
  B:0029H.5       SYMBOL        eabak
  -------         ENDDO         
  C:6E78H         LINE#         211
  C:6E78H         LINE#         212
  C:6E78H         LINE#         215
  C:6E7CH         LINE#         216
  C:6E7EH         LINE#         217
  C:6E8DH         LINE#         218
  C:6E99H         LINE#         219
  C:6EA5H         LINE#         220
  C:6EB4H         LINE#         221
  C:6EB8H         LINE#         222
  C:6EBCH         LINE#         223
  C:6EC4H         LINE#         224
  C:6EC8H         LINE#         252
  -------         ENDPROC       GASGAUGEVAROUT
  -------         ENDMOD        GASGAUGEINTER_V4_13

  -------         MODULE        BOOTAPP
  C:0000H         SYMBOL        _ICE_DUMMY_
  D:0080H         PUBLIC        P0
  D:0090H         PUBLIC        P1
  D:00A0H         PUBLIC        P2
  D:00B0H         PUBLIC        P3
  D:00C0H         PUBLIC        P4
  D:0080H         PUBLIC        P5
  B:00A8H.7       PUBLIC        EA
  C:7D29H         PUBLIC        ISPProcess
  -------         PROC          ISPPROCESS
  C:7D29H         LINE#         17
  C:7D29H         LINE#         18
  C:7D29H         LINE#         19
  C:7D35H         LINE#         20
  C:7D35H         LINE#         21
  C:7D37H         LINE#         22
  C:7D39H         LINE#         23
  C:7D3BH         LINE#         24
  C:7D3DH         LINE#         25
  C:7D3FH         LINE#         26
BL51 BANKED LINKER/LOCATER V6.22                                                      02/06/2025  15:28:46  PAGE 106


  C:7D42H         LINE#         27
  C:7D45H         LINE#         28
  C:7D45H         LINE#         29
  -------         ENDPROC       ISPPROCESS
  -------         ENDMOD        BOOTAPP

  -------         MODULE        BOOTIAP
  C:0000H         SYMBOL        _ICE_DUMMY_
  D:0080H         PUBLIC        P0
  D:0090H         PUBLIC        P1
  D:00A0H         PUBLIC        P2
  D:00B0H         PUBLIC        P3
  D:00C0H         PUBLIC        P4
  D:0080H         PUBLIC        P5
  C:0000H         PUBLIC        g_loadercode
  -------         ENDMOD        BOOTIAP

  -------         MODULE        ?C?FPADD
  C:1C81H         PUBLIC        ?C?FPADD
  C:1C7DH         PUBLIC        ?C?FPSUB
  -------         ENDMOD        ?C?FPADD

  -------         MODULE        ?C?FPMUL
  C:1D72H         PUBLIC        ?C?FPMUL
  -------         ENDMOD        ?C?FPMUL

  -------         MODULE        ?C?FPDIV
  C:1E7BH         PUBLIC        ?C?FPDIV
  -------         ENDMOD        ?C?FPDIV

  -------         MODULE        ?C?FCAST
  C:1F22H         PUBLIC        ?C?FCASTC
  C:1F1DH         PUBLIC        ?C?FCASTI
  C:1F18H         PUBLIC        ?C?FCASTL
  -------         ENDMOD        ?C?FCAST

  -------         MODULE        ?C?CASTF
  C:1F56H         PUBLIC        ?C?CASTF
  -------         ENDMOD        ?C?CASTF

  -------         MODULE        PRINTF
  X:02B7H         PUBLIC        ?_PRINTF?BYTE
  X:02B7H         PUBLIC        ?_SPRINTF?BYTE
  C:2C8EH         PUBLIC        _PRINTF
  C:2C88H         PUBLIC        _SPRINTF
  -------         ENDMOD        PRINTF

  -------         MODULE        ?C?FPROUND
  C:1FD7H         PUBLIC        ?C?FPROUND
  -------         ENDMOD        ?C?FPROUND

  -------         MODULE        ?C?FPCONVERT
  C:2014H         PUBLIC        ?C?FPCONVERT
  -------         ENDMOD        ?C?FPCONVERT

  -------         MODULE        ?C?FTNPWR
  C:2149H         PUBLIC        ?C?FTNPWR
BL51 BANKED LINKER/LOCATER V6.22                                                      02/06/2025  15:28:46  PAGE 107


  -------         ENDMOD        ?C?FTNPWR

  -------         MODULE        ?C?CLDPTR
  C:2189H         PUBLIC        ?C?CLDPTR
  -------         ENDMOD        ?C?CLDPTR

  -------         MODULE        ?C?CLDOPTR
  C:21A2H         PUBLIC        ?C?CLDOPTR
  -------         ENDMOD        ?C?CLDOPTR

  -------         MODULE        ?C?CSTPTR
  C:21CFH         PUBLIC        ?C?CSTPTR
  -------         ENDMOD        ?C?CSTPTR

  -------         MODULE        ?C?IMUL
  C:21E1H         PUBLIC        ?C?IMUL
  -------         ENDMOD        ?C?IMUL

  -------         MODULE        ?C?UIDIV
  C:21F3H         PUBLIC        ?C?UIDIV
  -------         ENDMOD        ?C?UIDIV

  -------         MODULE        ?C?IILDX
  C:2248H         PUBLIC        ?C?IILDX
  -------         ENDMOD        ?C?IILDX

  -------         MODULE        ?C?LADD
  C:225EH         PUBLIC        ?C?LADD
  -------         ENDMOD        ?C?LADD

  -------         MODULE        ?C?LSUB
  C:226BH         PUBLIC        ?C?LSUB
  -------         ENDMOD        ?C?LSUB

  -------         MODULE        ?C?LMUL
  C:2279H         PUBLIC        ?C?LMUL
  -------         ENDMOD        ?C?LMUL

  -------         MODULE        ?C?ULDIV
  C:2304H         PUBLIC        ?C?ULDIV
  -------         ENDMOD        ?C?ULDIV

  -------         MODULE        ?C?SLDIV
  C:7602H         PUBLIC        ?C?SLDIV
  -------         ENDMOD        ?C?SLDIV

  -------         MODULE        ?C?LOR
  C:2396H         PUBLIC        ?C?LOR
  -------         ENDMOD        ?C?LOR

  -------         MODULE        ?C?LNEG
  C:23A3H         PUBLIC        ?C?LNEG
  -------         ENDMOD        ?C?LNEG

  -------         MODULE        ?C?SLCMP
  C:23B1H         PUBLIC        ?C?SLCMP
  -------         ENDMOD        ?C?SLCMP
BL51 BANKED LINKER/LOCATER V6.22                                                      02/06/2025  15:28:46  PAGE 108



  -------         MODULE        ?C?ULCMP
  C:23C7H         PUBLIC        ?C?ULCMP
  -------         ENDMOD        ?C?ULCMP

  -------         MODULE        ?C?ULSHR
  C:23D8H         PUBLIC        ?C?ULSHR
  -------         ENDMOD        ?C?ULSHR

  -------         MODULE        ?C?SLSHR
  C:23EBH         PUBLIC        ?C?SLSHR
  -------         ENDMOD        ?C?SLSHR

  -------         MODULE        ?C?LSHL
  C:23FFH         PUBLIC        ?C?LSHL
  -------         ENDMOD        ?C?LSHL

  -------         MODULE        ?C?LLDIDATA
  C:2412H         PUBLIC        ?C?LLDIDATA
  -------         ENDMOD        ?C?LLDIDATA

  -------         MODULE        ?C?LLDXDATA
  C:241EH         PUBLIC        ?C?LLDXDATA
  -------         ENDMOD        ?C?LLDXDATA

  -------         MODULE        ?C?LLDIDATA0
  C:242AH         PUBLIC        ?C?LLDIDATA0
  -------         ENDMOD        ?C?LLDIDATA0

  -------         MODULE        ?C?LLDXDATA0
  C:2437H         PUBLIC        ?C?LLDXDATA0
  -------         ENDMOD        ?C?LLDXDATA0

  -------         MODULE        ?C?LILDXDATA
  C:244CH         PUBLIC        ?C?LILDXDATA
  C:2443H         PUBLIC        ?C?LILDXDATA1
  C:2445H         PUBLIC        ?C?LILDXDATA8
  -------         ENDMOD        ?C?LILDXDATA

  -------         MODULE        ?C?LSTIDATA
  C:2478H         PUBLIC        ?C?LSTIDATA
  -------         ENDMOD        ?C?LSTIDATA

  -------         MODULE        ?C?LSTXDATA
  C:2484H         PUBLIC        ?C?LSTXDATA
  -------         ENDMOD        ?C?LSTXDATA

  -------         MODULE        ?C?LSTKIDATA
  C:2490H         PUBLIC        ?C?LSTKIDATA
  -------         ENDMOD        ?C?LSTKIDATA

  -------         MODULE        ?C?LSTKXDATA
  C:24A9H         PUBLIC        ?C?LSTKXDATA
  -------         ENDMOD        ?C?LSTKXDATA

  -------         MODULE        ?C?OFFXADD
  C:24DAH         PUBLIC        ?C?OFFXADD
BL51 BANKED LINKER/LOCATER V6.22                                                      02/06/2025  15:28:46  PAGE 109


  -------         ENDMOD        ?C?OFFXADD

  -------         MODULE        ?C?PLDIXDATA
  C:24E6H         PUBLIC        ?C?PLDIXDATA
  -------         ENDMOD        ?C?PLDIXDATA

  -------         MODULE        ?C?PSTXDATA
  C:24FDH         PUBLIC        ?C?PSTXDATA
  -------         ENDMOD        ?C?PSTXDATA

  -------         MODULE        ?C?CCASE
  C:2506H         PUBLIC        ?C?CCASE
  -------         ENDMOD        ?C?CCASE

  -------         MODULE        ?C?LIMUL
  C:252CH         PUBLIC        ?C?LIMUL
  -------         ENDMOD        ?C?LIMUL



FUNCTION REGISTER MASKS


FUNCTION . . . . . . . . . REG MASK
-----------------------------------

AFEADCDIS. . . . . . . . . @0xf7ff
AFEADCEN . . . . . . . . . @0xf7ff
AFECADCDIS . . . . . . . . @0xf7ff
AFECADCEN. . . . . . . . . @0xf7ff
AFECHGERCHECKDIS . . . . . @0xf7ff
AFECHGERCHECKEN. . . . . . @0xf7ff
AFECLRFLG. . . . . . . . . @0xf7ff
AFEENTERPD . . . . . . . . @0xf7ff
AFEGETTEMPE. . . . . . . . @0xf7ff
AFEGETVOL. . . . . . . . . @0xf7ff
AFEINIT. . . . . . . . . . @0xf7ff
AFELOADCHECKDIS. . . . . . @0xf7ff
AFELOADCHECKEN . . . . . . @0xf7ff
AFERAMCHECK. . . . . . . . @0xf7ff
AFERDFLG . . . . . . . . . @0xf7ff
AFERDSTATUS. . . . . . . . @0xf7ff
AFETEMPADCDIS. . . . . . . @0xf7ff
AFETEMPADCEN . . . . . . . @0xf7ff
AFETWICHECK. . . . . . . . @0xf300
AFEWDTDIS. . . . . . . . . @0xf7ff
AFEWDTEN . . . . . . . . . @0xf7ff
BALPROCESS . . . . . . . . @0xf7ff
CALICURZERO. . . . . . . . @0xe301
CALIRTCTIME. . . . . . . . @0xf7ff
CHGERCHECK . . . . . . . . @0xf7ff
CTOCHECKVOL. . . . . . . . @0xf300
CTOTURNONCHECK . . . . . . @0xf300
E2PROMBKBOOT . . . . . . . @0xf7ff
E2PROMINIT . . . . . . . . @0xf7ff
E2PROMTWICHECK . . . . . . @0xf300
GASGAUGEVARIN. . . . . . . @0xffbf
BL51 BANKED LINKER/LOCATER V6.22                                                      02/06/2025  15:28:46  PAGE 110


GASGAUGEVAROUT . . . . . . @0xff8f
INITGPIO . . . . . . . . . @0xc000
INITIRQ. . . . . . . . . . @0xe000
INITVAR. . . . . . . . . . @0xf797
INTERRUPTINT4. . . . . . . @0xf301
INTERRUPTTIMER3. . . . . . @0xf300
INTERRUPTTIMER3APP . . . . @0xf300
INTERRUPTUART0 . . . . . . @0xe300
INTERRUPTUART0APPTX. . . . @0xf38f
KEYSCAN. . . . . . . . . . @0xf000
LEDAUTOOFF . . . . . . . . @0xf300
LEDDISPLAY . . . . . . . . @0xf303
LOADCHECK. . . . . . . . . @0xf7ff
LOWPOWERCHECK. . . . . . . @0xf301
LOWPOWERPROCESS. . . . . . @0xf7ff
MCUFLASHPROCESS. . . . . . @0xf7bf
MCUFLASHWRWAITCHECK. . . . @0xf300
MCUINTOIDLE. . . . . . . . @0xc000
MCUINTOPD. . . . . . . . . @0xc000
MOSCTRL. . . . . . . . . . @0xf7ff
MOSSTATUSCHECK . . . . . . @0xc000
PORPROTECTOTC. . . . . . . @0xf78f
PORPROTECTOTD. . . . . . . @0xf78f
PORPROTECTOV . . . . . . . @0xf782
PORPROTECTUTC. . . . . . . @0xf78f
PORPROTECTUTD. . . . . . . @0xf78f
PORPROTECTUV . . . . . . . @0xf782
PROTECTOCRECOVER . . . . . @0xf7ff
PROTECTOTC . . . . . . . . @0xf7af
PROTECTOTD . . . . . . . . @0xf7af
PROTECTOV. . . . . . . . . @0xf7ff
PROTECTUTC . . . . . . . . @0xf7af
PROTECTUTD . . . . . . . . @0xf7af
PROTECTUV. . . . . . . . . @0xf78b
RAMCHECKPROCESS. . . . . . @0xf300
RTCTWICHECK. . . . . . . . @0xf300
SYSPARAINIT. . . . . . . . @0xffbf
SYSTEMINTOPD . . . . . . . @0xf7ff
SYSTEMINTOSLEEP. . . . . . @0xf7ff
TWIINIT. . . . . . . . . . @0xe000
UART0CALICUROFFSET . . . . @0xf375
UART0CALIRTC . . . . . . . @0xf377
UART0CALITS1 . . . . . . . @0xf377
UART0CALITS2 . . . . . . . @0xf377
UART0CALIVOLTAGE . . . . . @0xf377
UART0CHECK . . . . . . . . @0xf300
UART0HANDSHAKE . . . . . . @0xe300
UART0IAPCHECKHANDSHAKE . . @0xf7bf
UART0RDCMDPROCESS. . . . . @0xf3ff
UART0RDE2PROM. . . . . . . @0xf7ff
UART0READSUBCLASSID. . . . @0xf375
UART0WRITEMANUFACTURE. . . @0xf375
UART1RDE2PROM. . . . . . . @0xf7ff
UART2RDE2PROM. . . . . . . @0xf7ff
WAKEUPPROCESS. . . . . . . @0xf7ff
_AFEALARMDIS . . . . . . . @0xf7ff
_AFEALARMEN. . . . . . . . @0xf7ff
BL51 BANKED LINKER/LOCATER V6.22                                                      02/06/2025  15:28:46  PAGE 111


_AFEBALCTL . . . . . . . . @0xf7ff
_AFEMOSCTL . . . . . . . . @0xf7ff
_AFEREADREG. . . . . . . . @0xf7ff
_AFEWRITEREG . . . . . . . @0xf7ff
_CRC8CAL . . . . . . . . . @0xf365
_DELAY1MS. . . . . . . . . @0xf03e
_E2PROMREAD. . . . . . . . @0xf7ff
_E2PROMWRITE . . . . . . . @0xf7ff
_GETCYCLEGAIN. . . . . . . @0xf7cf
_INTERRUPTINT4APP. . . . . @0xf301
_LEDGETDISNUM. . . . . . . @0xf001
_MCUCLOCKSET . . . . . . . @0xf301
_MCUFLASHBLANKCHECK. . . . @0xf31c
_MCUFLASHCHECKFLG. . . . . @0xf303
_MCUFLASHDATACHECK . . . . @0xf7af
_MCUFLASHREAD. . . . . . . @0xf307
_MCUFLASHWRITE . . . . . . @0xf7bf
_MCUFLASHWRONEBYTE . . . . @0xf035
_MCUFLASHWRSECTOR. . . . . @0xf33f
_MEMORYCOPY. . . . . . . . @0xf78d
_MEMORYSET . . . . . . . . @0xf781
_PUTCHAR . . . . . . . . . @0xc000
_RTCMODIFYTIME . . . . . . @0xf7ff
_RTCREAD . . . . . . . . . @0xf7ff
_RTCWRITE. . . . . . . . . @0xf7ff
_TWICHECKSTATUS. . . . . . @0xf00c
_TWIREAD . . . . . . . . . @0xf7ff
_TWIWRITE. . . . . . . . . @0xf7ff
_UART0READINFO . . . . . . @0xf37f
_UART0WRITEINFO. . . . . . @0xf7ff

*** WARNING L15: MULTIPLE CALL TO SEGMENT
    SEGMENT: ?PR?_MCUCLOCKSET?MCULIB
    CALLER1: ?PR?INTERRUPTINT4?INTERRUPT
    CALLER2: ?C_C51STARTUP

Program Size: data=154.7 xdata=1534 code=32641
LINK/LOCATE RUN COMPLETE.  1 WARNING(S),  0 ERROR(S)
